Archive member included to satisfy reference by file (symbol)

/usr/lib/gcc/arm-none-eabi/9.2.1/../../../arm-none-eabi/lib/thumb/v7e-m/nofp/libm.a(lib_a-s_ceil.o)
                              /home/ch/RIOT/examples/lorawan/bin/lora-e5-dev/semtech_loramac_mac_region/RegionCommon.o (ceil)
/usr/lib/gcc/arm-none-eabi/9.2.1/../../../arm-none-eabi/lib/thumb/v7e-m/nofp/libm.a(lib_a-s_floor.o)
                              /home/ch/RIOT/examples/lorawan/bin/lora-e5-dev/semtech_loramac_mac_region/RegionCommon.o (floor)
/usr/lib/gcc/arm-none-eabi/9.2.1/thumb/v7e-m/nofp/libgcc.a(_arm_muldf3.o)
                              /home/ch/RIOT/examples/lorawan/bin/lora-e5-dev/semtech_loramac_mac_region/RegionCommon.o (__aeabi_dmul)
/usr/lib/gcc/arm-none-eabi/9.2.1/thumb/v7e-m/nofp/libgcc.a(_arm_mulsf3.o)
                              /home/ch/RIOT/examples/lorawan/bin/lora-e5-dev/fmt/fmt.o (__aeabi_fmul)
/usr/lib/gcc/arm-none-eabi/9.2.1/thumb/v7e-m/nofp/libgcc.a(_arm_addsubdf3.o)
                              /home/ch/RIOT/examples/lorawan/bin/lora-e5-dev/semtech_loramac_mac_region/RegionCommon.o (__aeabi_dsub)
/usr/lib/gcc/arm-none-eabi/9.2.1/thumb/v7e-m/nofp/libgcc.a(_arm_muldivdf3.o)
                              /home/ch/RIOT/examples/lorawan/bin/lora-e5-dev/semtech_loramac_mac_region/RegionCommon.o (__aeabi_ddiv)
/usr/lib/gcc/arm-none-eabi/9.2.1/thumb/v7e-m/nofp/libgcc.a(_arm_cmpdf2.o)
                              /usr/lib/gcc/arm-none-eabi/9.2.1/../../../arm-none-eabi/lib/thumb/v7e-m/nofp/libm.a(lib_a-s_ceil.o) (__aeabi_dcmpgt)
/usr/lib/gcc/arm-none-eabi/9.2.1/thumb/v7e-m/nofp/libgcc.a(_arm_fixdfsi.o)
                              /home/ch/RIOT/examples/lorawan/bin/lora-e5-dev/semtech_loramac_mac_region/RegionCommon.o (__aeabi_d2iz)
/usr/lib/gcc/arm-none-eabi/9.2.1/thumb/v7e-m/nofp/libgcc.a(_arm_fixunsdfsi.o)
                              /home/ch/RIOT/examples/lorawan/bin/lora-e5-dev/semtech_loramac_mac_region/RegionCommon.o (__aeabi_d2uiz)
/usr/lib/gcc/arm-none-eabi/9.2.1/thumb/v7e-m/nofp/libgcc.a(_arm_addsubsf3.o)
                              /home/ch/RIOT/examples/lorawan/bin/lora-e5-dev/fmt/fmt.o (__aeabi_fsub)
/usr/lib/gcc/arm-none-eabi/9.2.1/thumb/v7e-m/nofp/libgcc.a(_arm_cmpsf2.o)
                              /home/ch/RIOT/examples/lorawan/bin/lora-e5-dev/fmt/fmt.o (__aeabi_fcmplt)
/usr/lib/gcc/arm-none-eabi/9.2.1/thumb/v7e-m/nofp/libgcc.a(_arm_fixunssfsi.o)
                              /home/ch/RIOT/examples/lorawan/bin/lora-e5-dev/fmt/fmt.o (__aeabi_f2uiz)
/usr/lib/gcc/arm-none-eabi/9.2.1/../../../arm-none-eabi/lib/thumb/v7e-m/nofp/libc_nano.a(lib_a-errno.o)
                              /home/ch/RIOT/examples/lorawan/bin/lora-e5-dev/newlib_syscalls_default/syscalls.o (__errno)
/usr/lib/gcc/arm-none-eabi/9.2.1/../../../arm-none-eabi/lib/thumb/v7e-m/nofp/libc_nano.a(lib_a-impure.o)
                              /usr/lib/gcc/arm-none-eabi/9.2.1/../../../arm-none-eabi/lib/thumb/v7e-m/nofp/libc_nano.a(lib_a-errno.o) (_impure_ptr)
/usr/lib/gcc/arm-none-eabi/9.2.1/../../../arm-none-eabi/lib/thumb/v7e-m/nofp/libc_nano.a(lib_a-init.o)
                              /home/ch/RIOT/examples/lorawan/bin/lora-e5-dev/cortexm_common/vectors_cortexm.o (__libc_init_array)
/usr/lib/gcc/arm-none-eabi/9.2.1/../../../arm-none-eabi/lib/thumb/v7e-m/nofp/libc_nano.a(lib_a-malloc.o)
                              /home/ch/RIOT/examples/lorawan/bin/lora-e5-dev/malloc_thread_safe/malloc_wrappers.o (malloc)
/usr/lib/gcc/arm-none-eabi/9.2.1/../../../arm-none-eabi/lib/thumb/v7e-m/nofp/libc_nano.a(lib_a-memcmp.o)
                              /home/ch/RIOT/examples/lorawan/bin/lora-e5-dev/core/atomic_c11.o (memcmp)
/usr/lib/gcc/arm-none-eabi/9.2.1/../../../arm-none-eabi/lib/thumb/v7e-m/nofp/libc_nano.a(lib_a-memcpy.o)
                              /home/ch/RIOT/examples/lorawan/bin/lora-e5-dev/core/atomic_c11.o (memcpy)
/usr/lib/gcc/arm-none-eabi/9.2.1/../../../arm-none-eabi/lib/thumb/v7e-m/nofp/libc_nano.a(lib_a-memmove.o)
                              /home/ch/RIOT/examples/lorawan/bin/lora-e5-dev/fmt/fmt.o (memmove)
/usr/lib/gcc/arm-none-eabi/9.2.1/../../../arm-none-eabi/lib/thumb/v7e-m/nofp/libc_nano.a(lib_a-memset.o)
                              /home/ch/RIOT/examples/lorawan/bin/lora-e5-dev/crypto/chacha20poly1305.o (memset)
/usr/lib/gcc/arm-none-eabi/9.2.1/../../../arm-none-eabi/lib/thumb/v7e-m/nofp/libc_nano.a(lib_a-mstats.o)
                              /home/ch/RIOT/examples/lorawan/bin/lora-e5-dev/newlib_syscalls_default/syscalls.o (mallinfo)
/usr/lib/gcc/arm-none-eabi/9.2.1/../../../arm-none-eabi/lib/thumb/v7e-m/nofp/libc_nano.a(lib_a-nano-freer.o)
                              /usr/lib/gcc/arm-none-eabi/9.2.1/../../../arm-none-eabi/lib/thumb/v7e-m/nofp/libc_nano.a(lib_a-malloc.o) (_free_r)
/usr/lib/gcc/arm-none-eabi/9.2.1/../../../arm-none-eabi/lib/thumb/v7e-m/nofp/libc_nano.a(lib_a-nano-mallinfor.o)
                              /usr/lib/gcc/arm-none-eabi/9.2.1/../../../arm-none-eabi/lib/thumb/v7e-m/nofp/libc_nano.a(lib_a-mstats.o) (_mallinfo_r)
/usr/lib/gcc/arm-none-eabi/9.2.1/../../../arm-none-eabi/lib/thumb/v7e-m/nofp/libc_nano.a(lib_a-nano-mallocr.o)
                              /usr/lib/gcc/arm-none-eabi/9.2.1/../../../arm-none-eabi/lib/thumb/v7e-m/nofp/libc_nano.a(lib_a-malloc.o) (_malloc_r)
/usr/lib/gcc/arm-none-eabi/9.2.1/../../../arm-none-eabi/lib/thumb/v7e-m/nofp/libc_nano.a(lib_a-nano-malloptr.o)
                              /usr/lib/gcc/arm-none-eabi/9.2.1/../../../arm-none-eabi/lib/thumb/v7e-m/nofp/libc_nano.a(lib_a-mstats.o) (_mallopt_r)
/usr/lib/gcc/arm-none-eabi/9.2.1/../../../arm-none-eabi/lib/thumb/v7e-m/nofp/libc_nano.a(lib_a-nano-mallstatsr.o)
                              /usr/lib/gcc/arm-none-eabi/9.2.1/../../../arm-none-eabi/lib/thumb/v7e-m/nofp/libc_nano.a(lib_a-mstats.o) (_malloc_stats_r)
/usr/lib/gcc/arm-none-eabi/9.2.1/../../../arm-none-eabi/lib/thumb/v7e-m/nofp/libc_nano.a(lib_a-nano-vfprintf_float.o)
                              (_printf_float)
/usr/lib/gcc/arm-none-eabi/9.2.1/../../../arm-none-eabi/lib/thumb/v7e-m/nofp/libc_nano.a(lib_a-nano-vfprintf_i.o)
                              /usr/lib/gcc/arm-none-eabi/9.2.1/../../../arm-none-eabi/lib/thumb/v7e-m/nofp/libc_nano.a(lib_a-nano-vfprintf_float.o) (_printf_common)
/usr/lib/gcc/arm-none-eabi/9.2.1/../../../arm-none-eabi/lib/thumb/v7e-m/nofp/libc_nano.a(lib_a-printf.o)
                              /home/ch/RIOT/examples/lorawan/bin/lora-e5-dev/application_lorawan/main.o (printf)
/usr/lib/gcc/arm-none-eabi/9.2.1/../../../arm-none-eabi/lib/thumb/v7e-m/nofp/libc_nano.a(lib_a-puts.o)
                              /home/ch/RIOT/examples/lorawan/bin/lora-e5-dev/application_lorawan/main.o (puts)
/usr/lib/gcc/arm-none-eabi/9.2.1/../../../arm-none-eabi/lib/thumb/v7e-m/nofp/libc_nano.a(lib_a-realloc.o)
                              /home/ch/RIOT/examples/lorawan/bin/lora-e5-dev/malloc_thread_safe/malloc_wrappers.o (realloc)
/usr/lib/gcc/arm-none-eabi/9.2.1/../../../arm-none-eabi/lib/thumb/v7e-m/nofp/libc_nano.a(lib_a-strlen.o)
                              /home/ch/RIOT/examples/lorawan/bin/lora-e5-dev/application_lorawan/main.o (strlen)
/usr/lib/gcc/arm-none-eabi/9.2.1/../../../arm-none-eabi/lib/thumb/v7e-m/nofp/libc_nano.a(lib_a-syswrite.o)
                              /home/ch/RIOT/examples/lorawan/bin/lora-e5-dev/fmt/fmt.o (write)
/usr/lib/gcc/arm-none-eabi/9.2.1/../../../arm-none-eabi/lib/thumb/v7e-m/nofp/libc_nano.a(lib_a-wbuf.o)
                              /usr/lib/gcc/arm-none-eabi/9.2.1/../../../arm-none-eabi/lib/thumb/v7e-m/nofp/libc_nano.a(lib_a-puts.o) (__swbuf_r)
/usr/lib/gcc/arm-none-eabi/9.2.1/../../../arm-none-eabi/lib/thumb/v7e-m/nofp/libc_nano.a(lib_a-wsetup.o)
                              /usr/lib/gcc/arm-none-eabi/9.2.1/../../../arm-none-eabi/lib/thumb/v7e-m/nofp/libc_nano.a(lib_a-puts.o) (__swsetup_r)
/usr/lib/gcc/arm-none-eabi/9.2.1/../../../arm-none-eabi/lib/thumb/v7e-m/nofp/libc_nano.a(lib_a-dtoa.o)
                              /usr/lib/gcc/arm-none-eabi/9.2.1/../../../arm-none-eabi/lib/thumb/v7e-m/nofp/libc_nano.a(lib_a-nano-vfprintf_float.o) (_dtoa_r)
/usr/lib/gcc/arm-none-eabi/9.2.1/../../../arm-none-eabi/lib/thumb/v7e-m/nofp/libc_nano.a(lib_a-fflush.o)
                              /usr/lib/gcc/arm-none-eabi/9.2.1/../../../arm-none-eabi/lib/thumb/v7e-m/nofp/libc_nano.a(lib_a-wbuf.o) (_fflush_r)
/usr/lib/gcc/arm-none-eabi/9.2.1/../../../arm-none-eabi/lib/thumb/v7e-m/nofp/libc_nano.a(lib_a-findfp.o)
                              /usr/lib/gcc/arm-none-eabi/9.2.1/../../../arm-none-eabi/lib/thumb/v7e-m/nofp/libc_nano.a(lib_a-mstats.o) (__sinit)
/usr/lib/gcc/arm-none-eabi/9.2.1/../../../arm-none-eabi/lib/thumb/v7e-m/nofp/libc_nano.a(lib_a-fprintf.o)
                              /usr/lib/gcc/arm-none-eabi/9.2.1/../../../arm-none-eabi/lib/thumb/v7e-m/nofp/libc_nano.a(lib_a-mstats.o) (fiprintf)
/usr/lib/gcc/arm-none-eabi/9.2.1/../../../arm-none-eabi/lib/thumb/v7e-m/nofp/libc_nano.a(lib_a-fwalk.o)
                              /usr/lib/gcc/arm-none-eabi/9.2.1/../../../arm-none-eabi/lib/thumb/v7e-m/nofp/libc_nano.a(lib_a-findfp.o) (_fwalk)
/usr/lib/gcc/arm-none-eabi/9.2.1/../../../arm-none-eabi/lib/thumb/v7e-m/nofp/libc_nano.a(lib_a-localeconv.o)
                              /usr/lib/gcc/arm-none-eabi/9.2.1/../../../arm-none-eabi/lib/thumb/v7e-m/nofp/libc_nano.a(lib_a-nano-vfprintf_float.o) (_localeconv_r)
/usr/lib/gcc/arm-none-eabi/9.2.1/../../../arm-none-eabi/lib/thumb/v7e-m/nofp/libc_nano.a(lib_a-makebuf.o)
                              /usr/lib/gcc/arm-none-eabi/9.2.1/../../../arm-none-eabi/lib/thumb/v7e-m/nofp/libc_nano.a(lib_a-wsetup.o) (__smakebuf_r)
/usr/lib/gcc/arm-none-eabi/9.2.1/../../../arm-none-eabi/lib/thumb/v7e-m/nofp/libc_nano.a(lib_a-memchr.o)
                              /usr/lib/gcc/arm-none-eabi/9.2.1/../../../arm-none-eabi/lib/thumb/v7e-m/nofp/libc_nano.a(lib_a-nano-vfprintf_i.o) (memchr)
/usr/lib/gcc/arm-none-eabi/9.2.1/../../../arm-none-eabi/lib/thumb/v7e-m/nofp/libc_nano.a(lib_a-mlock.o)
                              /usr/lib/gcc/arm-none-eabi/9.2.1/../../../arm-none-eabi/lib/thumb/v7e-m/nofp/libc_nano.a(lib_a-nano-freer.o) (__malloc_lock)
/usr/lib/gcc/arm-none-eabi/9.2.1/../../../arm-none-eabi/lib/thumb/v7e-m/nofp/libc_nano.a(lib_a-mprec.o)
                              /usr/lib/gcc/arm-none-eabi/9.2.1/../../../arm-none-eabi/lib/thumb/v7e-m/nofp/libc_nano.a(lib_a-dtoa.o) (_Balloc)
/usr/lib/gcc/arm-none-eabi/9.2.1/../../../arm-none-eabi/lib/thumb/v7e-m/nofp/libc_nano.a(lib_a-nano-callocr.o)
                              /usr/lib/gcc/arm-none-eabi/9.2.1/../../../arm-none-eabi/lib/thumb/v7e-m/nofp/libc_nano.a(lib_a-mprec.o) (_calloc_r)
/usr/lib/gcc/arm-none-eabi/9.2.1/../../../arm-none-eabi/lib/thumb/v7e-m/nofp/libc_nano.a(lib_a-nano-reallocr.o)
                              /usr/lib/gcc/arm-none-eabi/9.2.1/../../../arm-none-eabi/lib/thumb/v7e-m/nofp/libc_nano.a(lib_a-realloc.o) (_realloc_r)
/usr/lib/gcc/arm-none-eabi/9.2.1/../../../arm-none-eabi/lib/thumb/v7e-m/nofp/libc_nano.a(lib_a-nano-vfprintf.o)
                              /usr/lib/gcc/arm-none-eabi/9.2.1/../../../arm-none-eabi/lib/thumb/v7e-m/nofp/libc_nano.a(lib_a-printf.o) (_vfprintf_r)
/usr/lib/gcc/arm-none-eabi/9.2.1/../../../arm-none-eabi/lib/thumb/v7e-m/nofp/libc_nano.a(lib_a-stdio.o)
                              /usr/lib/gcc/arm-none-eabi/9.2.1/../../../arm-none-eabi/lib/thumb/v7e-m/nofp/libc_nano.a(lib_a-findfp.o) (__sread)
/usr/lib/gcc/arm-none-eabi/9.2.1/../../../arm-none-eabi/lib/thumb/v7e-m/nofp/libc_nano.a(lib_a-assert.o)
                              /usr/lib/gcc/arm-none-eabi/9.2.1/../../../arm-none-eabi/lib/thumb/v7e-m/nofp/libc_nano.a(lib_a-dtoa.o) (__assert_func)
/usr/lib/gcc/arm-none-eabi/9.2.1/../../../arm-none-eabi/lib/thumb/v7e-m/nofp/libc_nano.a(lib_a-fvwrite.o)
                              /usr/lib/gcc/arm-none-eabi/9.2.1/../../../arm-none-eabi/lib/thumb/v7e-m/nofp/libc_nano.a(lib_a-nano-vfprintf.o) (__sfvwrite_r)
/usr/lib/gcc/arm-none-eabi/9.2.1/../../../arm-none-eabi/lib/thumb/v7e-m/nofp/libc_nano.a(lib_a-locale.o)
                              /usr/lib/gcc/arm-none-eabi/9.2.1/../../../arm-none-eabi/lib/thumb/v7e-m/nofp/libc_nano.a(lib_a-localeconv.o) (__global_locale)
/usr/lib/gcc/arm-none-eabi/9.2.1/../../../arm-none-eabi/lib/thumb/v7e-m/nofp/libc_nano.a(lib_a-mbtowc_r.o)
                              /usr/lib/gcc/arm-none-eabi/9.2.1/../../../arm-none-eabi/lib/thumb/v7e-m/nofp/libc_nano.a(lib_a-locale.o) (__ascii_mbtowc)
/usr/lib/gcc/arm-none-eabi/9.2.1/../../../arm-none-eabi/lib/thumb/v7e-m/nofp/libc_nano.a(lib_a-nano-msizer.o)
                              /usr/lib/gcc/arm-none-eabi/9.2.1/../../../arm-none-eabi/lib/thumb/v7e-m/nofp/libc_nano.a(lib_a-nano-reallocr.o) (_malloc_usable_size_r)
/usr/lib/gcc/arm-none-eabi/9.2.1/../../../arm-none-eabi/lib/thumb/v7e-m/nofp/libc_nano.a(lib_a-strcmp.o)
                              /usr/lib/gcc/arm-none-eabi/9.2.1/../../../arm-none-eabi/lib/thumb/v7e-m/nofp/libc_nano.a(lib_a-locale.o) (strcmp)
/usr/lib/gcc/arm-none-eabi/9.2.1/../../../arm-none-eabi/lib/thumb/v7e-m/nofp/libc_nano.a(lib_a-wctomb_r.o)
                              /usr/lib/gcc/arm-none-eabi/9.2.1/../../../arm-none-eabi/lib/thumb/v7e-m/nofp/libc_nano.a(lib_a-locale.o) (__ascii_wctomb)
/usr/lib/gcc/arm-none-eabi/9.2.1/../../../arm-none-eabi/lib/thumb/v7e-m/nofp/libc_nano.a(lib_a-abort.o)
                              /usr/lib/gcc/arm-none-eabi/9.2.1/../../../arm-none-eabi/lib/thumb/v7e-m/nofp/libc_nano.a(lib_a-assert.o) (abort)
/usr/lib/gcc/arm-none-eabi/9.2.1/../../../arm-none-eabi/lib/thumb/v7e-m/nofp/libc_nano.a(lib_a-ctype_.o)
                              /usr/lib/gcc/arm-none-eabi/9.2.1/../../../arm-none-eabi/lib/thumb/v7e-m/nofp/libc_nano.a(lib_a-locale.o) (_ctype_)
/usr/lib/gcc/arm-none-eabi/9.2.1/../../../arm-none-eabi/lib/thumb/v7e-m/nofp/libc_nano.a(lib_a-signal.o)
                              /usr/lib/gcc/arm-none-eabi/9.2.1/../../../arm-none-eabi/lib/thumb/v7e-m/nofp/libc_nano.a(lib_a-abort.o) (raise)
/usr/lib/gcc/arm-none-eabi/9.2.1/thumb/v7e-m/nofp/libgcc.a(_arm_unorddf2.o)
                              /usr/lib/gcc/arm-none-eabi/9.2.1/../../../arm-none-eabi/lib/thumb/v7e-m/nofp/libc_nano.a(lib_a-nano-vfprintf_float.o) (__aeabi_dcmpun)

Discarded input sections

 .group         0x0000000000000000        0xc /home/ch/RIOT/examples/lorawan/bin/lora-e5-dev/application_lorawan/main.o
 .group         0x0000000000000000        0xc /home/ch/RIOT/examples/lorawan/bin/lora-e5-dev/application_lorawan/main.o
 .group         0x0000000000000000        0xc /home/ch/RIOT/examples/lorawan/bin/lora-e5-dev/application_lorawan/main.o
 .group         0x0000000000000000        0xc /home/ch/RIOT/examples/lorawan/bin/lora-e5-dev/application_lorawan/main.o
 .group         0x0000000000000000        0xc /home/ch/RIOT/examples/lorawan/bin/lora-e5-dev/application_lorawan/main.o
 .group         0x0000000000000000        0xc /home/ch/RIOT/examples/lorawan/bin/lora-e5-dev/application_lorawan/main.o
 .group         0x0000000000000000        0xc /home/ch/RIOT/examples/lorawan/bin/lora-e5-dev/application_lorawan/main.o
 .group         0x0000000000000000        0xc /home/ch/RIOT/examples/lorawan/bin/lora-e5-dev/application_lorawan/main.o
 .group         0x0000000000000000        0xc /home/ch/RIOT/examples/lorawan/bin/lora-e5-dev/application_lorawan/main.o
 .group         0x0000000000000000        0xc /home/ch/RIOT/examples/lorawan/bin/lora-e5-dev/application_lorawan/main.o
 .group         0x0000000000000000        0xc /home/ch/RIOT/examples/lorawan/bin/lora-e5-dev/application_lorawan/main.o
 .group         0x0000000000000000        0xc /home/ch/RIOT/examples/lorawan/bin/lora-e5-dev/application_lorawan/main.o
 .group         0x0000000000000000        0xc /home/ch/RIOT/examples/lorawan/bin/lora-e5-dev/application_lorawan/main.o
 .group         0x0000000000000000        0xc /home/ch/RIOT/examples/lorawan/bin/lora-e5-dev/application_lorawan/main.o
 .group         0x0000000000000000        0xc /home/ch/RIOT/examples/lorawan/bin/lora-e5-dev/application_lorawan/main.o
 .group         0x0000000000000000        0xc /home/ch/RIOT/examples/lorawan/bin/lora-e5-dev/application_lorawan/main.o
 .group         0x0000000000000000        0xc /home/ch/RIOT/examples/lorawan/bin/lora-e5-dev/application_lorawan/main.o
 .group         0x0000000000000000        0xc /home/ch/RIOT/examples/lorawan/bin/lora-e5-dev/application_lorawan/main.o
Memory Configuration

Name             Origin             Length             Attributes
ccmram           0x0000000010000000 0x0000000000000000
sram4            0x0000000028000000 0x0000000000000000
rom              0x0000000008000000 0x0000000000040000 xr
ram              0x0000000020000000 0x0000000000010000 w !xr
bkup_ram         0x0000000000000000 0x0000000000000000 w !xr
*default*        0x0000000000000000 0xffffffffffffffff

Linker script and memory map

LOAD /home/ch/RIOT/examples/lorawan/bin/lora-e5-dev/application_lorawan/main.o
LOAD /home/ch/RIOT/examples/lorawan/bin/lora-e5-dev/auto_init/auto_init.o
LOAD /home/ch/RIOT/examples/lorawan/bin/lora-e5-dev/board/board.o
LOAD /home/ch/RIOT/examples/lorawan/bin/lora-e5-dev/checksum/crc16_ccitt.o
LOAD /home/ch/RIOT/examples/lorawan/bin/lora-e5-dev/checksum/crc8.o
LOAD /home/ch/RIOT/examples/lorawan/bin/lora-e5-dev/checksum/fletcher16.o
LOAD /home/ch/RIOT/examples/lorawan/bin/lora-e5-dev/checksum/fletcher32.o
LOAD /home/ch/RIOT/examples/lorawan/bin/lora-e5-dev/checksum/ucrc16.o
LOAD /home/ch/RIOT/examples/lorawan/bin/lora-e5-dev/core/assert.o
LOAD /home/ch/RIOT/examples/lorawan/bin/lora-e5-dev/core/atomic_c11.o
LOAD /home/ch/RIOT/examples/lorawan/bin/lora-e5-dev/core/atomic_sync.o
LOAD /home/ch/RIOT/examples/lorawan/bin/lora-e5-dev/core/bitarithm.o
LOAD /home/ch/RIOT/examples/lorawan/bin/lora-e5-dev/core/clist.o
LOAD /home/ch/RIOT/examples/lorawan/bin/lora-e5-dev/core/cond.o
LOAD /home/ch/RIOT/examples/lorawan/bin/lora-e5-dev/core/init.o
LOAD /home/ch/RIOT/examples/lorawan/bin/lora-e5-dev/core/msg.o
LOAD /home/ch/RIOT/examples/lorawan/bin/lora-e5-dev/core/mutex.o
LOAD /home/ch/RIOT/examples/lorawan/bin/lora-e5-dev/core/panic.o
LOAD /home/ch/RIOT/examples/lorawan/bin/lora-e5-dev/core/priority_queue.o
LOAD /home/ch/RIOT/examples/lorawan/bin/lora-e5-dev/core/ringbuffer.o
LOAD /home/ch/RIOT/examples/lorawan/bin/lora-e5-dev/core/rmutex.o
LOAD /home/ch/RIOT/examples/lorawan/bin/lora-e5-dev/core/sched.o
LOAD /home/ch/RIOT/examples/lorawan/bin/lora-e5-dev/core/thread.o
LOAD /home/ch/RIOT/examples/lorawan/bin/lora-e5-dev/cortexm_common/cortexm_init.o
LOAD /home/ch/RIOT/examples/lorawan/bin/lora-e5-dev/cortexm_common/mpu.o
LOAD /home/ch/RIOT/examples/lorawan/bin/lora-e5-dev/cortexm_common/panic.o
LOAD /home/ch/RIOT/examples/lorawan/bin/lora-e5-dev/cortexm_common_periph/pm.o
LOAD /home/ch/RIOT/examples/lorawan/bin/lora-e5-dev/cortexm_common/thread_arch.o
LOAD /home/ch/RIOT/examples/lorawan/bin/lora-e5-dev/cortexm_common/vectors_cortexm.o
LOAD /home/ch/RIOT/examples/lorawan/bin/lora-e5-dev/cpu/cpu_common.o
LOAD /home/ch/RIOT/examples/lorawan/bin/lora-e5-dev/cpu/cpu_init.o
LOAD /home/ch/RIOT/examples/lorawan/bin/lora-e5-dev/crypto/aes.o
LOAD /home/ch/RIOT/examples/lorawan/bin/lora-e5-dev/crypto/chacha20poly1305.o
LOAD /home/ch/RIOT/examples/lorawan/bin/lora-e5-dev/crypto/chacha.o
LOAD /home/ch/RIOT/examples/lorawan/bin/lora-e5-dev/crypto/chacha_prng.o
LOAD /home/ch/RIOT/examples/lorawan/bin/lora-e5-dev/crypto/ciphers.o
LOAD /home/ch/RIOT/examples/lorawan/bin/lora-e5-dev/crypto/helper.o
LOAD /home/ch/RIOT/examples/lorawan/bin/lora-e5-dev/crypto/poly1305.o
LOAD /home/ch/RIOT/examples/lorawan/bin/lora-e5-dev/div/div.o
LOAD /home/ch/RIOT/examples/lorawan/bin/lora-e5-dev/driver_sx126x_hal/driver_sx126x_hal.o
LOAD /home/ch/RIOT/examples/lorawan/bin/lora-e5-dev/driver_sx126x/sx126x.o
LOAD /home/ch/RIOT/examples/lorawan/bin/lora-e5-dev/fmt/fmt.o
LOAD /home/ch/RIOT/examples/lorawan/bin/lora-e5-dev/frac/frac.o
LOAD /home/ch/RIOT/examples/lorawan/bin/lora-e5-dev/hashes/cmac.o
LOAD /home/ch/RIOT/examples/lorawan/bin/lora-e5-dev/hashes/hashes.o
LOAD /home/ch/RIOT/examples/lorawan/bin/lora-e5-dev/hashes/md5.o
LOAD /home/ch/RIOT/examples/lorawan/bin/lora-e5-dev/hashes/pbkdf2.o
LOAD /home/ch/RIOT/examples/lorawan/bin/lora-e5-dev/hashes/sha1.o
LOAD /home/ch/RIOT/examples/lorawan/bin/lora-e5-dev/hashes/sha224.o
LOAD /home/ch/RIOT/examples/lorawan/bin/lora-e5-dev/hashes/sha256.o
LOAD /home/ch/RIOT/examples/lorawan/bin/lora-e5-dev/hashes/sha2xx_common.o
LOAD /home/ch/RIOT/examples/lorawan/bin/lora-e5-dev/hashes/sha3.o
LOAD /home/ch/RIOT/examples/lorawan/bin/lora-e5-dev/iolist/iolist.o
LOAD /home/ch/RIOT/examples/lorawan/bin/lora-e5-dev/luid/luid.o
LOAD /home/ch/RIOT/examples/lorawan/bin/lora-e5-dev/malloc_thread_safe/malloc_wrappers.o
LOAD /home/ch/RIOT/examples/lorawan/bin/lora-e5-dev/newlib_syscalls_default/syscalls.o
LOAD /home/ch/RIOT/examples/lorawan/bin/lora-e5-dev/periph_common/cpuid.o
LOAD /home/ch/RIOT/examples/lorawan/bin/lora-e5-dev/periph_common/gpio.o
LOAD /home/ch/RIOT/examples/lorawan/bin/lora-e5-dev/periph_common/i2c.o
LOAD /home/ch/RIOT/examples/lorawan/bin/lora-e5-dev/periph_common/init.o
LOAD /home/ch/RIOT/examples/lorawan/bin/lora-e5-dev/periph_common/pm.o
LOAD /home/ch/RIOT/examples/lorawan/bin/lora-e5-dev/periph_common/spi.o
LOAD /home/ch/RIOT/examples/lorawan/bin/lora-e5-dev/periph_common/timer.o
LOAD /home/ch/RIOT/examples/lorawan/bin/lora-e5-dev/periph/gpio_all.o
LOAD /home/ch/RIOT/examples/lorawan/bin/lora-e5-dev/periph/i2c_1.o
LOAD /home/ch/RIOT/examples/lorawan/bin/lora-e5-dev/periph/pm.o
LOAD /home/ch/RIOT/examples/lorawan/bin/lora-e5-dev/periph/rtt_all.o
LOAD /home/ch/RIOT/examples/lorawan/bin/lora-e5-dev/periph/spi.o
LOAD /home/ch/RIOT/examples/lorawan/bin/lora-e5-dev/periph/timer.o
LOAD /home/ch/RIOT/examples/lorawan/bin/lora-e5-dev/periph/uart.o
LOAD /home/ch/RIOT/examples/lorawan/bin/lora-e5-dev/pm_layered/pm.o
LOAD /home/ch/RIOT/examples/lorawan/bin/lora-e5-dev/random/musl_lcg.o
LOAD /home/ch/RIOT/examples/lorawan/bin/lora-e5-dev/random/random.o
LOAD /home/ch/RIOT/examples/lorawan/bin/lora-e5-dev/scd30/scd30.o
LOAD /home/ch/RIOT/examples/lorawan/bin/lora-e5-dev/semtech_loramac_arch/utilities.o
LOAD /home/ch/RIOT/examples/lorawan/bin/lora-e5-dev/semtech_loramac_contrib/semtech_loramac_getset.o
LOAD /home/ch/RIOT/examples/lorawan/bin/lora-e5-dev/semtech_loramac_contrib/semtech_loramac.o
LOAD /home/ch/RIOT/examples/lorawan/bin/lora-e5-dev/semtech_loramac_contrib/semtech_loramac_radio.o
LOAD /home/ch/RIOT/examples/lorawan/bin/lora-e5-dev/semtech_loramac_contrib/semtech_loramac_timer.o
LOAD /home/ch/RIOT/examples/lorawan/bin/lora-e5-dev/semtech_loramac_crypto/cmac.o
LOAD /home/ch/RIOT/examples/lorawan/bin/lora-e5-dev/semtech_loramac_mac/LoRaMacCrypto.o
LOAD /home/ch/RIOT/examples/lorawan/bin/lora-e5-dev/semtech_loramac_mac/LoRaMac.o
LOAD /home/ch/RIOT/examples/lorawan/bin/lora-e5-dev/semtech_loramac_mac_region/RegionAS923.o
LOAD /home/ch/RIOT/examples/lorawan/bin/lora-e5-dev/semtech_loramac_mac_region/RegionAU915.o
LOAD /home/ch/RIOT/examples/lorawan/bin/lora-e5-dev/semtech_loramac_mac_region/RegionCN470.o
LOAD /home/ch/RIOT/examples/lorawan/bin/lora-e5-dev/semtech_loramac_mac_region/RegionCN779.o
LOAD /home/ch/RIOT/examples/lorawan/bin/lora-e5-dev/semtech_loramac_mac_region/RegionCommon.o
LOAD /home/ch/RIOT/examples/lorawan/bin/lora-e5-dev/semtech_loramac_mac_region/RegionEU433.o
LOAD /home/ch/RIOT/examples/lorawan/bin/lora-e5-dev/semtech_loramac_mac_region/RegionEU868.o
LOAD /home/ch/RIOT/examples/lorawan/bin/lora-e5-dev/semtech_loramac_mac_region/RegionIN865.o
LOAD /home/ch/RIOT/examples/lorawan/bin/lora-e5-dev/semtech_loramac_mac_region/RegionKR920.o
LOAD /home/ch/RIOT/examples/lorawan/bin/lora-e5-dev/semtech_loramac_mac_region/Region.o
LOAD /home/ch/RIOT/examples/lorawan/bin/lora-e5-dev/semtech_loramac_mac_region/RegionRU864.o
LOAD /home/ch/RIOT/examples/lorawan/bin/lora-e5-dev/semtech_loramac_mac_region/RegionUS915-Hybrid.o
LOAD /home/ch/RIOT/examples/lorawan/bin/lora-e5-dev/semtech_loramac_mac_region/RegionUS915.o
LOAD /home/ch/RIOT/examples/lorawan/bin/lora-e5-dev/stdio_uart/stdio_uart.o
LOAD /home/ch/RIOT/examples/lorawan/bin/lora-e5-dev/stm32_clk/stmclk_common.o
LOAD /home/ch/RIOT/examples/lorawan/bin/lora-e5-dev/stm32_clk/stmclk_l4wx.o
LOAD /home/ch/RIOT/examples/lorawan/bin/lora-e5-dev/stm32_vectors/STM32WLE5xx.o
LOAD /home/ch/RIOT/examples/lorawan/bin/lora-e5-dev/sx126x/sx126x_netdev.o
LOAD /home/ch/RIOT/examples/lorawan/bin/lora-e5-dev/sx126x/sx126x.o
LOAD /home/ch/RIOT/examples/lorawan/bin/lora-e5-dev/xtimer/xtimer_core.o
LOAD /home/ch/RIOT/examples/lorawan/bin/lora-e5-dev/xtimer/xtimer.o
LOAD /home/ch/RIOT/examples/lorawan/bin/lora-e5-dev/ztimer_core/convert_frac.o
LOAD /home/ch/RIOT/examples/lorawan/bin/lora-e5-dev/ztimer_core/convert.o
LOAD /home/ch/RIOT/examples/lorawan/bin/lora-e5-dev/ztimer_core/convert_shift.o
LOAD /home/ch/RIOT/examples/lorawan/bin/lora-e5-dev/ztimer_core/core.o
LOAD /home/ch/RIOT/examples/lorawan/bin/lora-e5-dev/ztimer_core/init.o
LOAD /home/ch/RIOT/examples/lorawan/bin/lora-e5-dev/ztimer_core/periodic.o
LOAD /home/ch/RIOT/examples/lorawan/bin/lora-e5-dev/ztimer_core/periph_rtt.o
LOAD /home/ch/RIOT/examples/lorawan/bin/lora-e5-dev/ztimer_core/periph_timer.o
LOAD /home/ch/RIOT/examples/lorawan/bin/lora-e5-dev/ztimer_core/util.o
LOAD /usr/lib/gcc/arm-none-eabi/9.2.1/../../../arm-none-eabi/lib/thumb/v7e-m/nofp/libm.a
LOAD /usr/lib/gcc/arm-none-eabi/9.2.1/thumb/v7e-m/nofp/libgcc.a
                0x0000000008000000                _rom_start_addr = 0x8000000
                0x0000000020000000                _ram_start_addr = 0x20000000
                0x0000000000040000                _rom_length = 0x40000
                0x0000000000010000                _ram_length = 0x10000
LOAD /usr/lib/gcc/arm-none-eabi/9.2.1/../../../arm-none-eabi/lib/thumb/v7e-m/nofp/libc_nano.a
START GROUP
LOAD /usr/lib/gcc/arm-none-eabi/9.2.1/thumb/v7e-m/nofp/libgcc.a
LOAD /usr/lib/gcc/arm-none-eabi/9.2.1/../../../arm-none-eabi/lib/thumb/v7e-m/nofp/libg_nano.a
LOAD /usr/lib/gcc/arm-none-eabi/9.2.1/../../../arm-none-eabi/lib/thumb/v7e-m/nofp/libc_nano.a
END GROUP
START GROUP
LOAD /usr/lib/gcc/arm-none-eabi/9.2.1/thumb/v7e-m/nofp/libgcc.a
LOAD /usr/lib/gcc/arm-none-eabi/9.2.1/../../../arm-none-eabi/lib/thumb/v7e-m/nofp/libc_nano.a
END GROUP
                0x0000000000000000                ccmram_length = DEFINED (ccmram_len)?ccmram_len:0x0
                0x0000000000000000                sram4_length = DEFINED (sram4_length)?sram4_length:0x0

.heap2          0x0000000000000000        0x0
                0x0000000000000000                _sheap2 = .
                0x0000000028000000                _eheap2 = (ORIGIN (sram4) + LENGTH (sram4))
                0x0000000000000000                _rom_offset = DEFINED (_rom_offset)?_rom_offset:0x0
                0x0000000000040000                _fw_rom_length = DEFINED (_fw_rom_length)?_fw_rom_length:(_rom_length - _rom_offset)
                0x0000000000000001                ASSERT ((_fw_rom_length <= (_rom_length - _rom_offset)), Specified firmware size does not fit in ROM)
                0x0000000000000000                _backup_ram_start_addr = DEFINED (_backup_ram_start_addr)?_backup_ram_start_addr:0x0
                0x0000000000000000                _backup_ram_len = DEFINED (_backup_ram_len)?_backup_ram_len:0x0

.text           0x0000000008000000     0xd7fc
                0x0000000008000000                . = ALIGN (0x4)
                0x0000000008000000                _sfixed = .
                0x0000000008000000                _isr_vectors = DEFINED (_isr_vectors)?_isr_vectors:.
 *(SORT_BY_NAME(.vectors*))
 .vectors.0     0x0000000008000000       0x40 /home/ch/RIOT/examples/lorawan/bin/lora-e5-dev/cortexm_common/vectors_cortexm.o
                0x0000000008000000                cortex_vector_base
 .vectors.1     0x0000000008000040       0xf8 /home/ch/RIOT/examples/lorawan/bin/lora-e5-dev/stm32_vectors/STM32WLE5xx.o
                0x0000000008000040                vector_cpu
 *(.text .text.* .gnu.linkonce.t.*)
 .text._alarm_cb
                0x0000000008000138       0x18 /home/ch/RIOT/examples/lorawan/bin/lora-e5-dev/application_lorawan/main.o
 .text.sender   0x0000000008000150       0x70 /home/ch/RIOT/examples/lorawan/bin/lora-e5-dev/application_lorawan/main.o
 .text.startup.main
                0x00000000080001c0       0xfc /home/ch/RIOT/examples/lorawan/bin/lora-e5-dev/application_lorawan/main.o
                0x00000000080001c0                main
 .text.auto_init
                0x00000000080002bc       0x12 /home/ch/RIOT/examples/lorawan/bin/lora-e5-dev/auto_init/auto_init.o
                0x00000000080002bc                auto_init
 *fill*         0x00000000080002ce        0x2 
 .text.board_init
                0x00000000080002d0       0x5c /home/ch/RIOT/examples/lorawan/bin/lora-e5-dev/board/board.o
                0x00000000080002d0                board_init
 .text.lora_e5_dev_sx126x_set_rf_mode
                0x000000000800032c       0x3c /home/ch/RIOT/examples/lorawan/bin/lora-e5-dev/board/board.o
                0x000000000800032c                lora_e5_dev_sx126x_set_rf_mode
 .text.main_trampoline
                0x0000000008000368       0x18 /home/ch/RIOT/examples/lorawan/bin/lora-e5-dev/core/init.o
 .text.kernel_init
                0x0000000008000380       0x34 /home/ch/RIOT/examples/lorawan/bin/lora-e5-dev/core/init.o
                0x0000000008000380                kernel_init
 .text._msg_receive
                0x00000000080003b4       0xec /home/ch/RIOT/examples/lorawan/bin/lora-e5-dev/core/msg.o
 .text.queue_msg
                0x00000000080004a0       0x2a /home/ch/RIOT/examples/lorawan/bin/lora-e5-dev/core/msg.o
 *fill*         0x00000000080004ca        0x2 
 .text._msg_send_oneway
                0x00000000080004cc       0x44 /home/ch/RIOT/examples/lorawan/bin/lora-e5-dev/core/msg.o
 .text._msg_send
                0x0000000008000510       0xa4 /home/ch/RIOT/examples/lorawan/bin/lora-e5-dev/core/msg.o
 .text.msg_send_to_self
                0x00000000080005b4       0x28 /home/ch/RIOT/examples/lorawan/bin/lora-e5-dev/core/msg.o
                0x00000000080005b4                msg_send_to_self
 .text.msg_send_int
                0x00000000080005dc        0x8 /home/ch/RIOT/examples/lorawan/bin/lora-e5-dev/core/msg.o
                0x00000000080005dc                msg_send_int
 .text.msg_send
                0x00000000080005e4       0x2c /home/ch/RIOT/examples/lorawan/bin/lora-e5-dev/core/msg.o
                0x00000000080005e4                msg_send
 .text.msg_send_receive
                0x0000000008000610       0x54 /home/ch/RIOT/examples/lorawan/bin/lora-e5-dev/core/msg.o
                0x0000000008000610                msg_send_receive
 .text.msg_reply
                0x0000000008000664       0x54 /home/ch/RIOT/examples/lorawan/bin/lora-e5-dev/core/msg.o
                0x0000000008000664                msg_reply
 .text.msg_receive
                0x00000000080006b8        0x6 /home/ch/RIOT/examples/lorawan/bin/lora-e5-dev/core/msg.o
                0x00000000080006b8                msg_receive
 *fill*         0x00000000080006be        0x2 
 .text.msg_init_queue
                0x00000000080006c0       0x28 /home/ch/RIOT/examples/lorawan/bin/lora-e5-dev/core/msg.o
                0x00000000080006c0                msg_init_queue
 .text.mutex_lock
                0x00000000080006e8       0x68 /home/ch/RIOT/examples/lorawan/bin/lora-e5-dev/core/mutex.o
                0x00000000080006e8                mutex_lock
 .text.mutex_unlock
                0x0000000008000750       0x44 /home/ch/RIOT/examples/lorawan/bin/lora-e5-dev/core/mutex.o
                0x0000000008000750                mutex_unlock
 .text.panic_app
                0x0000000008000794        0x2 /home/ch/RIOT/examples/lorawan/bin/lora-e5-dev/core/panic.o
                0x0000000008000794                panic_app
 *fill*         0x0000000008000796        0x2 
 .text.core_panic
                0x0000000008000798       0x50 /home/ch/RIOT/examples/lorawan/bin/lora-e5-dev/core/panic.o
                0x0000000008000798                core_panic
 .text._unschedule
                0x00000000080007e8       0x24 /home/ch/RIOT/examples/lorawan/bin/lora-e5-dev/core/sched.o
 .text.sched_run
                0x000000000800080c       0x6c /home/ch/RIOT/examples/lorawan/bin/lora-e5-dev/core/sched.o
                0x000000000800080c                sched_run
 .text.sched_set_status
                0x0000000008000878       0x84 /home/ch/RIOT/examples/lorawan/bin/lora-e5-dev/core/sched.o
                0x0000000008000878                sched_set_status
 .text.sched_switch
                0x00000000080008fc       0x3c /home/ch/RIOT/examples/lorawan/bin/lora-e5-dev/core/sched.o
                0x00000000080008fc                sched_switch
 .text.sched_task_exit
                0x0000000008000938       0x3c /home/ch/RIOT/examples/lorawan/bin/lora-e5-dev/core/sched.o
                0x0000000008000938                sched_task_exit
 .text.thread_getname
                0x0000000008000974       0x1c /home/ch/RIOT/examples/lorawan/bin/lora-e5-dev/core/thread.o
                0x0000000008000974                thread_getname
 .text.thread_add_to_list
                0x0000000008000990       0x30 /home/ch/RIOT/examples/lorawan/bin/lora-e5-dev/core/thread.o
                0x0000000008000990                thread_add_to_list
 .text.thread_create
                0x00000000080009c0       0xe8 /home/ch/RIOT/examples/lorawan/bin/lora-e5-dev/core/thread.o
                0x00000000080009c0                thread_create
 .text.cortexm_init
                0x0000000008000aa8       0x40 /home/ch/RIOT/examples/lorawan/bin/lora-e5-dev/cortexm_common/cortexm_init.o
                0x0000000008000aa8                cortexm_init
 .text.panic_arch
                0x0000000008000ae8       0x1c /home/ch/RIOT/examples/lorawan/bin/lora-e5-dev/cortexm_common/panic.o
                0x0000000008000ae8                panic_arch
 .text.thread_stack_init
                0x0000000008000b04       0x68 /home/ch/RIOT/examples/lorawan/bin/lora-e5-dev/cortexm_common/thread_arch.o
                0x0000000008000b04                thread_stack_init
 .text.cpu_switch_context_exit
                0x0000000008000b6c       0x18 /home/ch/RIOT/examples/lorawan/bin/lora-e5-dev/cortexm_common/thread_arch.o
                0x0000000008000b6c                cpu_switch_context_exit
 .text.isr_pendsv
                0x0000000008000b84       0x38 /home/ch/RIOT/examples/lorawan/bin/lora-e5-dev/cortexm_common/thread_arch.o
                0x0000000008000b84                isr_pendsv
 .text.isr_svc  0x0000000008000bbc       0x10 /home/ch/RIOT/examples/lorawan/bin/lora-e5-dev/cortexm_common/thread_arch.o
                0x0000000008000bbc                isr_svc
 .text.sched_arch_idle
                0x0000000008000bcc       0x10 /home/ch/RIOT/examples/lorawan/bin/lora-e5-dev/cortexm_common/thread_arch.o
                0x0000000008000bcc                sched_arch_idle
 .text.hard_fault_default
                0x0000000008000bdc       0x44 /home/ch/RIOT/examples/lorawan/bin/lora-e5-dev/cortexm_common/vectors_cortexm.o
                0x0000000008000bdc                hard_fault_default
 .text.nmi_default
                0x0000000008000c20       0x10 /home/ch/RIOT/examples/lorawan/bin/lora-e5-dev/cortexm_common/vectors_cortexm.o
                0x0000000008000c20                nmi_default
 .text.mem_manage_default
                0x0000000008000c30       0x10 /home/ch/RIOT/examples/lorawan/bin/lora-e5-dev/cortexm_common/vectors_cortexm.o
                0x0000000008000c30                mem_manage_default
 .text.bus_fault_default
                0x0000000008000c40       0x10 /home/ch/RIOT/examples/lorawan/bin/lora-e5-dev/cortexm_common/vectors_cortexm.o
                0x0000000008000c40                bus_fault_default
 .text.usage_fault_default
                0x0000000008000c50       0x10 /home/ch/RIOT/examples/lorawan/bin/lora-e5-dev/cortexm_common/vectors_cortexm.o
                0x0000000008000c50                usage_fault_default
 .text.debug_mon_default
                0x0000000008000c60       0x10 /home/ch/RIOT/examples/lorawan/bin/lora-e5-dev/cortexm_common/vectors_cortexm.o
                0x0000000008000c60                debug_mon_default
 .text.dummy_handler_default
                0x0000000008000c70       0x10 /home/ch/RIOT/examples/lorawan/bin/lora-e5-dev/cortexm_common/vectors_cortexm.o
                0x0000000008000c70                dummy_handler_default
                0x0000000008000c70                isr_systick
 .text.pre_startup
                0x0000000008000c80        0x2 /home/ch/RIOT/examples/lorawan/bin/lora-e5-dev/cortexm_common/vectors_cortexm.o
                0x0000000008000c80                pre_startup
 .text.post_startup
                0x0000000008000c82        0x2 /home/ch/RIOT/examples/lorawan/bin/lora-e5-dev/cortexm_common/vectors_cortexm.o
                0x0000000008000c82                post_startup
 .text.reset_handler_default
                0x0000000008000c84       0x70 /home/ch/RIOT/examples/lorawan/bin/lora-e5-dev/cortexm_common/vectors_cortexm.o
                0x0000000008000c84                reset_handler_default
 .text.hard_fault_handler
                0x0000000008000cf4      0x1bc /home/ch/RIOT/examples/lorawan/bin/lora-e5-dev/cortexm_common/vectors_cortexm.o
                0x0000000008000cf4                hard_fault_handler
 .text.periph_apb_clk
                0x0000000008000eb0       0x18 /home/ch/RIOT/examples/lorawan/bin/lora-e5-dev/cpu/cpu_common.o
                0x0000000008000eb0                periph_apb_clk
 .text.periph_timer_clk
                0x0000000008000ec8       0x20 /home/ch/RIOT/examples/lorawan/bin/lora-e5-dev/cpu/cpu_common.o
                0x0000000008000ec8                periph_timer_clk
 .text.periph_clk_en
                0x0000000008000ee8       0x68 /home/ch/RIOT/examples/lorawan/bin/lora-e5-dev/cpu/cpu_common.o
                0x0000000008000ee8                periph_clk_en
 .text.periph_clk_dis
                0x0000000008000f50       0x72 /home/ch/RIOT/examples/lorawan/bin/lora-e5-dev/cpu/cpu_common.o
                0x0000000008000f50                periph_clk_dis
 .text.cpu_init
                0x0000000008000fc2       0x16 /home/ch/RIOT/examples/lorawan/bin/lora-e5-dev/cpu/cpu_init.o
                0x0000000008000fc2                cpu_init
 .text.aes_init
                0x0000000008000fd8       0x22 /home/ch/RIOT/examples/lorawan/bin/lora-e5-dev/crypto/aes.o
                0x0000000008000fd8                aes_init
 *fill*         0x0000000008000ffa        0x2 
 .text.aes_set_encrypt_key.constprop.0
                0x0000000008000ffc       0xf0 /home/ch/RIOT/examples/lorawan/bin/lora-e5-dev/crypto/aes.o
 .text.aes_encrypt
                0x00000000080010ec      0x358 /home/ch/RIOT/examples/lorawan/bin/lora-e5-dev/crypto/aes.o
                0x00000000080010ec                aes_encrypt
 .text.sx126x_is_stm32wl.part.0
                0x0000000008001444       0x10 /home/ch/RIOT/examples/lorawan/bin/lora-e5-dev/driver_sx126x_hal/driver_sx126x_hal.o
 .text.sx126x_hal_reset
                0x0000000008001454       0x88 /home/ch/RIOT/examples/lorawan/bin/lora-e5-dev/driver_sx126x_hal/driver_sx126x_hal.o
                0x0000000008001454                sx126x_hal_reset
 .text.sx126x_hal_wakeup
                0x00000000080014dc       0x48 /home/ch/RIOT/examples/lorawan/bin/lora-e5-dev/driver_sx126x_hal/driver_sx126x_hal.o
                0x00000000080014dc                sx126x_hal_wakeup
 .text.sx126x_radio_wait_until_ready
                0x0000000008001524       0x24 /home/ch/RIOT/examples/lorawan/bin/lora-e5-dev/driver_sx126x_hal/driver_sx126x_hal.o
 .text.sx126x_hal_write
                0x0000000008001548       0xa8 /home/ch/RIOT/examples/lorawan/bin/lora-e5-dev/driver_sx126x_hal/driver_sx126x_hal.o
                0x0000000008001548                sx126x_hal_write
 .text.sx126x_hal_read
                0x00000000080015f0       0x88 /home/ch/RIOT/examples/lorawan/bin/lora-e5-dev/driver_sx126x_hal/driver_sx126x_hal.o
                0x00000000080015f0                sx126x_hal_read
 .text.sx126x_set_standby
                0x0000000008001678       0x1e /home/ch/RIOT/examples/lorawan/bin/lora-e5-dev/driver_sx126x/sx126x.o
                0x0000000008001678                sx126x_set_standby
 .text.sx126x_set_tx_with_timeout_in_rtc_step
                0x0000000008001696       0x26 /home/ch/RIOT/examples/lorawan/bin/lora-e5-dev/driver_sx126x/sx126x.o
                0x0000000008001696                sx126x_set_tx_with_timeout_in_rtc_step
 .text.sx126x_set_tx
                0x00000000080016bc       0x10 /home/ch/RIOT/examples/lorawan/bin/lora-e5-dev/driver_sx126x/sx126x.o
                0x00000000080016bc                sx126x_set_tx
 .text.sx126x_set_rx_with_timeout_in_rtc_step
                0x00000000080016cc       0x26 /home/ch/RIOT/examples/lorawan/bin/lora-e5-dev/driver_sx126x/sx126x.o
                0x00000000080016cc                sx126x_set_rx_with_timeout_in_rtc_step
 .text.sx126x_set_rx
                0x00000000080016f2       0x10 /home/ch/RIOT/examples/lorawan/bin/lora-e5-dev/driver_sx126x/sx126x.o
                0x00000000080016f2                sx126x_set_rx
 .text.sx126x_stop_timer_on_preamble
                0x0000000008001702       0x1e /home/ch/RIOT/examples/lorawan/bin/lora-e5-dev/driver_sx126x/sx126x.o
                0x0000000008001702                sx126x_stop_timer_on_preamble
 .text.sx126x_set_reg_mode
                0x0000000008001720       0x1e /home/ch/RIOT/examples/lorawan/bin/lora-e5-dev/driver_sx126x/sx126x.o
                0x0000000008001720                sx126x_set_reg_mode
 .text.sx126x_set_pa_cfg
                0x000000000800173e       0x32 /home/ch/RIOT/examples/lorawan/bin/lora-e5-dev/driver_sx126x/sx126x.o
                0x000000000800173e                sx126x_set_pa_cfg
 .text.sx126x_write_register
                0x0000000008001770       0x22 /home/ch/RIOT/examples/lorawan/bin/lora-e5-dev/driver_sx126x/sx126x.o
                0x0000000008001770                sx126x_write_register
 .text.sx126x_read_register
                0x0000000008001792       0x26 /home/ch/RIOT/examples/lorawan/bin/lora-e5-dev/driver_sx126x/sx126x.o
                0x0000000008001792                sx126x_read_register
 .text.sx126x_write_buffer
                0x00000000080017b8       0x1c /home/ch/RIOT/examples/lorawan/bin/lora-e5-dev/driver_sx126x/sx126x.o
                0x00000000080017b8                sx126x_write_buffer
 .text.sx126x_read_buffer
                0x00000000080017d4       0x22 /home/ch/RIOT/examples/lorawan/bin/lora-e5-dev/driver_sx126x/sx126x.o
                0x00000000080017d4                sx126x_read_buffer
 .text.sx126x_set_dio_irq_params
                0x00000000080017f6       0x48 /home/ch/RIOT/examples/lorawan/bin/lora-e5-dev/driver_sx126x/sx126x.o
                0x00000000080017f6                sx126x_set_dio_irq_params
 .text.sx126x_get_irq_status
                0x000000000800183e       0x34 /home/ch/RIOT/examples/lorawan/bin/lora-e5-dev/driver_sx126x/sx126x.o
                0x000000000800183e                sx126x_get_irq_status
 .text.sx126x_clear_irq_status
                0x0000000008001872       0x24 /home/ch/RIOT/examples/lorawan/bin/lora-e5-dev/driver_sx126x/sx126x.o
                0x0000000008001872                sx126x_clear_irq_status
 .text.sx126x_get_and_clear_irq_status
                0x0000000008001896       0x3c /home/ch/RIOT/examples/lorawan/bin/lora-e5-dev/driver_sx126x/sx126x.o
                0x0000000008001896                sx126x_get_and_clear_irq_status
 .text.sx126x_set_rf_freq_in_pll_steps
                0x00000000080018d2       0x30 /home/ch/RIOT/examples/lorawan/bin/lora-e5-dev/driver_sx126x/sx126x.o
                0x00000000080018d2                sx126x_set_rf_freq_in_pll_steps
 .text.sx126x_set_pkt_type
                0x0000000008001902       0x1e /home/ch/RIOT/examples/lorawan/bin/lora-e5-dev/driver_sx126x/sx126x.o
                0x0000000008001902                sx126x_set_pkt_type
 .text.sx126x_get_pkt_type
                0x0000000008001920       0x38 /home/ch/RIOT/examples/lorawan/bin/lora-e5-dev/driver_sx126x/sx126x.o
                0x0000000008001920                sx126x_get_pkt_type
 .text.sx126x_set_tx_params
                0x0000000008001958       0x22 /home/ch/RIOT/examples/lorawan/bin/lora-e5-dev/driver_sx126x/sx126x.o
                0x0000000008001958                sx126x_set_tx_params
 .text.sx126x_set_lora_mod_params
                0x000000000800197a       0x78 /home/ch/RIOT/examples/lorawan/bin/lora-e5-dev/driver_sx126x/sx126x.o
                0x000000000800197a                sx126x_set_lora_mod_params
 .text.sx126x_set_lora_pkt_params
                0x00000000080019f2       0x80 /home/ch/RIOT/examples/lorawan/bin/lora-e5-dev/driver_sx126x/sx126x.o
                0x00000000080019f2                sx126x_set_lora_pkt_params
 .text.sx126x_get_status
                0x0000000008001a72       0x34 /home/ch/RIOT/examples/lorawan/bin/lora-e5-dev/driver_sx126x/sx126x.o
                0x0000000008001a72                sx126x_get_status
 .text.sx126x_get_rx_buffer_status
                0x0000000008001aa6       0x32 /home/ch/RIOT/examples/lorawan/bin/lora-e5-dev/driver_sx126x/sx126x.o
                0x0000000008001aa6                sx126x_get_rx_buffer_status
 .text.sx126x_get_lora_pkt_status
                0x0000000008001ad8       0x54 /home/ch/RIOT/examples/lorawan/bin/lora-e5-dev/driver_sx126x/sx126x.o
                0x0000000008001ad8                sx126x_get_lora_pkt_status
 .text.sx126x_get_rssi_inst
                0x0000000008001b2c       0x34 /home/ch/RIOT/examples/lorawan/bin/lora-e5-dev/driver_sx126x/sx126x.o
                0x0000000008001b2c                sx126x_get_rssi_inst
 .text.sx126x_reset
                0x0000000008001b60        0x4 /home/ch/RIOT/examples/lorawan/bin/lora-e5-dev/driver_sx126x/sx126x.o
                0x0000000008001b60                sx126x_reset
 .text.sx126x_get_random_numbers
                0x0000000008001b64       0xd0 /home/ch/RIOT/examples/lorawan/bin/lora-e5-dev/driver_sx126x/sx126x.o
                0x0000000008001b64                sx126x_get_random_numbers
 .text.sx126x_convert_freq_in_hz_to_pll_step
                0x0000000008001c34       0x1e /home/ch/RIOT/examples/lorawan/bin/lora-e5-dev/driver_sx126x/sx126x.o
                0x0000000008001c34                sx126x_convert_freq_in_hz_to_pll_step
 .text.sx126x_set_rf_freq
                0x0000000008001c52       0x16 /home/ch/RIOT/examples/lorawan/bin/lora-e5-dev/driver_sx126x/sx126x.o
                0x0000000008001c52                sx126x_set_rf_freq
 .text.sx126x_cfg_rx_boosted
                0x0000000008001c68       0x20 /home/ch/RIOT/examples/lorawan/bin/lora-e5-dev/driver_sx126x/sx126x.o
                0x0000000008001c68                sx126x_cfg_rx_boosted
 .text.sx126x_set_lora_sync_word
                0x0000000008001c88       0x4e /home/ch/RIOT/examples/lorawan/bin/lora-e5-dev/driver_sx126x/sx126x.o
                0x0000000008001c88                sx126x_set_lora_sync_word
 .text.fmt_strlen
                0x0000000008001cd6       0x10 /home/ch/RIOT/examples/lorawan/bin/lora-e5-dev/fmt/fmt.o
                0x0000000008001cd6                fmt_strlen
 .text.fmt_hex_byte
                0x0000000008001ce6       0x46 /home/ch/RIOT/examples/lorawan/bin/lora-e5-dev/fmt/fmt.o
                0x0000000008001ce6                fmt_hex_byte
 .text.fmt_hex_bytes
                0x0000000008001d2c       0x34 /home/ch/RIOT/examples/lorawan/bin/lora-e5-dev/fmt/fmt.o
                0x0000000008001d2c                fmt_hex_bytes
 .text.gcd32    0x0000000008001d60       0x40 /home/ch/RIOT/examples/lorawan/bin/lora-e5-dev/frac/frac.o
                0x0000000008001d60                gcd32
 .text.frac_init
                0x0000000008001da0       0xb4 /home/ch/RIOT/examples/lorawan/bin/lora-e5-dev/frac/frac.o
                0x0000000008001da0                frac_init
 .text.luid_base
                0x0000000008001e54       0x64 /home/ch/RIOT/examples/lorawan/bin/lora-e5-dev/luid/luid.o
                0x0000000008001e54                luid_base
 .text.luid_get
                0x0000000008001eb8       0x1c /home/ch/RIOT/examples/lorawan/bin/lora-e5-dev/luid/luid.o
                0x0000000008001eb8                luid_get
 .text.__wrap_malloc
                0x0000000008001ed4       0x38 /home/ch/RIOT/examples/lorawan/bin/lora-e5-dev/malloc_thread_safe/malloc_wrappers.o
                0x0000000008001ed4                __wrap_malloc
 .text._init    0x0000000008001f0c        0x2 /home/ch/RIOT/examples/lorawan/bin/lora-e5-dev/newlib_syscalls_default/syscalls.o
                0x0000000008001f0c                _init
 .text._fini    0x0000000008001f0e        0x2 /home/ch/RIOT/examples/lorawan/bin/lora-e5-dev/newlib_syscalls_default/syscalls.o
                0x0000000008001f0e                _fini
 .text._exit    0x0000000008001f10       0x14 /home/ch/RIOT/examples/lorawan/bin/lora-e5-dev/newlib_syscalls_default/syscalls.o
                0x0000000008001f10                _exit
 .text._sbrk_r  0x0000000008001f24       0x40 /home/ch/RIOT/examples/lorawan/bin/lora-e5-dev/newlib_syscalls_default/syscalls.o
                0x0000000008001f24                _sbrk_r
 .text._getpid_r
                0x0000000008001f64        0xc /home/ch/RIOT/examples/lorawan/bin/lora-e5-dev/newlib_syscalls_default/syscalls.o
                0x0000000008001f64                _getpid_r
 .text._kill_r  0x0000000008001f70        0xa /home/ch/RIOT/examples/lorawan/bin/lora-e5-dev/newlib_syscalls_default/syscalls.o
                0x0000000008001f70                _kill_r
 .text._read_r  0x0000000008001f7a        0x8 /home/ch/RIOT/examples/lorawan/bin/lora-e5-dev/newlib_syscalls_default/syscalls.o
                0x0000000008001f7a                _read_r
 .text._write_r
                0x0000000008001f82        0x8 /home/ch/RIOT/examples/lorawan/bin/lora-e5-dev/newlib_syscalls_default/syscalls.o
                0x0000000008001f82                _write_r
 .text._close_r
                0x0000000008001f8a        0xa /home/ch/RIOT/examples/lorawan/bin/lora-e5-dev/newlib_syscalls_default/syscalls.o
                0x0000000008001f8a                _close_r
 .text._lseek_r
                0x0000000008001f94        0xa /home/ch/RIOT/examples/lorawan/bin/lora-e5-dev/newlib_syscalls_default/syscalls.o
                0x0000000008001f94                _lseek_r
 .text._fstat_r
                0x0000000008001f9e        0xa /home/ch/RIOT/examples/lorawan/bin/lora-e5-dev/newlib_syscalls_default/syscalls.o
                0x0000000008001f9e                _fstat_r
 .text._isatty_r
                0x0000000008001fa8       0x10 /home/ch/RIOT/examples/lorawan/bin/lora-e5-dev/newlib_syscalls_default/syscalls.o
                0x0000000008001fa8                _isatty_r
 .text.cpuid_get
                0x0000000008001fb8        0xc /home/ch/RIOT/examples/lorawan/bin/lora-e5-dev/periph_common/cpuid.o
                0x0000000008001fb8                cpuid_get
 .text.periph_init
                0x0000000008001fc4       0x1c /home/ch/RIOT/examples/lorawan/bin/lora-e5-dev/periph_common/init.o
                0x0000000008001fc4                periph_init
 .text.timer_set
                0x0000000008001fe0       0x22 /home/ch/RIOT/examples/lorawan/bin/lora-e5-dev/periph_common/timer.o
                0x0000000008001fe0                timer_set
 .text.gpio_init
                0x0000000008002002       0x68 /home/ch/RIOT/examples/lorawan/bin/lora-e5-dev/periph/gpio_all.o
                0x0000000008002002                gpio_init
 .text.gpio_init_af
                0x000000000800206a       0x58 /home/ch/RIOT/examples/lorawan/bin/lora-e5-dev/periph/gpio_all.o
                0x000000000800206a                gpio_init_af
 .text.gpio_set
                0x00000000080020c2       0x12 /home/ch/RIOT/examples/lorawan/bin/lora-e5-dev/periph/gpio_all.o
                0x00000000080020c2                gpio_set
 .text.gpio_clear
                0x00000000080020d4       0x14 /home/ch/RIOT/examples/lorawan/bin/lora-e5-dev/periph/gpio_all.o
                0x00000000080020d4                gpio_clear
 .text.isr_exti
                0x00000000080020e8       0x5c /home/ch/RIOT/examples/lorawan/bin/lora-e5-dev/periph/gpio_all.o
                0x00000000080020e8                isr_exti
 .text.i2c_init
                0x0000000008002144       0x98 /home/ch/RIOT/examples/lorawan/bin/lora-e5-dev/periph/i2c_1.o
                0x0000000008002144                i2c_init
 .text.isr_i2c2_er
                0x00000000080021dc       0x10 /home/ch/RIOT/examples/lorawan/bin/lora-e5-dev/periph/i2c_1.o
                0x00000000080021dc                isr_i2c2_er
 .text.pm_set   0x00000000080021ec       0x74 /home/ch/RIOT/examples/lorawan/bin/lora-e5-dev/periph/pm.o
                0x00000000080021ec                pm_set
 .text.rtt_get_counter
                0x0000000008002260       0x10 /home/ch/RIOT/examples/lorawan/bin/lora-e5-dev/periph/rtt_all.o
                0x0000000008002260                rtt_get_counter
 .text.rtt_set_alarm
                0x0000000008002270       0x44 /home/ch/RIOT/examples/lorawan/bin/lora-e5-dev/periph/rtt_all.o
                0x0000000008002270                rtt_set_alarm
 .text.rtt_clear_alarm
                0x00000000080022b4        0xc /home/ch/RIOT/examples/lorawan/bin/lora-e5-dev/periph/rtt_all.o
                0x00000000080022b4                rtt_clear_alarm
 .text.rtt_poweron
                0x00000000080022c0        0xa /home/ch/RIOT/examples/lorawan/bin/lora-e5-dev/periph/rtt_all.o
                0x00000000080022c0                rtt_poweron
 *fill*         0x00000000080022ca        0x2 
 .text.rtt_init
                0x00000000080022cc       0x70 /home/ch/RIOT/examples/lorawan/bin/lora-e5-dev/periph/rtt_all.o
                0x00000000080022cc                rtt_init
 .text.isr_lptim1
                0x000000000800233c       0x64 /home/ch/RIOT/examples/lorawan/bin/lora-e5-dev/periph/rtt_all.o
                0x000000000800233c                isr_lptim1
 .text.spi_init_pins
                0x00000000080023a0       0x5c /home/ch/RIOT/examples/lorawan/bin/lora-e5-dev/periph/spi.o
                0x00000000080023a0                spi_init_pins
 .text.spi_init
                0x00000000080023fc       0x5c /home/ch/RIOT/examples/lorawan/bin/lora-e5-dev/periph/spi.o
                0x00000000080023fc                spi_init
 .text.spi_init_cs
                0x0000000008002458       0x64 /home/ch/RIOT/examples/lorawan/bin/lora-e5-dev/periph/spi.o
                0x0000000008002458                spi_init_cs
 .text.spi_acquire
                0x00000000080024bc       0xc4 /home/ch/RIOT/examples/lorawan/bin/lora-e5-dev/periph/spi.o
                0x00000000080024bc                spi_acquire
 .text.spi_release
                0x0000000008002580       0x3c /home/ch/RIOT/examples/lorawan/bin/lora-e5-dev/periph/spi.o
                0x0000000008002580                spi_release
 .text.spi_transfer_bytes
                0x00000000080025bc       0xe0 /home/ch/RIOT/examples/lorawan/bin/lora-e5-dev/periph/spi.o
                0x00000000080025bc                spi_transfer_bytes
 .text.timer_set_absolute
                0x000000000800269c       0x38 /home/ch/RIOT/examples/lorawan/bin/lora-e5-dev/periph/timer.o
                0x000000000800269c                timer_set_absolute
 .text.timer_clear
                0x00000000080026d4       0x28 /home/ch/RIOT/examples/lorawan/bin/lora-e5-dev/periph/timer.o
                0x00000000080026d4                timer_clear
 .text.timer_read
                0x00000000080026fc       0x10 /home/ch/RIOT/examples/lorawan/bin/lora-e5-dev/periph/timer.o
                0x00000000080026fc                timer_read
 .text.timer_start
                0x000000000800270c       0x14 /home/ch/RIOT/examples/lorawan/bin/lora-e5-dev/periph/timer.o
                0x000000000800270c                timer_start
 .text.timer_init
                0x0000000008002720       0x54 /home/ch/RIOT/examples/lorawan/bin/lora-e5-dev/periph/timer.o
                0x0000000008002720                timer_init
 .text.isr_tim2
                0x0000000008002774       0x74 /home/ch/RIOT/examples/lorawan/bin/lora-e5-dev/periph/timer.o
                0x0000000008002774                isr_tim2
 .text.irq_handler
                0x00000000080027e8       0x54 /home/ch/RIOT/examples/lorawan/bin/lora-e5-dev/periph/uart.o
 .text.uart_enable_clock
                0x000000000800283c       0x30 /home/ch/RIOT/examples/lorawan/bin/lora-e5-dev/periph/uart.o
 .text.uart_init
                0x000000000800286c       0xa8 /home/ch/RIOT/examples/lorawan/bin/lora-e5-dev/periph/uart.o
                0x000000000800286c                uart_init
 .text.uart_write
                0x0000000008002914       0x40 /home/ch/RIOT/examples/lorawan/bin/lora-e5-dev/periph/uart.o
                0x0000000008002914                uart_write
 .text.isr_usart1
                0x0000000008002954        0x6 /home/ch/RIOT/examples/lorawan/bin/lora-e5-dev/periph/uart.o
                0x0000000008002954                isr_usart1
 .text.isr_usart2
                0x000000000800295a        0x6 /home/ch/RIOT/examples/lorawan/bin/lora-e5-dev/periph/uart.o
                0x000000000800295a                isr_usart2
 .text.isr_lpuart1
                0x0000000008002960        0x6 /home/ch/RIOT/examples/lorawan/bin/lora-e5-dev/periph/uart.o
                0x0000000008002960                isr_lpuart1
 *fill*         0x0000000008002966        0x2 
 .text.pm_set_lowest
                0x0000000008002968       0x3c /home/ch/RIOT/examples/lorawan/bin/lora-e5-dev/pm_layered/pm.o
                0x0000000008002968                pm_set_lowest
 .text.pm_block
                0x00000000080029a4       0x2c /home/ch/RIOT/examples/lorawan/bin/lora-e5-dev/pm_layered/pm.o
                0x00000000080029a4                pm_block
 .text.pm_unblock
                0x00000000080029d0       0x2c /home/ch/RIOT/examples/lorawan/bin/lora-e5-dev/pm_layered/pm.o
                0x00000000080029d0                pm_unblock
 .text.pm_off   0x00000000080029fc       0x10 /home/ch/RIOT/examples/lorawan/bin/lora-e5-dev/pm_layered/pm.o
                0x00000000080029fc                pm_off
 .text.random_init
                0x0000000008002a0c       0x10 /home/ch/RIOT/examples/lorawan/bin/lora-e5-dev/random/musl_lcg.o
                0x0000000008002a0c                random_init
 .text.random_uint32
                0x0000000008002a1c       0x30 /home/ch/RIOT/examples/lorawan/bin/lora-e5-dev/random/musl_lcg.o
                0x0000000008002a1c                random_uint32
 .text.auto_init_random
                0x0000000008002a4c       0x18 /home/ch/RIOT/examples/lorawan/bin/lora-e5-dev/random/random.o
                0x0000000008002a4c                auto_init_random
 .text.random_uint32_range
                0x0000000008002a64       0x48 /home/ch/RIOT/examples/lorawan/bin/lora-e5-dev/random/random.o
                0x0000000008002a64                random_uint32_range
 .text.srand1   0x0000000008002aac        0x2 /home/ch/RIOT/examples/lorawan/bin/lora-e5-dev/semtech_loramac_arch/utilities.o
                0x0000000008002aac                srand1
 .text.randr    0x0000000008002aae       0x16 /home/ch/RIOT/examples/lorawan/bin/lora-e5-dev/semtech_loramac_arch/utilities.o
                0x0000000008002aae                randr
 .text.memcpy1  0x0000000008002ac4        0x4 /home/ch/RIOT/examples/lorawan/bin/lora-e5-dev/semtech_loramac_arch/utilities.o
                0x0000000008002ac4                memcpy1
 .text.memcpyr  0x0000000008002ac8       0x14 /home/ch/RIOT/examples/lorawan/bin/lora-e5-dev/semtech_loramac_arch/utilities.o
                0x0000000008002ac8                memcpyr
 .text.memset1  0x0000000008002adc        0x4 /home/ch/RIOT/examples/lorawan/bin/lora-e5-dev/semtech_loramac_arch/utilities.o
                0x0000000008002adc                memset1
 .text._semtech_loramac_set_rx2_params.isra.0
                0x0000000008002ae0       0x30 /home/ch/RIOT/examples/lorawan/bin/lora-e5-dev/semtech_loramac_contrib/semtech_loramac_getset.o
 .text.semtech_loramac_set_deveui
                0x0000000008002b10        0x8 /home/ch/RIOT/examples/lorawan/bin/lora-e5-dev/semtech_loramac_contrib/semtech_loramac_getset.o
                0x0000000008002b10                semtech_loramac_set_deveui
 .text.semtech_loramac_set_appeui
                0x0000000008002b18        0x8 /home/ch/RIOT/examples/lorawan/bin/lora-e5-dev/semtech_loramac_contrib/semtech_loramac_getset.o
                0x0000000008002b18                semtech_loramac_set_appeui
 .text.semtech_loramac_set_appkey
                0x0000000008002b20        0x8 /home/ch/RIOT/examples/lorawan/bin/lora-e5-dev/semtech_loramac_contrib/semtech_loramac_getset.o
                0x0000000008002b20                semtech_loramac_set_appkey
 .text.semtech_loramac_set_class
                0x0000000008002b28       0x28 /home/ch/RIOT/examples/lorawan/bin/lora-e5-dev/semtech_loramac_contrib/semtech_loramac_getset.o
                0x0000000008002b28                semtech_loramac_set_class
 .text.semtech_loramac_set_dr
                0x0000000008002b50       0x28 /home/ch/RIOT/examples/lorawan/bin/lora-e5-dev/semtech_loramac_contrib/semtech_loramac_getset.o
                0x0000000008002b50                semtech_loramac_set_dr
 .text.semtech_loramac_get_dr
                0x0000000008002b78       0x28 /home/ch/RIOT/examples/lorawan/bin/lora-e5-dev/semtech_loramac_contrib/semtech_loramac_getset.o
                0x0000000008002b78                semtech_loramac_get_dr
 .text.semtech_loramac_set_adr
                0x0000000008002ba0       0x28 /home/ch/RIOT/examples/lorawan/bin/lora-e5-dev/semtech_loramac_contrib/semtech_loramac_getset.o
                0x0000000008002ba0                semtech_loramac_set_adr
 .text.semtech_loramac_set_public_network
                0x0000000008002bc8       0x28 /home/ch/RIOT/examples/lorawan/bin/lora-e5-dev/semtech_loramac_contrib/semtech_loramac_getset.o
                0x0000000008002bc8                semtech_loramac_set_public_network
 .text.semtech_loramac_set_netid
                0x0000000008002bf0       0x26 /home/ch/RIOT/examples/lorawan/bin/lora-e5-dev/semtech_loramac_contrib/semtech_loramac_getset.o
                0x0000000008002bf0                semtech_loramac_set_netid
 .text.semtech_loramac_set_tx_port
                0x0000000008002c16        0x4 /home/ch/RIOT/examples/lorawan/bin/lora-e5-dev/semtech_loramac_contrib/semtech_loramac_getset.o
                0x0000000008002c16                semtech_loramac_set_tx_port
 .text.semtech_loramac_set_tx_mode
                0x0000000008002c1a        0x4 /home/ch/RIOT/examples/lorawan/bin/lora-e5-dev/semtech_loramac_contrib/semtech_loramac_getset.o
                0x0000000008002c1a                semtech_loramac_set_tx_mode
 .text.semtech_loramac_set_system_max_rx_error
                0x0000000008002c1e       0x26 /home/ch/RIOT/examples/lorawan/bin/lora-e5-dev/semtech_loramac_contrib/semtech_loramac_getset.o
                0x0000000008002c1e                semtech_loramac_set_system_max_rx_error
 .text.semtech_loramac_set_min_rx_symbols
                0x0000000008002c44       0x28 /home/ch/RIOT/examples/lorawan/bin/lora-e5-dev/semtech_loramac_contrib/semtech_loramac_getset.o
                0x0000000008002c44                semtech_loramac_set_min_rx_symbols
 .text.semtech_loramac_set_rx2_dr
                0x0000000008002c6c       0x2c /home/ch/RIOT/examples/lorawan/bin/lora-e5-dev/semtech_loramac_contrib/semtech_loramac_getset.o
                0x0000000008002c6c                semtech_loramac_set_rx2_dr
 .text.mlme_indication
                0x0000000008002c98       0x24 /home/ch/RIOT/examples/lorawan/bin/lora-e5-dev/semtech_loramac_contrib/semtech_loramac.o
 .text.mlme_confirm
                0x0000000008002cbc       0x24 /home/ch/RIOT/examples/lorawan/bin/lora-e5-dev/semtech_loramac_contrib/semtech_loramac.o
 .text.mcps_indication
                0x0000000008002ce0       0x24 /home/ch/RIOT/examples/lorawan/bin/lora-e5-dev/semtech_loramac_contrib/semtech_loramac.o
 .text.mcps_confirm
                0x0000000008002d04       0x24 /home/ch/RIOT/examples/lorawan/bin/lora-e5-dev/semtech_loramac_contrib/semtech_loramac.o
 .text._semtech_loramac_event_cb
                0x0000000008002d28       0x9c /home/ch/RIOT/examples/lorawan/bin/lora-e5-dev/semtech_loramac_contrib/semtech_loramac.o
 .text._semtech_loramac_event_loop
                0x0000000008002dc4       0xf0 /home/ch/RIOT/examples/lorawan/bin/lora-e5-dev/semtech_loramac_contrib/semtech_loramac.o
                0x0000000008002dc4                _semtech_loramac_event_loop
 .text._join    0x0000000008002eb4       0xd4 /home/ch/RIOT/examples/lorawan/bin/lora-e5-dev/semtech_loramac_contrib/semtech_loramac.o
 .text._send    0x0000000008002f88       0x98 /home/ch/RIOT/examples/lorawan/bin/lora-e5-dev/semtech_loramac_contrib/semtech_loramac.o
 .text._init_loramac
                0x0000000008003020       0x8c /home/ch/RIOT/examples/lorawan/bin/lora-e5-dev/semtech_loramac_contrib/semtech_loramac.o
                0x0000000008003020                _init_loramac
 .text.semtech_loramac_init
                0x00000000080030ac       0x64 /home/ch/RIOT/examples/lorawan/bin/lora-e5-dev/semtech_loramac_contrib/semtech_loramac.o
                0x00000000080030ac                semtech_loramac_init
 .text.semtech_loramac_is_mac_joined
                0x0000000008003110       0x28 /home/ch/RIOT/examples/lorawan/bin/lora-e5-dev/semtech_loramac_contrib/semtech_loramac.o
                0x0000000008003110                semtech_loramac_is_mac_joined
 .text.semtech_loramac_join
                0x0000000008003138       0x58 /home/ch/RIOT/examples/lorawan/bin/lora-e5-dev/semtech_loramac_contrib/semtech_loramac.o
                0x0000000008003138                semtech_loramac_join
 .text.semtech_loramac_send
                0x0000000008003190       0x5c /home/ch/RIOT/examples/lorawan/bin/lora-e5-dev/semtech_loramac_contrib/semtech_loramac.o
                0x0000000008003190                semtech_loramac_send
 .text.SX127XGetStatus
                0x00000000080031ec       0x38 /home/ch/RIOT/examples/lorawan/bin/lora-e5-dev/semtech_loramac_contrib/semtech_loramac_radio.o
                0x00000000080031ec                SX127XGetStatus
 .text.SX127XSetModem
                0x0000000008003224       0x24 /home/ch/RIOT/examples/lorawan/bin/lora-e5-dev/semtech_loramac_contrib/semtech_loramac_radio.o
                0x0000000008003224                SX127XSetModem
 .text.SX127XSetChannel
                0x0000000008003248       0x20 /home/ch/RIOT/examples/lorawan/bin/lora-e5-dev/semtech_loramac_contrib/semtech_loramac_radio.o
                0x0000000008003248                SX127XSetChannel
 .text.SX127XRandom
                0x0000000008003268       0x20 /home/ch/RIOT/examples/lorawan/bin/lora-e5-dev/semtech_loramac_contrib/semtech_loramac_radio.o
                0x0000000008003268                SX127XRandom
 .text.SX127XSetRxConfig
                0x0000000008003288      0x108 /home/ch/RIOT/examples/lorawan/bin/lora-e5-dev/semtech_loramac_contrib/semtech_loramac_radio.o
                0x0000000008003288                SX127XSetRxConfig
 .text.SX127XSetTxConfig
                0x0000000008003390       0xe8 /home/ch/RIOT/examples/lorawan/bin/lora-e5-dev/semtech_loramac_contrib/semtech_loramac_radio.o
                0x0000000008003390                SX127XSetTxConfig
 .text.SX127XSend
                0x0000000008003478       0x20 /home/ch/RIOT/examples/lorawan/bin/lora-e5-dev/semtech_loramac_contrib/semtech_loramac_radio.o
                0x0000000008003478                SX127XSend
 .text.SX127XSleep
                0x0000000008003498       0x20 /home/ch/RIOT/examples/lorawan/bin/lora-e5-dev/semtech_loramac_contrib/semtech_loramac_radio.o
                0x0000000008003498                SX127XSleep
 .text.SX127XStandby
                0x00000000080034b8       0x24 /home/ch/RIOT/examples/lorawan/bin/lora-e5-dev/semtech_loramac_contrib/semtech_loramac_radio.o
                0x00000000080034b8                SX127XStandby
 .text.SX127XRx
                0x00000000080034dc       0x38 /home/ch/RIOT/examples/lorawan/bin/lora-e5-dev/semtech_loramac_contrib/semtech_loramac_radio.o
                0x00000000080034dc                SX127XRx
 .text.SX127XStartCad
                0x0000000008003514        0x2 /home/ch/RIOT/examples/lorawan/bin/lora-e5-dev/semtech_loramac_contrib/semtech_loramac_radio.o
                0x0000000008003514                SX127XStartCad
 *fill*         0x0000000008003516        0x2 
 .text.SX127XRssi
                0x0000000008003518       0x20 /home/ch/RIOT/examples/lorawan/bin/lora-e5-dev/semtech_loramac_contrib/semtech_loramac_radio.o
                0x0000000008003518                SX127XRssi
 .text.SX127XWrite
                0x0000000008003538        0x2 /home/ch/RIOT/examples/lorawan/bin/lora-e5-dev/semtech_loramac_contrib/semtech_loramac_radio.o
                0x0000000008003538                SX127XWrite
 .text.SX127XRead
                0x000000000800353a        0x4 /home/ch/RIOT/examples/lorawan/bin/lora-e5-dev/semtech_loramac_contrib/semtech_loramac_radio.o
                0x000000000800353a                SX127XRead
 .text.SX127XWriteBuffer
                0x000000000800353e        0x2 /home/ch/RIOT/examples/lorawan/bin/lora-e5-dev/semtech_loramac_contrib/semtech_loramac_radio.o
                0x000000000800353e                SX127XWriteBuffer
 .text.SX127XSetMaxPayloadLength
                0x0000000008003540       0x20 /home/ch/RIOT/examples/lorawan/bin/lora-e5-dev/semtech_loramac_contrib/semtech_loramac_radio.o
                0x0000000008003540                SX127XSetMaxPayloadLength
 .text.SX127XCheckRfFrequency
                0x0000000008003560        0x4 /home/ch/RIOT/examples/lorawan/bin/lora-e5-dev/semtech_loramac_contrib/semtech_loramac_radio.o
                0x0000000008003560                SX127XCheckRfFrequency
 .text.SX127XSetTxContinuousWave
                0x0000000008003564        0x2 /home/ch/RIOT/examples/lorawan/bin/lora-e5-dev/semtech_loramac_contrib/semtech_loramac_radio.o
                0x0000000008003564                SX127XSetTxContinuousWave
 *fill*         0x0000000008003566        0x2 
 .text.SX127XSetPublicNetwork
                0x0000000008003568       0x28 /home/ch/RIOT/examples/lorawan/bin/lora-e5-dev/semtech_loramac_contrib/semtech_loramac_radio.o
                0x0000000008003568                SX127XSetPublicNetwork
 .text.SX127XGetWakeupTime
                0x0000000008003590        0x4 /home/ch/RIOT/examples/lorawan/bin/lora-e5-dev/semtech_loramac_contrib/semtech_loramac_radio.o
                0x0000000008003590                SX127XGetWakeupTime
 .text.SX127XRxBoosted
                0x0000000008003594        0x2 /home/ch/RIOT/examples/lorawan/bin/lora-e5-dev/semtech_loramac_contrib/semtech_loramac_radio.o
                0x0000000008003594                SX127XRxBoosted
 .text.SX127XSetRxDutyCycle
                0x0000000008003596        0x2 /home/ch/RIOT/examples/lorawan/bin/lora-e5-dev/semtech_loramac_contrib/semtech_loramac_radio.o
                0x0000000008003596                SX127XSetRxDutyCycle
 .text.SX127XIsChannelFree
                0x0000000008003598       0x50 /home/ch/RIOT/examples/lorawan/bin/lora-e5-dev/semtech_loramac_contrib/semtech_loramac_radio.o
                0x0000000008003598                SX127XIsChannelFree
 .text.SX127XTimeOnAir
                0x00000000080035e8       0xcc /home/ch/RIOT/examples/lorawan/bin/lora-e5-dev/semtech_loramac_contrib/semtech_loramac_radio.o
                0x00000000080035e8                SX127XTimeOnAir
 .text.SX127XInit
                0x00000000080036b4       0x24 /home/ch/RIOT/examples/lorawan/bin/lora-e5-dev/semtech_loramac_contrib/semtech_loramac_radio.o
                0x00000000080036b4                SX127XInit
 .text.SX127XReadBuffer
                0x00000000080036d8        0x2 /home/ch/RIOT/examples/lorawan/bin/lora-e5-dev/semtech_loramac_contrib/semtech_loramac_radio.o
                0x00000000080036d8                SX127XReadBuffer
 .text.SX127XIrqProcess
                0x00000000080036da        0x2 /home/ch/RIOT/examples/lorawan/bin/lora-e5-dev/semtech_loramac_contrib/semtech_loramac_radio.o
                0x00000000080036da                SX127XIrqProcess
 .text.ztimer_now
                0x00000000080036dc       0x10 /home/ch/RIOT/examples/lorawan/bin/lora-e5-dev/semtech_loramac_contrib/semtech_loramac_timer.o
 .text.TimerInit
                0x00000000080036ec       0x18 /home/ch/RIOT/examples/lorawan/bin/lora-e5-dev/semtech_loramac_contrib/semtech_loramac_timer.o
                0x00000000080036ec                TimerInit
 .text.TimerStart
                0x0000000008003704       0x38 /home/ch/RIOT/examples/lorawan/bin/lora-e5-dev/semtech_loramac_contrib/semtech_loramac_timer.o
                0x0000000008003704                TimerStart
 .text.TimerStop
                0x000000000800373c       0x14 /home/ch/RIOT/examples/lorawan/bin/lora-e5-dev/semtech_loramac_contrib/semtech_loramac_timer.o
                0x000000000800373c                TimerStop
 .text.TimerSetValue
                0x0000000008003750       0x20 /home/ch/RIOT/examples/lorawan/bin/lora-e5-dev/semtech_loramac_contrib/semtech_loramac_timer.o
                0x0000000008003750                TimerSetValue
 .text.TimerGetCurrentTime
                0x0000000008003770        0xc /home/ch/RIOT/examples/lorawan/bin/lora-e5-dev/semtech_loramac_contrib/semtech_loramac_timer.o
                0x0000000008003770                TimerGetCurrentTime
 .text.TimerGetElapsedTime
                0x000000000800377c       0x14 /home/ch/RIOT/examples/lorawan/bin/lora-e5-dev/semtech_loramac_contrib/semtech_loramac_timer.o
                0x000000000800377c                TimerGetElapsedTime
 .text.AES_CMAC_Init
                0x0000000008003790       0x14 /home/ch/RIOT/examples/lorawan/bin/lora-e5-dev/semtech_loramac_crypto/cmac.o
                0x0000000008003790                AES_CMAC_Init
 .text.AES_CMAC_SetKey
                0x00000000080037a4        0x6 /home/ch/RIOT/examples/lorawan/bin/lora-e5-dev/semtech_loramac_crypto/cmac.o
                0x00000000080037a4                AES_CMAC_SetKey
 .text.AES_CMAC_Update
                0x00000000080037aa       0xb0 /home/ch/RIOT/examples/lorawan/bin/lora-e5-dev/semtech_loramac_crypto/cmac.o
                0x00000000080037aa                AES_CMAC_Update
 .text.AES_CMAC_Final
                0x000000000800385a      0x15e /home/ch/RIOT/examples/lorawan/bin/lora-e5-dev/semtech_loramac_crypto/cmac.o
                0x000000000800385a                AES_CMAC_Final
 .text.LoRaMacComputeMic
                0x00000000080039b8       0x78 /home/ch/RIOT/examples/lorawan/bin/lora-e5-dev/semtech_loramac_mac/LoRaMacCrypto.o
                0x00000000080039b8                LoRaMacComputeMic
 .text.LoRaMacPayloadEncrypt
                0x0000000008003a30       0xd8 /home/ch/RIOT/examples/lorawan/bin/lora-e5-dev/semtech_loramac_mac/LoRaMacCrypto.o
                0x0000000008003a30                LoRaMacPayloadEncrypt
 .text.LoRaMacPayloadDecrypt
                0x0000000008003b08        0xe /home/ch/RIOT/examples/lorawan/bin/lora-e5-dev/semtech_loramac_mac/LoRaMacCrypto.o
                0x0000000008003b08                LoRaMacPayloadDecrypt
 *fill*         0x0000000008003b16        0x2 
 .text.LoRaMacJoinComputeMic
                0x0000000008003b18       0x40 /home/ch/RIOT/examples/lorawan/bin/lora-e5-dev/semtech_loramac_mac/LoRaMacCrypto.o
                0x0000000008003b18                LoRaMacJoinComputeMic
 .text.LoRaMacJoinDecrypt
                0x0000000008003b58       0x38 /home/ch/RIOT/examples/lorawan/bin/lora-e5-dev/semtech_loramac_mac/LoRaMacCrypto.o
                0x0000000008003b58                LoRaMacJoinDecrypt
 .text.LoRaMacJoinComputeSKeys
                0x0000000008003b90       0x88 /home/ch/RIOT/examples/lorawan/bin/lora-e5-dev/semtech_loramac_mac/LoRaMacCrypto.o
                0x0000000008003b90                LoRaMacJoinComputeSKeys
 .text.ValidatePayloadLength
                0x0000000008003c18       0x54 /home/ch/RIOT/examples/lorawan/bin/lora-e5-dev/semtech_loramac_mac/LoRaMac.o
 .text.ResetMacParameters
                0x0000000008003c6c       0xe8 /home/ch/RIOT/examples/lorawan/bin/lora-e5-dev/semtech_loramac_mac/LoRaMac.o
 .text.OnAckTimeoutTimerEvent
                0x0000000008003d54       0x4c /home/ch/RIOT/examples/lorawan/bin/lora-e5-dev/semtech_loramac_mac/LoRaMac.o
 .text.OnRxWindow1TimerEvent
                0x0000000008003da0       0x80 /home/ch/RIOT/examples/lorawan/bin/lora-e5-dev/semtech_loramac_mac/LoRaMac.o
 .text.OnRxWindow2TimerEvent
                0x0000000008003e20       0x80 /home/ch/RIOT/examples/lorawan/bin/lora-e5-dev/semtech_loramac_mac/LoRaMac.o
 .text.OpenContinuousRx2Window
                0x0000000008003ea0       0x14 /home/ch/RIOT/examples/lorawan/bin/lora-e5-dev/semtech_loramac_mac/LoRaMac.o
 .text.OnRadioRxTimeout
                0x0000000008003eb4       0xa4 /home/ch/RIOT/examples/lorawan/bin/lora-e5-dev/semtech_loramac_mac/LoRaMac.o
 .text.OnRadioTxTimeout
                0x0000000008003f58       0x40 /home/ch/RIOT/examples/lorawan/bin/lora-e5-dev/semtech_loramac_mac/LoRaMac.o
 .text.OnRadioRxError
                0x0000000008003f98       0xa4 /home/ch/RIOT/examples/lorawan/bin/lora-e5-dev/semtech_loramac_mac/LoRaMac.o
 .text.OnRadioTxDone
                0x000000000800403c      0x144 /home/ch/RIOT/examples/lorawan/bin/lora-e5-dev/semtech_loramac_mac/LoRaMac.o
 .text.ProcessMacCommands
                0x0000000008004180      0x450 /home/ch/RIOT/examples/lorawan/bin/lora-e5-dev/semtech_loramac_mac/LoRaMac.o
 .text.PrepareFrame
                0x00000000080045d0      0x388 /home/ch/RIOT/examples/lorawan/bin/lora-e5-dev/semtech_loramac_mac/LoRaMac.o
                0x00000000080045d0                PrepareFrame
 .text.SendFrameOnChannel
                0x0000000008004958       0xb8 /home/ch/RIOT/examples/lorawan/bin/lora-e5-dev/semtech_loramac_mac/LoRaMac.o
                0x0000000008004958                SendFrameOnChannel
 .text.ScheduleTx
                0x0000000008004a10      0x1a0 /home/ch/RIOT/examples/lorawan/bin/lora-e5-dev/semtech_loramac_mac/LoRaMac.o
 .text.Send     0x0000000008004bb0       0x48 /home/ch/RIOT/examples/lorawan/bin/lora-e5-dev/semtech_loramac_mac/LoRaMac.o
                0x0000000008004bb0                Send
 .text.OnTxDelayedTimerEvent
                0x0000000008004bf8       0x24 /home/ch/RIOT/examples/lorawan/bin/lora-e5-dev/semtech_loramac_mac/LoRaMac.o
 .text.OnMacStateCheckTimerEvent
                0x0000000008004c1c      0x2e0 /home/ch/RIOT/examples/lorawan/bin/lora-e5-dev/semtech_loramac_mac/LoRaMac.o
 .text.PrepareRxDoneAbort
                0x0000000008004efc       0x38 /home/ch/RIOT/examples/lorawan/bin/lora-e5-dev/semtech_loramac_mac/LoRaMac.o
 .text.OnRadioRxDone
                0x0000000008004f34      0x508 /home/ch/RIOT/examples/lorawan/bin/lora-e5-dev/semtech_loramac_mac/LoRaMac.o
 .text.SetTxContinuousWave
                0x000000000800543c       0x64 /home/ch/RIOT/examples/lorawan/bin/lora-e5-dev/semtech_loramac_mac/LoRaMac.o
                0x000000000800543c                SetTxContinuousWave
 .text.SetTxContinuousWave1
                0x00000000080054a0       0x40 /home/ch/RIOT/examples/lorawan/bin/lora-e5-dev/semtech_loramac_mac/LoRaMac.o
                0x00000000080054a0                SetTxContinuousWave1
 .text.LoRaMacInitialization
                0x00000000080054e0      0x294 /home/ch/RIOT/examples/lorawan/bin/lora-e5-dev/semtech_loramac_mac/LoRaMac.o
                0x00000000080054e0                LoRaMacInitialization
 .text.LoRaMacQueryTxPossible
                0x0000000008005774       0xf0 /home/ch/RIOT/examples/lorawan/bin/lora-e5-dev/semtech_loramac_mac/LoRaMac.o
                0x0000000008005774                LoRaMacQueryTxPossible
 .text.LoRaMacMibGetRequestConfirm
                0x0000000008005864      0x140 /home/ch/RIOT/examples/lorawan/bin/lora-e5-dev/semtech_loramac_mac/LoRaMac.o
                0x0000000008005864                LoRaMacMibGetRequestConfirm
 .text.LoRaMacMibSetRequestConfirm
                0x00000000080059a4      0x2e8 /home/ch/RIOT/examples/lorawan/bin/lora-e5-dev/semtech_loramac_mac/LoRaMac.o
                0x00000000080059a4                LoRaMacMibSetRequestConfirm
 .text.LoRaMacMlmeRequest
                0x0000000008005c8c      0x140 /home/ch/RIOT/examples/lorawan/bin/lora-e5-dev/semtech_loramac_mac/LoRaMac.o
                0x0000000008005c8c                LoRaMacMlmeRequest
 .text.LoRaMacMcpsRequest
                0x0000000008005dcc      0x148 /home/ch/RIOT/examples/lorawan/bin/lora-e5-dev/semtech_loramac_mac/LoRaMac.o
                0x0000000008005dcc                LoRaMacMcpsRequest
 .text.RegionCommonGetJoinDc
                0x0000000008005f14       0x24 /home/ch/RIOT/examples/lorawan/bin/lora-e5-dev/semtech_loramac_mac_region/RegionCommon.o
                0x0000000008005f14                RegionCommonGetJoinDc
 .text.RegionCommonChanVerifyDr
                0x0000000008005f38       0x68 /home/ch/RIOT/examples/lorawan/bin/lora-e5-dev/semtech_loramac_mac_region/RegionCommon.o
                0x0000000008005f38                RegionCommonChanVerifyDr
 .text.RegionCommonValueInRange
                0x0000000008005fa0       0x12 /home/ch/RIOT/examples/lorawan/bin/lora-e5-dev/semtech_loramac_mac_region/RegionCommon.o
                0x0000000008005fa0                RegionCommonValueInRange
 .text.RegionCommonChanDisable
                0x0000000008005fb2       0x32 /home/ch/RIOT/examples/lorawan/bin/lora-e5-dev/semtech_loramac_mac_region/RegionCommon.o
                0x0000000008005fb2                RegionCommonChanDisable
 .text.RegionCommonCountChannels
                0x0000000008005fe4       0x3c /home/ch/RIOT/examples/lorawan/bin/lora-e5-dev/semtech_loramac_mac_region/RegionCommon.o
                0x0000000008005fe4                RegionCommonCountChannels
 .text.RegionCommonChanMaskCopy
                0x0000000008006020       0x1e /home/ch/RIOT/examples/lorawan/bin/lora-e5-dev/semtech_loramac_mac_region/RegionCommon.o
                0x0000000008006020                RegionCommonChanMaskCopy
 .text.RegionCommonSetBandTxDone
                0x000000000800603e        0xa /home/ch/RIOT/examples/lorawan/bin/lora-e5-dev/semtech_loramac_mac_region/RegionCommon.o
                0x000000000800603e                RegionCommonSetBandTxDone
 .text.RegionCommonUpdateBandTimeOff
                0x0000000008006048       0x9c /home/ch/RIOT/examples/lorawan/bin/lora-e5-dev/semtech_loramac_mac_region/RegionCommon.o
                0x0000000008006048                RegionCommonUpdateBandTimeOff
 .text.RegionCommonParseLinkAdrReq
                0x00000000080060e4       0x34 /home/ch/RIOT/examples/lorawan/bin/lora-e5-dev/semtech_loramac_mac_region/RegionCommon.o
                0x00000000080060e4                RegionCommonParseLinkAdrReq
 .text.RegionCommonLinkAdrReqVerifyParams
                0x0000000008006118       0x8e /home/ch/RIOT/examples/lorawan/bin/lora-e5-dev/semtech_loramac_mac_region/RegionCommon.o
                0x0000000008006118                RegionCommonLinkAdrReqVerifyParams
 *fill*         0x00000000080061a6        0x2 
 .text.RegionCommonComputeSymbolTimeLoRa
                0x00000000080061a8       0x34 /home/ch/RIOT/examples/lorawan/bin/lora-e5-dev/semtech_loramac_mac_region/RegionCommon.o
                0x00000000080061a8                RegionCommonComputeSymbolTimeLoRa
 .text.RegionCommonComputeSymbolTimeFsk
                0x00000000080061dc       0x18 /home/ch/RIOT/examples/lorawan/bin/lora-e5-dev/semtech_loramac_mac_region/RegionCommon.o
                0x00000000080061dc                RegionCommonComputeSymbolTimeFsk
 .text.RegionCommonComputeRxWindowParameters
                0x00000000080061f4       0xbc /home/ch/RIOT/examples/lorawan/bin/lora-e5-dev/semtech_loramac_mac_region/RegionCommon.o
                0x00000000080061f4                RegionCommonComputeRxWindowParameters
 .text.RegionCommonComputeTxPower
                0x00000000080062b0       0x2a /home/ch/RIOT/examples/lorawan/bin/lora-e5-dev/semtech_loramac_mac_region/RegionCommon.o
                0x00000000080062b0                RegionCommonComputeTxPower
 .text.RegionCommonCalcBackOff
                0x00000000080062da       0x4a /home/ch/RIOT/examples/lorawan/bin/lora-e5-dev/semtech_loramac_mac_region/RegionCommon.o
                0x00000000080062da                RegionCommonCalcBackOff
 .text.VerifyTxFreq
                0x0000000008006324       0x98 /home/ch/RIOT/examples/lorawan/bin/lora-e5-dev/semtech_loramac_mac_region/RegionEU868.o
 .text.RegionEU868GetPhyParam
                0x00000000080063bc       0xc0 /home/ch/RIOT/examples/lorawan/bin/lora-e5-dev/semtech_loramac_mac_region/RegionEU868.o
                0x00000000080063bc                RegionEU868GetPhyParam
 .text.RegionEU868SetBandTxDone
                0x000000000800647c       0x24 /home/ch/RIOT/examples/lorawan/bin/lora-e5-dev/semtech_loramac_mac_region/RegionEU868.o
                0x000000000800647c                RegionEU868SetBandTxDone
 .text.RegionEU868InitDefaults
                0x00000000080064a0       0x68 /home/ch/RIOT/examples/lorawan/bin/lora-e5-dev/semtech_loramac_mac_region/RegionEU868.o
                0x00000000080064a0                RegionEU868InitDefaults
 .text.RegionEU868Verify
                0x0000000008006508       0x34 /home/ch/RIOT/examples/lorawan/bin/lora-e5-dev/semtech_loramac_mac_region/RegionEU868.o
                0x0000000008006508                RegionEU868Verify
 .text.RegionEU868ChanMaskSet
                0x000000000800653c       0x34 /home/ch/RIOT/examples/lorawan/bin/lora-e5-dev/semtech_loramac_mac_region/RegionEU868.o
                0x000000000800653c                RegionEU868ChanMaskSet
 .text.RegionEU868AdrNext
                0x0000000008006570       0x78 /home/ch/RIOT/examples/lorawan/bin/lora-e5-dev/semtech_loramac_mac_region/RegionEU868.o
                0x0000000008006570                RegionEU868AdrNext
 .text.RegionEU868ComputeRxWindowParameters
                0x00000000080065e8       0x84 /home/ch/RIOT/examples/lorawan/bin/lora-e5-dev/semtech_loramac_mac_region/RegionEU868.o
                0x00000000080065e8                RegionEU868ComputeRxWindowParameters
 .text.RegionEU868RxConfig
                0x000000000800666c       0xe0 /home/ch/RIOT/examples/lorawan/bin/lora-e5-dev/semtech_loramac_mac_region/RegionEU868.o
                0x000000000800666c                RegionEU868RxConfig
 .text.RegionEU868TxConfig
                0x000000000800674c      0x10c /home/ch/RIOT/examples/lorawan/bin/lora-e5-dev/semtech_loramac_mac_region/RegionEU868.o
                0x000000000800674c                RegionEU868TxConfig
 .text.RegionEU868LinkAdrReq
                0x0000000008006858      0x144 /home/ch/RIOT/examples/lorawan/bin/lora-e5-dev/semtech_loramac_mac_region/RegionEU868.o
                0x0000000008006858                RegionEU868LinkAdrReq
 .text.RegionEU868RxParamSetupReq
                0x000000000800699c       0x44 /home/ch/RIOT/examples/lorawan/bin/lora-e5-dev/semtech_loramac_mac_region/RegionEU868.o
                0x000000000800699c                RegionEU868RxParamSetupReq
 .text.RegionEU868TxParamSetupReq
                0x00000000080069e0        0x6 /home/ch/RIOT/examples/lorawan/bin/lora-e5-dev/semtech_loramac_mac_region/RegionEU868.o
                0x00000000080069e0                RegionEU868TxParamSetupReq
 *fill*         0x00000000080069e6        0x2 
 .text.RegionEU868DlChannelReq
                0x00000000080069e8       0x44 /home/ch/RIOT/examples/lorawan/bin/lora-e5-dev/semtech_loramac_mac_region/RegionEU868.o
                0x00000000080069e8                RegionEU868DlChannelReq
 .text.RegionEU868AlternateDr
                0x0000000008006a2c        0x2 /home/ch/RIOT/examples/lorawan/bin/lora-e5-dev/semtech_loramac_mac_region/RegionEU868.o
                0x0000000008006a2c                RegionEU868AlternateDr
 *fill*         0x0000000008006a2e        0x2 
 .text.RegionEU868CalcBackOff
                0x0000000008006a30       0x38 /home/ch/RIOT/examples/lorawan/bin/lora-e5-dev/semtech_loramac_mac_region/RegionEU868.o
                0x0000000008006a30                RegionEU868CalcBackOff
 .text.RegionEU868NextChannel
                0x0000000008006a68      0x114 /home/ch/RIOT/examples/lorawan/bin/lora-e5-dev/semtech_loramac_mac_region/RegionEU868.o
                0x0000000008006a68                RegionEU868NextChannel
 .text.RegionEU868ChannelAdd
                0x0000000008006b7c       0xe4 /home/ch/RIOT/examples/lorawan/bin/lora-e5-dev/semtech_loramac_mac_region/RegionEU868.o
                0x0000000008006b7c                RegionEU868ChannelAdd
 .text.RegionEU868ChannelsRemove
                0x0000000008006c60       0x30 /home/ch/RIOT/examples/lorawan/bin/lora-e5-dev/semtech_loramac_mac_region/RegionEU868.o
                0x0000000008006c60                RegionEU868ChannelsRemove
 .text.RegionEU868ApplyCFList
                0x0000000008006c90       0x78 /home/ch/RIOT/examples/lorawan/bin/lora-e5-dev/semtech_loramac_mac_region/RegionEU868.o
                0x0000000008006c90                RegionEU868ApplyCFList
 .text.RegionEU868NewChannelReq
                0x0000000008006d08       0x3c /home/ch/RIOT/examples/lorawan/bin/lora-e5-dev/semtech_loramac_mac_region/RegionEU868.o
                0x0000000008006d08                RegionEU868NewChannelReq
 .text.RegionEU868SetContinuousWave
                0x0000000008006d44       0x4c /home/ch/RIOT/examples/lorawan/bin/lora-e5-dev/semtech_loramac_mac_region/RegionEU868.o
                0x0000000008006d44                RegionEU868SetContinuousWave
 .text.RegionEU868ApplyDrOffset
                0x0000000008006d90        0xc /home/ch/RIOT/examples/lorawan/bin/lora-e5-dev/semtech_loramac_mac_region/RegionEU868.o
                0x0000000008006d90                RegionEU868ApplyDrOffset
 .text.RegionIsActive
                0x0000000008006d9c        0x8 /home/ch/RIOT/examples/lorawan/bin/lora-e5-dev/semtech_loramac_mac_region/Region.o
                0x0000000008006d9c                RegionIsActive
 .text.RegionGetPhyParam
                0x0000000008006da4        0xe /home/ch/RIOT/examples/lorawan/bin/lora-e5-dev/semtech_loramac_mac_region/Region.o
                0x0000000008006da4                RegionGetPhyParam
 .text.RegionSetBandTxDone
                0x0000000008006db2        0xc /home/ch/RIOT/examples/lorawan/bin/lora-e5-dev/semtech_loramac_mac_region/Region.o
                0x0000000008006db2                RegionSetBandTxDone
 .text.RegionInitDefaults
                0x0000000008006dbe        0xc /home/ch/RIOT/examples/lorawan/bin/lora-e5-dev/semtech_loramac_mac_region/Region.o
                0x0000000008006dbe                RegionInitDefaults
 .text.RegionVerify
                0x0000000008006dca       0x12 /home/ch/RIOT/examples/lorawan/bin/lora-e5-dev/semtech_loramac_mac_region/Region.o
                0x0000000008006dca                RegionVerify
 .text.RegionApplyCFList
                0x0000000008006ddc        0xc /home/ch/RIOT/examples/lorawan/bin/lora-e5-dev/semtech_loramac_mac_region/Region.o
                0x0000000008006ddc                RegionApplyCFList
 .text.RegionChanMaskSet
                0x0000000008006de8        0xe /home/ch/RIOT/examples/lorawan/bin/lora-e5-dev/semtech_loramac_mac_region/Region.o
                0x0000000008006de8                RegionChanMaskSet
 .text.RegionAdrNext
                0x0000000008006df6       0x1c /home/ch/RIOT/examples/lorawan/bin/lora-e5-dev/semtech_loramac_mac_region/Region.o
                0x0000000008006df6                RegionAdrNext
 .text.RegionComputeRxWindowParameters
                0x0000000008006e12       0x1a /home/ch/RIOT/examples/lorawan/bin/lora-e5-dev/semtech_loramac_mac_region/Region.o
                0x0000000008006e12                RegionComputeRxWindowParameters
 .text.RegionRxConfig
                0x0000000008006e2c       0x12 /home/ch/RIOT/examples/lorawan/bin/lora-e5-dev/semtech_loramac_mac_region/Region.o
                0x0000000008006e2c                RegionRxConfig
 .text.RegionTxConfig
                0x0000000008006e3e       0x1a /home/ch/RIOT/examples/lorawan/bin/lora-e5-dev/semtech_loramac_mac_region/Region.o
                0x0000000008006e3e                RegionTxConfig
 .text.RegionLinkAdrReq
                0x0000000008006e58       0x20 /home/ch/RIOT/examples/lorawan/bin/lora-e5-dev/semtech_loramac_mac_region/Region.o
                0x0000000008006e58                RegionLinkAdrReq
 .text.RegionRxParamSetupReq
                0x0000000008006e78        0xe /home/ch/RIOT/examples/lorawan/bin/lora-e5-dev/semtech_loramac_mac_region/Region.o
                0x0000000008006e78                RegionRxParamSetupReq
 .text.RegionNewChannelReq
                0x0000000008006e86        0xe /home/ch/RIOT/examples/lorawan/bin/lora-e5-dev/semtech_loramac_mac_region/Region.o
                0x0000000008006e86                RegionNewChannelReq
 .text.RegionTxParamSetupReq
                0x0000000008006e94        0xe /home/ch/RIOT/examples/lorawan/bin/lora-e5-dev/semtech_loramac_mac_region/Region.o
                0x0000000008006e94                RegionTxParamSetupReq
 .text.RegionDlChannelReq
                0x0000000008006ea2        0xe /home/ch/RIOT/examples/lorawan/bin/lora-e5-dev/semtech_loramac_mac_region/Region.o
                0x0000000008006ea2                RegionDlChannelReq
 .text.RegionAlternateDr
                0x0000000008006eb0        0xe /home/ch/RIOT/examples/lorawan/bin/lora-e5-dev/semtech_loramac_mac_region/Region.o
                0x0000000008006eb0                RegionAlternateDr
 .text.RegionCalcBackOff
                0x0000000008006ebe        0xc /home/ch/RIOT/examples/lorawan/bin/lora-e5-dev/semtech_loramac_mac_region/Region.o
                0x0000000008006ebe                RegionCalcBackOff
 .text.RegionNextChannel
                0x0000000008006eca       0x1c /home/ch/RIOT/examples/lorawan/bin/lora-e5-dev/semtech_loramac_mac_region/Region.o
                0x0000000008006eca                RegionNextChannel
 .text.RegionSetContinuousWave
                0x0000000008006ee6        0xc /home/ch/RIOT/examples/lorawan/bin/lora-e5-dev/semtech_loramac_mac_region/Region.o
                0x0000000008006ee6                RegionSetContinuousWave
 .text.RegionApplyDrOffset
                0x0000000008006ef2       0x1a /home/ch/RIOT/examples/lorawan/bin/lora-e5-dev/semtech_loramac_mac_region/Region.o
                0x0000000008006ef2                RegionApplyDrOffset
 .text.stdio_init
                0x0000000008006f0c        0xe /home/ch/RIOT/examples/lorawan/bin/lora-e5-dev/stdio_uart/stdio_uart.o
                0x0000000008006f0c                stdio_init
 .text.stdio_read
                0x0000000008006f1a        0x6 /home/ch/RIOT/examples/lorawan/bin/lora-e5-dev/stdio_uart/stdio_uart.o
                0x0000000008006f1a                stdio_read
 .text.stdio_write
                0x0000000008006f20       0x12 /home/ch/RIOT/examples/lorawan/bin/lora-e5-dev/stdio_uart/stdio_uart.o
                0x0000000008006f20                stdio_write
 .text.stmclk_enable_hsi
                0x0000000008006f32       0x14 /home/ch/RIOT/examples/lorawan/bin/lora-e5-dev/stm32_clk/stmclk_common.o
                0x0000000008006f32                stmclk_enable_hsi
 .text.stmclk_disable_hsi
                0x0000000008006f46        0xe /home/ch/RIOT/examples/lorawan/bin/lora-e5-dev/stm32_clk/stmclk_common.o
                0x0000000008006f46                stmclk_disable_hsi
 .text.stmclk_dbp_unlock
                0x0000000008006f54       0x10 /home/ch/RIOT/examples/lorawan/bin/lora-e5-dev/stm32_clk/stmclk_common.o
                0x0000000008006f54                stmclk_dbp_unlock
 .text.stmclk_dbp_lock
                0x0000000008006f64       0x10 /home/ch/RIOT/examples/lorawan/bin/lora-e5-dev/stm32_clk/stmclk_common.o
                0x0000000008006f64                stmclk_dbp_lock
 .text.stmclk_enable_lfclk
                0x0000000008006f74       0x3e /home/ch/RIOT/examples/lorawan/bin/lora-e5-dev/stm32_clk/stmclk_common.o
                0x0000000008006f74                stmclk_enable_lfclk
 *fill*         0x0000000008006fb2        0x2 
 .text.stmclk_init_sysclk
                0x0000000008006fb4       0xa8 /home/ch/RIOT/examples/lorawan/bin/lora-e5-dev/stm32_clk/stmclk_l4wx.o
                0x0000000008006fb4                stmclk_init_sysclk
 .text.dummy_handler
                0x000000000800705c        0x4 /home/ch/RIOT/examples/lorawan/bin/lora-e5-dev/stm32_vectors/STM32WLE5xx.o
                0x000000000800705c                isr_lptim2
                0x000000000800705c                isr_rtc_wkup
                0x000000000800705c                isr_hsem
                0x000000000800705c                isr_dac
                0x000000000800705c                isr_tim16
                0x000000000800705c                isr_dma1_channel4
                0x000000000800705c                isr_dma2_channel7
                0x000000000800705c                isr_i2c1_ev
                0x000000000800705c                isr_tim1_brk
                0x000000000800705c                isr_dma1_channel5
                0x000000000800705c                isr_dma1_channel2
                0x000000000800705c                isr_pka
                0x000000000800705c                isr_dma2_channel6
                0x000000000800705c                isr_dma1_channel7
                0x000000000800705c                isr_i2c3_ev
                0x000000000800705c                isr_tim1_up
                0x000000000800705c                isr_dma2_channel4
                0x000000000800705c                isr_spi2
                0x000000000800705c                isr_tim1_trg_com
                0x000000000800705c                isr_dma1_channel1
                0x000000000800705c                dummy_handler
                0x000000000800705c                isr_adc
                0x000000000800705c                isr_aes
                0x000000000800705c                isr_comp
                0x000000000800705c                isr_spi1
                0x000000000800705c                isr_rcc
                0x000000000800705c                isr_tamp_stamp_lsecss_ssru
                0x000000000800705c                isr_flash
                0x000000000800705c                isr_dma2_channel5
                0x000000000800705c                isr_i2c3_er
                0x000000000800705c                isr_tim1_cc
                0x000000000800705c                isr_lptim3
                0x000000000800705c                isr_subghzspi
                0x000000000800705c                isr_dma2_channel1
                0x000000000800705c                isr_tim17
                0x000000000800705c                isr_dma1_channel6
                0x000000000800705c                isr_pvd_pvm
                0x000000000800705c                isr_rng
                0x000000000800705c                isr_dmamux1_ovr
                0x000000000800705c                isr_i2c2_ev
                0x000000000800705c                isr_dma2_channel2
                0x000000000800705c                isr_dma2_channel3
                0x000000000800705c                isr_rtc_alarm
                0x000000000800705c                isr_dma1_channel3
                0x000000000800705c                isr_i2c1_er
                0x000000000800705c                isr_wwdg
 .text._set     0x0000000008007060      0x214 /home/ch/RIOT/examples/lorawan/bin/lora-e5-dev/sx126x/sx126x_netdev.o
 .text._get     0x0000000008007274      0x150 /home/ch/RIOT/examples/lorawan/bin/lora-e5-dev/sx126x/sx126x_netdev.o
 .text._recv    0x00000000080073c4       0x4c /home/ch/RIOT/examples/lorawan/bin/lora-e5-dev/sx126x/sx126x_netdev.o
 .text._send    0x0000000008007410       0x68 /home/ch/RIOT/examples/lorawan/bin/lora-e5-dev/sx126x/sx126x_netdev.o
 .text._isr     0x0000000008007478       0x7c /home/ch/RIOT/examples/lorawan/bin/lora-e5-dev/sx126x/sx126x_netdev.o
 .text._init    0x00000000080074f4       0x28 /home/ch/RIOT/examples/lorawan/bin/lora-e5-dev/sx126x/sx126x_netdev.o
 .text.isr_subghz_radio
                0x000000000800751c       0x48 /home/ch/RIOT/examples/lorawan/bin/lora-e5-dev/sx126x/sx126x_netdev.o
                0x000000000800751c                isr_subghz_radio
 .text.sx126x_setup
                0x0000000008007564        0xc /home/ch/RIOT/examples/lorawan/bin/lora-e5-dev/sx126x/sx126x.o
                0x0000000008007564                sx126x_setup
 .text.sx126x_get_channel
                0x0000000008007570        0x4 /home/ch/RIOT/examples/lorawan/bin/lora-e5-dev/sx126x/sx126x.o
                0x0000000008007570                sx126x_get_channel
 .text.sx126x_set_channel
                0x0000000008007574        0x6 /home/ch/RIOT/examples/lorawan/bin/lora-e5-dev/sx126x/sx126x.o
                0x0000000008007574                sx126x_set_channel
 *fill*         0x000000000800757a        0x2 
 .text.sx126x_init
                0x000000000800757c       0xb4 /home/ch/RIOT/examples/lorawan/bin/lora-e5-dev/sx126x/sx126x.o
                0x000000000800757c                sx126x_init
 .text.sx126x_get_bandwidth
                0x0000000008007630        0x8 /home/ch/RIOT/examples/lorawan/bin/lora-e5-dev/sx126x/sx126x.o
                0x0000000008007630                sx126x_get_bandwidth
 .text.sx126x_set_bandwidth
                0x0000000008007638       0x34 /home/ch/RIOT/examples/lorawan/bin/lora-e5-dev/sx126x/sx126x.o
                0x0000000008007638                sx126x_set_bandwidth
 .text.sx126x_get_spreading_factor
                0x000000000800766c        0x4 /home/ch/RIOT/examples/lorawan/bin/lora-e5-dev/sx126x/sx126x.o
                0x000000000800766c                sx126x_get_spreading_factor
 .text.sx126x_set_spreading_factor
                0x0000000008007670       0x30 /home/ch/RIOT/examples/lorawan/bin/lora-e5-dev/sx126x/sx126x.o
                0x0000000008007670                sx126x_set_spreading_factor
 .text.sx126x_get_coding_rate
                0x00000000080076a0        0x4 /home/ch/RIOT/examples/lorawan/bin/lora-e5-dev/sx126x/sx126x.o
                0x00000000080076a0                sx126x_get_coding_rate
 .text.sx126x_set_coding_rate
                0x00000000080076a4        0xa /home/ch/RIOT/examples/lorawan/bin/lora-e5-dev/sx126x/sx126x.o
                0x00000000080076a4                sx126x_set_coding_rate
 .text.sx126x_get_lora_payload_length
                0x00000000080076ae       0x12 /home/ch/RIOT/examples/lorawan/bin/lora-e5-dev/sx126x/sx126x.o
                0x00000000080076ae                sx126x_get_lora_payload_length
 .text.sx126x_set_lora_payload_length
                0x00000000080076c0        0xa /home/ch/RIOT/examples/lorawan/bin/lora-e5-dev/sx126x/sx126x.o
                0x00000000080076c0                sx126x_set_lora_payload_length
 .text.sx126x_get_lora_crc
                0x00000000080076ca        0x4 /home/ch/RIOT/examples/lorawan/bin/lora-e5-dev/sx126x/sx126x.o
                0x00000000080076ca                sx126x_get_lora_crc
 .text.sx126x_set_lora_crc
                0x00000000080076ce        0xa /home/ch/RIOT/examples/lorawan/bin/lora-e5-dev/sx126x/sx126x.o
                0x00000000080076ce                sx126x_set_lora_crc
 .text.sx126x_set_lora_implicit_header
                0x00000000080076d8        0xa /home/ch/RIOT/examples/lorawan/bin/lora-e5-dev/sx126x/sx126x.o
                0x00000000080076d8                sx126x_set_lora_implicit_header
 .text.sx126x_set_lora_preamble_length
                0x00000000080076e2        0xc /home/ch/RIOT/examples/lorawan/bin/lora-e5-dev/sx126x/sx126x.o
                0x00000000080076e2                sx126x_set_lora_preamble_length
 .text.sx126x_get_lora_iq_invert
                0x00000000080076ee        0x4 /home/ch/RIOT/examples/lorawan/bin/lora-e5-dev/sx126x/sx126x.o
                0x00000000080076ee                sx126x_get_lora_iq_invert
 .text.sx126x_set_lora_iq_invert
                0x00000000080076f2        0xa /home/ch/RIOT/examples/lorawan/bin/lora-e5-dev/sx126x/sx126x.o
                0x00000000080076f2                sx126x_set_lora_iq_invert
 .text._add_timer_to_list
                0x00000000080076fc       0x34 /home/ch/RIOT/examples/lorawan/bin/lora-e5-dev/xtimer/xtimer_core.o
 .text._remove_timer_from_list
                0x0000000008007730       0x18 /home/ch/RIOT/examples/lorawan/bin/lora-e5-dev/xtimer/xtimer_core.o
 .text.ztimer_now
                0x0000000008007748       0x10 /home/ch/RIOT/examples/lorawan/bin/lora-e5-dev/xtimer/xtimer_core.o
 .text._xtimer_now64
                0x0000000008007758       0x40 /home/ch/RIOT/examples/lorawan/bin/lora-e5-dev/xtimer/xtimer_core.o
 .text._schedule_earliest_lltimer
                0x0000000008007798       0x58 /home/ch/RIOT/examples/lorawan/bin/lora-e5-dev/xtimer/xtimer_core.o
 .text._xtimer_now
                0x00000000080077f0        0x8 /home/ch/RIOT/examples/lorawan/bin/lora-e5-dev/xtimer/xtimer_core.o
                0x00000000080077f0                _xtimer_now
 .text.xtimer_init
                0x00000000080077f8        0xe /home/ch/RIOT/examples/lorawan/bin/lora-e5-dev/xtimer/xtimer_core.o
                0x00000000080077f8                xtimer_init
 *fill*         0x0000000008007806        0x2 
 .text._ztimer_callback
                0x0000000008007808      0x118 /home/ch/RIOT/examples/lorawan/bin/lora-e5-dev/xtimer/xtimer_core.o
 .text.ztimer_convert_frac_op_now
                0x0000000008007920       0x3e /home/ch/RIOT/examples/lorawan/bin/lora-e5-dev/ztimer_core/convert_frac.o
 .text.ztimer_convert_frac_op_set
                0x000000000800795e       0x34 /home/ch/RIOT/examples/lorawan/bin/lora-e5-dev/ztimer_core/convert_frac.o
 *fill*         0x0000000008007992        0x2 
 .text.ztimer_convert_frac_init
                0x0000000008007994       0x9c /home/ch/RIOT/examples/lorawan/bin/lora-e5-dev/ztimer_core/convert_frac.o
                0x0000000008007994                ztimer_convert_frac_init
 .text.ztimer_convert_cancel
                0x0000000008007a30        0xa /home/ch/RIOT/examples/lorawan/bin/lora-e5-dev/ztimer_core/convert.o
                0x0000000008007a30                ztimer_convert_cancel
 .text._is_set  0x0000000008007a3a       0x18 /home/ch/RIOT/examples/lorawan/bin/lora-e5-dev/ztimer_core/core.o
 .text._now_next
                0x0000000008007a52       0x2a /home/ch/RIOT/examples/lorawan/bin/lora-e5-dev/ztimer_core/core.o
 .text._ztimer_update
                0x0000000008007a7c       0x28 /home/ch/RIOT/examples/lorawan/bin/lora-e5-dev/ztimer_core/core.o
 .text._del_entry_from_list
                0x0000000008007aa4       0x64 /home/ch/RIOT/examples/lorawan/bin/lora-e5-dev/ztimer_core/core.o
 .text._ztimer_now_extend
                0x0000000008007b08       0x40 /home/ch/RIOT/examples/lorawan/bin/lora-e5-dev/ztimer_core/core.o
                0x0000000008007b08                _ztimer_now_extend
 .text.ztimer_now
                0x0000000008007b48       0x10 /home/ch/RIOT/examples/lorawan/bin/lora-e5-dev/ztimer_core/core.o
 .text._ztimer_update_head_offset
                0x0000000008007b58       0x32 /home/ch/RIOT/examples/lorawan/bin/lora-e5-dev/ztimer_core/core.o
 .text.ztimer_remove
                0x0000000008007b8a       0x32 /home/ch/RIOT/examples/lorawan/bin/lora-e5-dev/ztimer_core/core.o
                0x0000000008007b8a                ztimer_remove
 .text.ztimer_set
                0x0000000008007bbc       0x9c /home/ch/RIOT/examples/lorawan/bin/lora-e5-dev/ztimer_core/core.o
                0x0000000008007bbc                ztimer_set
 .text.ztimer_handler
                0x0000000008007c58       0x94 /home/ch/RIOT/examples/lorawan/bin/lora-e5-dev/ztimer_core/core.o
                0x0000000008007c58                ztimer_handler
 .text.ztimer_init
                0x0000000008007cec       0x48 /home/ch/RIOT/examples/lorawan/bin/lora-e5-dev/ztimer_core/init.o
                0x0000000008007cec                ztimer_init
 .text._ztimer_periph_rtt_cancel
                0x0000000008007d34        0x4 /home/ch/RIOT/examples/lorawan/bin/lora-e5-dev/ztimer_core/periph_rtt.o
 .text._ztimer_periph_rtt_now
                0x0000000008007d38        0x4 /home/ch/RIOT/examples/lorawan/bin/lora-e5-dev/ztimer_core/periph_rtt.o
 .text._ztimer_periph_rtt_set
                0x0000000008007d3c       0x2c /home/ch/RIOT/examples/lorawan/bin/lora-e5-dev/ztimer_core/periph_rtt.o
 .text._ztimer_periph_rtt_callback
                0x0000000008007d68        0x4 /home/ch/RIOT/examples/lorawan/bin/lora-e5-dev/ztimer_core/periph_rtt.o
 .text.ztimer_periph_rtt_init
                0x0000000008007d6c       0x30 /home/ch/RIOT/examples/lorawan/bin/lora-e5-dev/ztimer_core/periph_rtt.o
                0x0000000008007d6c                ztimer_periph_rtt_init
 .text._ztimer_periph_timer_callback
                0x0000000008007d9c        0x4 /home/ch/RIOT/examples/lorawan/bin/lora-e5-dev/ztimer_core/periph_timer.o
 .text._ztimer_periph_timer_cancel
                0x0000000008007da0        0x8 /home/ch/RIOT/examples/lorawan/bin/lora-e5-dev/ztimer_core/periph_timer.o
 .text._ztimer_periph_timer_now
                0x0000000008007da8        0x6 /home/ch/RIOT/examples/lorawan/bin/lora-e5-dev/ztimer_core/periph_timer.o
 .text._ztimer_periph_timer_set
                0x0000000008007dae       0x10 /home/ch/RIOT/examples/lorawan/bin/lora-e5-dev/ztimer_core/periph_timer.o
 *fill*         0x0000000008007dbe        0x2 
 .text.ztimer_periph_timer_init
                0x0000000008007dc0       0x44 /home/ch/RIOT/examples/lorawan/bin/lora-e5-dev/ztimer_core/periph_timer.o
                0x0000000008007dc0                ztimer_periph_timer_init
 .text._callback_unlock_mutex
                0x0000000008007e04        0x4 /home/ch/RIOT/examples/lorawan/bin/lora-e5-dev/ztimer_core/util.o
 .text._callback_msg
                0x0000000008007e08        0x8 /home/ch/RIOT/examples/lorawan/bin/lora-e5-dev/ztimer_core/util.o
 .text.ztimer_sleep
                0x0000000008007e10       0x48 /home/ch/RIOT/examples/lorawan/bin/lora-e5-dev/ztimer_core/util.o
                0x0000000008007e10                ztimer_sleep
 .text.ztimer_set_msg
                0x0000000008007e58       0x18 /home/ch/RIOT/examples/lorawan/bin/lora-e5-dev/ztimer_core/util.o
                0x0000000008007e58                ztimer_set_msg
 .text          0x0000000008007e70      0x108 /usr/lib/gcc/arm-none-eabi/9.2.1/../../../arm-none-eabi/lib/thumb/v7e-m/nofp/libm.a(lib_a-s_ceil.o)
                0x0000000008007e70                ceil
 .text          0x0000000008007f78      0x108 /usr/lib/gcc/arm-none-eabi/9.2.1/../../../arm-none-eabi/lib/thumb/v7e-m/nofp/libm.a(lib_a-s_floor.o)
                0x0000000008007f78                floor
 .text          0x0000000008008080      0x378 /usr/lib/gcc/arm-none-eabi/9.2.1/thumb/v7e-m/nofp/libgcc.a(_arm_addsubdf3.o)
                0x0000000008008080                __aeabi_drsub
                0x0000000008008088                __aeabi_dsub
                0x0000000008008088                __subdf3
                0x000000000800808c                __adddf3
                0x000000000800808c                __aeabi_dadd
                0x0000000008008304                __aeabi_ui2d
                0x0000000008008304                __floatunsidf
                0x0000000008008324                __floatsidf
                0x0000000008008324                __aeabi_i2d
                0x0000000008008348                __extendsfdf2
                0x0000000008008348                __aeabi_f2d
                0x000000000800838c                __aeabi_ul2d
                0x000000000800838c                __floatundidf
                0x000000000800839c                __floatdidf
                0x000000000800839c                __aeabi_l2d
 .text          0x00000000080083f8      0x424 /usr/lib/gcc/arm-none-eabi/9.2.1/thumb/v7e-m/nofp/libgcc.a(_arm_muldivdf3.o)
                0x00000000080083f8                __aeabi_dmul
                0x00000000080083f8                __muldf3
                0x000000000800864c                __aeabi_ddiv
                0x000000000800864c                __divdf3
 .text          0x000000000800881c      0x110 /usr/lib/gcc/arm-none-eabi/9.2.1/thumb/v7e-m/nofp/libgcc.a(_arm_cmpdf2.o)
                0x000000000800881c                __gtdf2
                0x000000000800881c                __gedf2
                0x0000000008008824                __ltdf2
                0x0000000008008824                __ledf2
                0x000000000800882c                __cmpdf2
                0x000000000800882c                __eqdf2
                0x000000000800882c                __nedf2
                0x00000000080088a8                __aeabi_cdrcmple
                0x00000000080088b8                __aeabi_cdcmple
                0x00000000080088b8                __aeabi_cdcmpeq
                0x00000000080088c8                __aeabi_dcmpeq
                0x00000000080088dc                __aeabi_dcmplt
                0x00000000080088f0                __aeabi_dcmple
                0x0000000008008904                __aeabi_dcmpge
                0x0000000008008918                __aeabi_dcmpgt
 .text          0x000000000800892c       0x50 /usr/lib/gcc/arm-none-eabi/9.2.1/thumb/v7e-m/nofp/libgcc.a(_arm_fixdfsi.o)
                0x000000000800892c                __fixdfsi
                0x000000000800892c                __aeabi_d2iz
 .text          0x000000000800897c       0x40 /usr/lib/gcc/arm-none-eabi/9.2.1/thumb/v7e-m/nofp/libgcc.a(_arm_fixunsdfsi.o)
                0x000000000800897c                __fixunsdfsi
                0x000000000800897c                __aeabi_d2uiz
 .text          0x00000000080089bc      0x21c /usr/lib/gcc/arm-none-eabi/9.2.1/thumb/v7e-m/nofp/libgcc.a(_arm_addsubsf3.o)
                0x00000000080089bc                __aeabi_frsub
                0x00000000080089c4                __subsf3
                0x00000000080089c4                __aeabi_fsub
                0x00000000080089c8                __aeabi_fadd
                0x00000000080089c8                __addsf3
                0x0000000008008b28                __aeabi_ui2f
                0x0000000008008b28                __floatunsisf
                0x0000000008008b30                __aeabi_i2f
                0x0000000008008b30                __floatsisf
                0x0000000008008b4c                __floatundisf
                0x0000000008008b4c                __aeabi_ul2f
                0x0000000008008b5c                __floatdisf
                0x0000000008008b5c                __aeabi_l2f
 .text          0x0000000008008bd8       0x48 /usr/lib/gcc/arm-none-eabi/9.2.1/../../../arm-none-eabi/lib/thumb/v7e-m/nofp/libc_nano.a(lib_a-init.o)
                0x0000000008008bd8                __libc_init_array
 .text          0x0000000008008c20       0x20 /usr/lib/gcc/arm-none-eabi/9.2.1/../../../arm-none-eabi/lib/thumb/v7e-m/nofp/libc_nano.a(lib_a-malloc.o)
                0x0000000008008c20                malloc
                0x0000000008008c30                free
 .text          0x0000000008008c40      0x134 /usr/lib/gcc/arm-none-eabi/9.2.1/../../../arm-none-eabi/lib/thumb/v7e-m/nofp/libc_nano.a(lib_a-memcpy.o)
                0x0000000008008c40                memcpy
 .text          0x0000000008008d74       0xd0 /usr/lib/gcc/arm-none-eabi/9.2.1/../../../arm-none-eabi/lib/thumb/v7e-m/nofp/libc_nano.a(lib_a-memmove.o)
                0x0000000008008d74                memmove
 .text          0x0000000008008e44       0xa0 /usr/lib/gcc/arm-none-eabi/9.2.1/../../../arm-none-eabi/lib/thumb/v7e-m/nofp/libc_nano.a(lib_a-memset.o)
                0x0000000008008e44                memset
 .text          0x0000000008008ee4       0xac /usr/lib/gcc/arm-none-eabi/9.2.1/../../../arm-none-eabi/lib/thumb/v7e-m/nofp/libc_nano.a(lib_a-nano-freer.o)
                0x0000000008008ee4                _free_r
 .text          0x0000000008008f90       0xc8 /usr/lib/gcc/arm-none-eabi/9.2.1/../../../arm-none-eabi/lib/thumb/v7e-m/nofp/libc_nano.a(lib_a-nano-mallocr.o)
                0x0000000008008f90                _malloc_r
 .text          0x0000000008009058      0x6c0 /usr/lib/gcc/arm-none-eabi/9.2.1/../../../arm-none-eabi/lib/thumb/v7e-m/nofp/libc_nano.a(lib_a-nano-vfprintf_float.o)
                0x0000000008009058                __cvt
                0x000000000800914c                __exponent
                0x00000000080091d8                _printf_float
 .text          0x0000000008009718      0x3c4 /usr/lib/gcc/arm-none-eabi/9.2.1/../../../arm-none-eabi/lib/thumb/v7e-m/nofp/libc_nano.a(lib_a-nano-vfprintf_i.o)
                0x0000000008009718                _printf_common
                0x0000000008009844                _printf_i
 .text          0x0000000008009adc       0x68 /usr/lib/gcc/arm-none-eabi/9.2.1/../../../arm-none-eabi/lib/thumb/v7e-m/nofp/libc_nano.a(lib_a-printf.o)
                0x0000000008009adc                _printf_r
                0x0000000008009adc                _iprintf_r
                0x0000000008009b0c                printf
                0x0000000008009b0c                iprintf
 .text          0x0000000008009b44       0xe8 /usr/lib/gcc/arm-none-eabi/9.2.1/../../../arm-none-eabi/lib/thumb/v7e-m/nofp/libc_nano.a(lib_a-puts.o)
                0x0000000008009b44                _puts_r
                0x0000000008009c1c                puts
 *fill*         0x0000000008009c2c       0x14 
 .text          0x0000000008009c40       0xdc /usr/lib/gcc/arm-none-eabi/9.2.1/../../../arm-none-eabi/lib/thumb/v7e-m/nofp/libc_nano.a(lib_a-strlen.o)
                0x0000000008009c40                strlen
 .text          0x0000000008009d1c       0xc0 /usr/lib/gcc/arm-none-eabi/9.2.1/../../../arm-none-eabi/lib/thumb/v7e-m/nofp/libc_nano.a(lib_a-wbuf.o)
                0x0000000008009d1c                __swbuf_r
                0x0000000008009dcc                __swbuf
 .text          0x0000000008009ddc      0x100 /usr/lib/gcc/arm-none-eabi/9.2.1/../../../arm-none-eabi/lib/thumb/v7e-m/nofp/libc_nano.a(lib_a-wsetup.o)
                0x0000000008009ddc                __swsetup_r
 *fill*         0x0000000008009edc        0x4 
 .text          0x0000000008009ee0     0x104c /usr/lib/gcc/arm-none-eabi/9.2.1/../../../arm-none-eabi/lib/thumb/v7e-m/nofp/libc_nano.a(lib_a-dtoa.o)
                0x000000000800a004                _dtoa_r
 .text          0x000000000800af2c      0x1b0 /usr/lib/gcc/arm-none-eabi/9.2.1/../../../arm-none-eabi/lib/thumb/v7e-m/nofp/libc_nano.a(lib_a-fflush.o)
                0x000000000800af2c                __sflush_r
                0x000000000800b058                _fflush_r
                0x000000000800b0b8                fflush
 .text          0x000000000800b0dc      0x210 /usr/lib/gcc/arm-none-eabi/9.2.1/../../../arm-none-eabi/lib/thumb/v7e-m/nofp/libc_nano.a(lib_a-findfp.o)
                0x000000000800b0e0                _cleanup_r
                0x000000000800b0f0                __sfmoreglue
                0x000000000800b120                __sfp
                0x000000000800b298                _cleanup
                0x000000000800b2ac                __sinit
                0x000000000800b2b4                __sfp_lock_acquire
                0x000000000800b2b8                __sfp_lock_release
                0x000000000800b2bc                __sinit_lock_acquire
                0x000000000800b2c0                __sinit_lock_release
                0x000000000800b2c4                __fp_lock_all
                0x000000000800b2d8                __fp_unlock_all
 .text          0x000000000800b2ec       0x44 /usr/lib/gcc/arm-none-eabi/9.2.1/../../../arm-none-eabi/lib/thumb/v7e-m/nofp/libc_nano.a(lib_a-fprintf.o)
                0x000000000800b2ec                _fprintf_r
                0x000000000800b2ec                _fiprintf_r
                0x000000000800b308                fprintf
                0x000000000800b308                fiprintf
 .text          0x000000000800b330       0xa0 /usr/lib/gcc/arm-none-eabi/9.2.1/../../../arm-none-eabi/lib/thumb/v7e-m/nofp/libc_nano.a(lib_a-fwalk.o)
                0x000000000800b330                _fwalk
                0x000000000800b37c                _fwalk_reent
 .text          0x000000000800b3d0       0x14 /usr/lib/gcc/arm-none-eabi/9.2.1/../../../arm-none-eabi/lib/thumb/v7e-m/nofp/libc_nano.a(lib_a-localeconv.o)
                0x000000000800b3d0                __localeconv_l
                0x000000000800b3d4                _localeconv_r
                0x000000000800b3dc                localeconv
 .text          0x000000000800b3e4       0xf0 /usr/lib/gcc/arm-none-eabi/9.2.1/../../../arm-none-eabi/lib/thumb/v7e-m/nofp/libc_nano.a(lib_a-makebuf.o)
                0x000000000800b3e4                __swhatbuf_r
                0x000000000800b440                __smakebuf_r
 *fill*         0x000000000800b4d4        0xc 
 .text          0x000000000800b4e0       0xa0 /usr/lib/gcc/arm-none-eabi/9.2.1/../../../arm-none-eabi/lib/thumb/v7e-m/nofp/libc_nano.a(lib_a-memchr.o)
                0x000000000800b4e0                memchr
 .text          0x000000000800b580        0x8 /usr/lib/gcc/arm-none-eabi/9.2.1/../../../arm-none-eabi/lib/thumb/v7e-m/nofp/libc_nano.a(lib_a-mlock.o)
                0x000000000800b580                __malloc_lock
                0x000000000800b584                __malloc_unlock
 .text          0x000000000800b588      0xa08 /usr/lib/gcc/arm-none-eabi/9.2.1/../../../arm-none-eabi/lib/thumb/v7e-m/nofp/libc_nano.a(lib_a-mprec.o)
                0x000000000800b588                _Balloc
                0x000000000800b608                _Bfree
                0x000000000800b654                __multadd
                0x000000000800b6f4                __s2b
                0x000000000800b7a0                __hi0bits
                0x000000000800b7e0                __lo0bits
                0x000000000800b840                __i2b
                0x000000000800b86c                __multiply
                0x000000000800b9b8                __pow5mult
                0x000000000800ba7c                __lshift
                0x000000000800bb44                __mcmp
                0x000000000800bb7c                __mdiff
                0x000000000800bca4                __ulp
                0x000000000800bce4                __b2d
                0x000000000800bd9c                __d2b
                0x000000000800be60                __ratio
                0x000000000800bebc                _mprec_log10
                0x000000000800bef4                __copybits
                0x000000000800bf3c                __any_on
 .text          0x000000000800bf90       0x1c /usr/lib/gcc/arm-none-eabi/9.2.1/../../../arm-none-eabi/lib/thumb/v7e-m/nofp/libc_nano.a(lib_a-nano-callocr.o)
                0x000000000800bf90                _calloc_r
 .text          0x000000000800bfac       0x4c /usr/lib/gcc/arm-none-eabi/9.2.1/../../../arm-none-eabi/lib/thumb/v7e-m/nofp/libc_nano.a(lib_a-nano-reallocr.o)
                0x000000000800bfac                _realloc_r
 .text          0x000000000800bff8      0x360 /usr/lib/gcc/arm-none-eabi/9.2.1/../../../arm-none-eabi/lib/thumb/v7e-m/nofp/libc_nano.a(lib_a-nano-vfprintf.o)
                0x000000000800c030                __sfputs_r
                0x000000000800c060                __sprint_r
                0x000000000800c07c                _vfiprintf_r
                0x000000000800c07c                _vfprintf_r
                0x000000000800c340                vfiprintf
                0x000000000800c340                vfprintf
 .text          0x000000000800c358       0x90 /usr/lib/gcc/arm-none-eabi/9.2.1/../../../arm-none-eabi/lib/thumb/v7e-m/nofp/libc_nano.a(lib_a-stdio.o)
                0x000000000800c358                __sread
                0x000000000800c37c                __seofread
                0x000000000800c380                __swrite
                0x000000000800c3c0                __sseek
                0x000000000800c3e0                __sclose
 .text          0x000000000800c3e8       0x48 /usr/lib/gcc/arm-none-eabi/9.2.1/../../../arm-none-eabi/lib/thumb/v7e-m/nofp/libc_nano.a(lib_a-assert.o)
                0x000000000800c3e8                __assert_func
                0x000000000800c424                __assert
 .text          0x000000000800c430      0x308 /usr/lib/gcc/arm-none-eabi/9.2.1/../../../arm-none-eabi/lib/thumb/v7e-m/nofp/libc_nano.a(lib_a-fvwrite.o)
                0x000000000800c430                __sfvwrite_r
 .text          0x000000000800c738       0x40 /usr/lib/gcc/arm-none-eabi/9.2.1/../../../arm-none-eabi/lib/thumb/v7e-m/nofp/libc_nano.a(lib_a-mbtowc_r.o)
                0x000000000800c738                _mbtowc_r
                0x000000000800c74c                __ascii_mbtowc
 .text          0x000000000800c778       0x10 /usr/lib/gcc/arm-none-eabi/9.2.1/../../../arm-none-eabi/lib/thumb/v7e-m/nofp/libc_nano.a(lib_a-nano-msizer.o)
                0x000000000800c778                _malloc_usable_size_r
 .text          0x000000000800c788       0x30 /usr/lib/gcc/arm-none-eabi/9.2.1/../../../arm-none-eabi/lib/thumb/v7e-m/nofp/libc_nano.a(lib_a-wctomb_r.o)
                0x000000000800c788                _wctomb_r
                0x000000000800c79c                __ascii_wctomb
 .text          0x000000000800c7b8       0x10 /usr/lib/gcc/arm-none-eabi/9.2.1/../../../arm-none-eabi/lib/thumb/v7e-m/nofp/libc_nano.a(lib_a-abort.o)
                0x000000000800c7b8                abort
 .text          0x000000000800c7c8      0x150 /usr/lib/gcc/arm-none-eabi/9.2.1/../../../arm-none-eabi/lib/thumb/v7e-m/nofp/libc_nano.a(lib_a-signal.o)
                0x000000000800c7f0                _init_signal_r
                0x000000000800c7fc                _signal_r
                0x000000000800c830                _raise_r
                0x000000000800c884                __sigtramp_r
                0x000000000800c8d4                raise
                0x000000000800c8e4                signal
                0x000000000800c8f4                _init_signal
                0x000000000800c908                __sigtramp
 .text          0x000000000800c918       0x2c /usr/lib/gcc/arm-none-eabi/9.2.1/thumb/v7e-m/nofp/libgcc.a(_arm_unorddf2.o)
                0x000000000800c918                __aeabi_dcmpun
                0x000000000800c918                __unorddf2
 *(.glue_7t)
 .glue_7t       0x000000000800c944        0x0 linker stubs
 *(.glue_7)
 .glue_7        0x000000000800c944        0x0 linker stubs
 *(.rodata .rodata* .gnu.linkonce.r.*)
 .rodata.sender.str1.1
                0x000000000800c944       0x43 /home/ch/RIOT/examples/lorawan/bin/lora-e5-dev/application_lorawan/main.o
 .rodata.main.str1.1
                0x000000000800c987       0xcc /home/ch/RIOT/examples/lorawan/bin/lora-e5-dev/application_lorawan/main.o
                                         0xdd (size before relaxing)
 *fill*         0x000000000800ca53        0x1 
 .rodata.sx126x_params
                0x000000000800ca54       0x20 /home/ch/RIOT/examples/lorawan/bin/lora-e5-dev/application_lorawan/main.o
 .rodata.main_trampoline.str1.1
                0x000000000800ca74       0x3b /home/ch/RIOT/examples/lorawan/bin/lora-e5-dev/core/init.o
 .rodata.kernel_init.str1.1
                0x000000000800caaf        0x5 /home/ch/RIOT/examples/lorawan/bin/lora-e5-dev/core/init.o
 .rodata.core_panic.str1.1
                0x000000000800cab4       0x2e /home/ch/RIOT/examples/lorawan/bin/lora-e5-dev/core/panic.o
 .rodata.assert_crash_message
                0x000000000800cae2       0x12 /home/ch/RIOT/examples/lorawan/bin/lora-e5-dev/core/panic.o
                0x000000000800cae2                assert_crash_message
 .rodata._unschedule.str1.1
                0x000000000800caf4       0x2f /home/ch/RIOT/examples/lorawan/bin/lora-e5-dev/core/sched.o
 .rodata.panic_arch.str1.1
                0x000000000800cb23        0xf /home/ch/RIOT/examples/lorawan/bin/lora-e5-dev/cortexm_common/panic.o
 .rodata.nmi_default.str1.1
                0x000000000800cb32        0xc /home/ch/RIOT/examples/lorawan/bin/lora-e5-dev/cortexm_common/vectors_cortexm.o
 .rodata.mem_manage_default.str1.1
                0x000000000800cb3e       0x13 /home/ch/RIOT/examples/lorawan/bin/lora-e5-dev/cortexm_common/vectors_cortexm.o
 .rodata.bus_fault_default.str1.1
                0x000000000800cb51       0x12 /home/ch/RIOT/examples/lorawan/bin/lora-e5-dev/cortexm_common/vectors_cortexm.o
 .rodata.usage_fault_default.str1.1
                0x000000000800cb63       0x14 /home/ch/RIOT/examples/lorawan/bin/lora-e5-dev/cortexm_common/vectors_cortexm.o
 .rodata.debug_mon_default.str1.1
                0x000000000800cb77       0x12 /home/ch/RIOT/examples/lorawan/bin/lora-e5-dev/cortexm_common/vectors_cortexm.o
 .rodata.dummy_handler_default.str1.1
                0x000000000800cb89        0xe /home/ch/RIOT/examples/lorawan/bin/lora-e5-dev/cortexm_common/vectors_cortexm.o
 .rodata.hard_fault_handler.str1.1
                0x000000000800cb97      0x233 /home/ch/RIOT/examples/lorawan/bin/lora-e5-dev/cortexm_common/vectors_cortexm.o
 .rodata.apbmul
                0x000000000800cdca        0x4 /home/ch/RIOT/examples/lorawan/bin/lora-e5-dev/cpu/cpu_common.o
 *fill*         0x000000000800cdce        0x2 
 .rodata.Te0    0x000000000800cdd0      0x400 /home/ch/RIOT/examples/lorawan/bin/lora-e5-dev/crypto/aes.o
 .rodata.rcon   0x000000000800d1d0       0x28 /home/ch/RIOT/examples/lorawan/bin/lora-e5-dev/crypto/aes.o
 .rodata        0x000000000800d1f8        0x3 /home/ch/RIOT/examples/lorawan/bin/lora-e5-dev/driver_sx126x/sx126x.o
 .rodata._exit.str1.1
                0x000000000800d1fb       0x1a /home/ch/RIOT/examples/lorawan/bin/lora-e5-dev/newlib_syscalls_default/syscalls.o
 *fill*         0x000000000800d215        0x3 
 .rodata.spi_config
                0x000000000800d218       0x40 /home/ch/RIOT/examples/lorawan/bin/lora-e5-dev/periph/spi.o
 .rodata.timer_config
                0x000000000800d258       0x10 /home/ch/RIOT/examples/lorawan/bin/lora-e5-dev/periph/timer.o
 .rodata.uart_config
                0x000000000800d268       0x54 /home/ch/RIOT/examples/lorawan/bin/lora-e5-dev/periph/uart.o
 .rodata.semtech_loramac_init.str1.1
                0x000000000800d2bc        0xc /home/ch/RIOT/examples/lorawan/bin/lora-e5-dev/semtech_loramac_contrib/semtech_loramac.o
 .rodata.CSWTCH.34
                0x000000000800d2c8        0xc /home/ch/RIOT/examples/lorawan/bin/lora-e5-dev/semtech_loramac_contrib/semtech_loramac.o
 .rodata        0x000000000800d2d4       0x18 /home/ch/RIOT/examples/lorawan/bin/lora-e5-dev/semtech_loramac_contrib/semtech_loramac_radio.o
 .rodata.Radio  0x000000000800d2ec       0x6c /home/ch/RIOT/examples/lorawan/bin/lora-e5-dev/semtech_loramac_contrib/semtech_loramac_radio.o
                0x000000000800d2ec                Radio
 .rodata.LoRaMacMaxEirpTable
                0x000000000800d358       0x10 /home/ch/RIOT/examples/lorawan/bin/lora-e5-dev/semtech_loramac_mac/LoRaMac.o
 .rodata        0x000000000800d368       0x24 /home/ch/RIOT/examples/lorawan/bin/lora-e5-dev/semtech_loramac_mac_region/RegionEU868.o
 .rodata.BandwidthsEU868
                0x000000000800d38c       0x20 /home/ch/RIOT/examples/lorawan/bin/lora-e5-dev/semtech_loramac_mac_region/RegionEU868.o
 .rodata.CSWTCH.48
                0x000000000800d3ac        0x7 /home/ch/RIOT/examples/lorawan/bin/lora-e5-dev/semtech_loramac_mac_region/RegionEU868.o
 .rodata.DataratesEU868
                0x000000000800d3b3        0x8 /home/ch/RIOT/examples/lorawan/bin/lora-e5-dev/semtech_loramac_mac_region/RegionEU868.o
 .rodata.MaxPayloadOfDatarateEU868
                0x000000000800d3bb        0x8 /home/ch/RIOT/examples/lorawan/bin/lora-e5-dev/semtech_loramac_mac_region/RegionEU868.o
 .rodata.MaxPayloadOfDatarateRepeaterEU868
                0x000000000800d3c3        0x8 /home/ch/RIOT/examples/lorawan/bin/lora-e5-dev/semtech_loramac_mac_region/RegionEU868.o
 *fill*         0x000000000800d3cb        0x1 
 .rodata.sx126x_driver
                0x000000000800d3cc       0x1c /home/ch/RIOT/examples/lorawan/bin/lora-e5-dev/sx126x/sx126x_netdev.o
                0x000000000800d3cc                sx126x_driver
 .rodata._bw_khz
                0x000000000800d3e8        0x6 /home/ch/RIOT/examples/lorawan/bin/lora-e5-dev/sx126x/sx126x.o
 .rodata.hpa_cfg
                0x000000000800d3ee        0x4 /home/ch/RIOT/examples/lorawan/bin/lora-e5-dev/sx126x/sx126x.o
                0x000000000800d3ee                hpa_cfg
 .rodata.lpa_cfg
                0x000000000800d3f2        0x4 /home/ch/RIOT/examples/lorawan/bin/lora-e5-dev/sx126x/sx126x.o
                0x000000000800d3f2                lpa_cfg
 *fill*         0x000000000800d3f6        0x2 
 .rodata.ztimer_convert_frac_ops
                0x000000000800d3f8        0xc /home/ch/RIOT/examples/lorawan/bin/lora-e5-dev/ztimer_core/convert_frac.o
 .rodata.ZTIMER_MSEC
                0x000000000800d404        0x4 /home/ch/RIOT/examples/lorawan/bin/lora-e5-dev/ztimer_core/init.o
                0x000000000800d404                ZTIMER_MSEC
 .rodata.ZTIMER_USEC
                0x000000000800d408        0x4 /home/ch/RIOT/examples/lorawan/bin/lora-e5-dev/ztimer_core/init.o
                0x000000000800d408                ZTIMER_USEC
 .rodata._ztimer_periph_rtt_ops
                0x000000000800d40c        0xc /home/ch/RIOT/examples/lorawan/bin/lora-e5-dev/ztimer_core/periph_rtt.o
 .rodata._ztimer_periph_timer_ops
                0x000000000800d418        0xc /home/ch/RIOT/examples/lorawan/bin/lora-e5-dev/ztimer_core/periph_timer.o
 .rodata        0x000000000800d424        0x4 /usr/lib/gcc/arm-none-eabi/9.2.1/../../../arm-none-eabi/lib/thumb/v7e-m/nofp/libc_nano.a(lib_a-impure.o)
                0x000000000800d424                _global_impure_ptr
 .rodata.str1.4
                0x000000000800d428       0x12 /usr/lib/gcc/arm-none-eabi/9.2.1/../../../arm-none-eabi/lib/thumb/v7e-m/nofp/libc_nano.a(lib_a-nano-vfprintf_float.o)
 *fill*         0x000000000800d43a        0x2 
 .rodata.str1.4
                0x000000000800d43c       0x25 /usr/lib/gcc/arm-none-eabi/9.2.1/../../../arm-none-eabi/lib/thumb/v7e-m/nofp/libc_nano.a(lib_a-nano-vfprintf_i.o)
 *fill*         0x000000000800d461        0x3 
 .rodata.str1.4
                0x000000000800d464       0x6d /usr/lib/gcc/arm-none-eabi/9.2.1/../../../arm-none-eabi/lib/thumb/v7e-m/nofp/libc_nano.a(lib_a-dtoa.o)
                                         0x71 (size before relaxing)
 *fill*         0x000000000800d4d1        0x3 
 .rodata        0x000000000800d4d4       0x60 /usr/lib/gcc/arm-none-eabi/9.2.1/../../../arm-none-eabi/lib/thumb/v7e-m/nofp/libc_nano.a(lib_a-findfp.o)
                0x000000000800d4d4                __sf_fake_stderr
                0x000000000800d4f4                __sf_fake_stdout
                0x000000000800d514                __sf_fake_stdin
 *fill*         0x000000000800d534        0x4 
 .rodata        0x000000000800d538      0x128 /usr/lib/gcc/arm-none-eabi/9.2.1/../../../arm-none-eabi/lib/thumb/v7e-m/nofp/libc_nano.a(lib_a-mprec.o)
                0x000000000800d548                __mprec_tens
                0x000000000800d610                __mprec_tinytens
                0x000000000800d638                __mprec_bigtens
 .rodata.str1.4
                0x000000000800d660       0x33 /usr/lib/gcc/arm-none-eabi/9.2.1/../../../arm-none-eabi/lib/thumb/v7e-m/nofp/libc_nano.a(lib_a-mprec.o)
                                         0x5d (size before relaxing)
 *fill*         0x000000000800d693        0x1 
 .rodata.str1.4
                0x000000000800d694       0x13 /usr/lib/gcc/arm-none-eabi/9.2.1/../../../arm-none-eabi/lib/thumb/v7e-m/nofp/libc_nano.a(lib_a-nano-vfprintf.o)
 *fill*         0x000000000800d6a7        0x1 
 .rodata.str1.4
                0x000000000800d6a8       0x3f /usr/lib/gcc/arm-none-eabi/9.2.1/../../../arm-none-eabi/lib/thumb/v7e-m/nofp/libc_nano.a(lib_a-assert.o)
                                         0x43 (size before relaxing)
 *fill*         0x000000000800d6e7        0x1 
 .rodata.str1.4
                0x000000000800d6e8        0xe /usr/lib/gcc/arm-none-eabi/9.2.1/../../../arm-none-eabi/lib/thumb/v7e-m/nofp/libc_nano.a(lib_a-locale.o)
                                         0x12 (size before relaxing)
 *fill*         0x000000000800d6f6        0x2 
 .rodata        0x000000000800d6f8      0x101 /usr/lib/gcc/arm-none-eabi/9.2.1/../../../arm-none-eabi/lib/thumb/v7e-m/nofp/libc_nano.a(lib_a-ctype_.o)
                0x000000000800d6f8                _ctype_
 *(SORT_BY_NAME(.roxfa.*))
 *(.ARM.extab* .gnu.linkonce.armextab.*)
                0x000000000800d7fc                . = ALIGN (0x4)
 *fill*         0x000000000800d7f9        0x3 
 *(.init)
                0x000000000800d7fc                . = ALIGN (0x4)
                0x000000000800d7fc                __preinit_array_start = .
 *(.preinit_array)
                0x000000000800d7fc                __preinit_array_end = .
                0x000000000800d7fc                . = ALIGN (0x4)
                0x000000000800d7fc                __init_array_start = .
 *(SORT_BY_NAME(.init_array.*))
 *(.init_array)
                0x000000000800d7fc                __init_array_end = .
                0x000000000800d7fc                . = ALIGN (0x4)
 *crtbegin.o(.ctors)
 *(EXCLUDE_FILE(*crtend.o) .ctors)
 *(SORT_BY_NAME(.ctors.*))
 *crtend.o(.ctors)
                0x000000000800d7fc                . = ALIGN (0x4)
 *(.fini)
                0x000000000800d7fc                . = ALIGN (0x4)
                0x000000000800d7fc                __fini_array_start = .
 *(.fini_array)
 *(SORT_BY_NAME(.fini_array.*))
                0x000000000800d7fc                __fini_array_end = .
 *crtbegin.o(.dtors)
 *(EXCLUDE_FILE(*crtend.o) .dtors)
 *(SORT_BY_NAME(.dtors.*))
 *crtend.o(.dtors)
                0x000000000800d7fc                . = ALIGN (0x4)
                0x000000000800d7fc                _efixed = .

.vfp11_veneer   0x000000000800d7fc        0x0
 .vfp11_veneer  0x000000000800d7fc        0x0 linker stubs

.v4_bx          0x000000000800d7fc        0x0
 .v4_bx         0x000000000800d7fc        0x0 linker stubs

.iplt           0x000000000800d7fc        0x0
 .iplt          0x000000000800d7fc        0x0 /home/ch/RIOT/examples/lorawan/bin/lora-e5-dev/application_lorawan/main.o

.igot.plt       0x000000000800d7fc        0x0
 .igot.plt      0x000000000800d7fc        0x0 /home/ch/RIOT/examples/lorawan/bin/lora-e5-dev/application_lorawan/main.o

.rel.dyn        0x000000000800d7fc        0x0
 .rel.iplt      0x000000000800d7fc        0x0 /home/ch/RIOT/examples/lorawan/bin/lora-e5-dev/application_lorawan/main.o

.tdata          0x000000000800d7fc        0x0
                0x000000000800d7fc                __tdata_start = .
 *(.tdata .tdata.* .gnu.linkonce.td.*)
                0x000000000800d7fc                __tdata_end = .
                0x000000000800d7fc                __tdata_source = LOADADDR (.tdata)
                0x0000000000000000                __tdata_size = SIZEOF (.tdata)

.tbss           0x000000000800d7fc        0x0
 *(.tbss .tbss.* .gnu.linkonce.tb.*)
 *(.tcommon)
                0x000000000800d7fc                __tbss_end = .
                0x0000000000000000                __tls_size = (__tbss_end - __tdata_start)
                0x0000000000000000                __tbss_size = (__tls_size - __tdata_size)
                [!provide]                        PROVIDE (__exidx_start = .)

.ARM.exidx
 *(.ARM.exidx* .gnu.linkonce.armexidx.*)
                [!provide]                        PROVIDE (__exidx_end = .)
                0x000000000800d7fc                . = ALIGN (0x4)

.eh_frame
 *(.eh_frame)
                0x000000000800d7fc                . = ALIGN (0x4)
                0x000000000800d7fc                _etext = .

.stack          0x0000000020000000      0x200
 *(.puf)
                0x0000000020000000                . = ALIGN (0x8)
                0x0000000020000000                _sstack = .
 *(.isr_stack)
 .isr_stack     0x0000000020000000      0x200 /home/ch/RIOT/examples/lorawan/bin/lora-e5-dev/cortexm_common/vectors_cortexm.o
                0x0000000020000000                isr_stack
                0x0000000020000200                . = ALIGN (0x8)
                0x0000000020000200                _estack = .

.relocate       0x0000000020000200      0x28c load address 0x000000000800d7fc
                0x0000000020000200                . = ALIGN (0x4)
                0x0000000020000200                _srelocate = .
 *(.ramfunc .ramfunc.*)
 *(.data .data.*)
 .data.heap_top
                0x0000000020000200        0x4 /home/ch/RIOT/examples/lorawan/bin/lora-e5-dev/newlib_syscalls_default/syscalls.o
 .data.pm_blocker
                0x0000000020000204        0x4 /home/ch/RIOT/examples/lorawan/bin/lora-e5-dev/pm_layered/pm.o
 .data.MicBlockB0
                0x0000000020000208       0x10 /home/ch/RIOT/examples/lorawan/bin/lora-e5-dev/semtech_loramac_mac/LoRaMacCrypto.o
 .data.aBlock   0x0000000020000218       0x10 /home/ch/RIOT/examples/lorawan/bin/lora-e5-dev/semtech_loramac_mac/LoRaMacCrypto.o
 .data.AckTimeoutRetries
                0x0000000020000228        0x1 /home/ch/RIOT/examples/lorawan/bin/lora-e5-dev/semtech_loramac_mac/LoRaMac.o
 .data.AckTimeoutRetriesCounter
                0x0000000020000229        0x1 /home/ch/RIOT/examples/lorawan/bin/lora-e5-dev/semtech_loramac_mac/LoRaMac.o
 .data.IsRxWindowsEnabled
                0x000000002000022a        0x1 /home/ch/RIOT/examples/lorawan/bin/lora-e5-dev/semtech_loramac_mac/LoRaMac.o
 *fill*         0x000000002000022b        0x1 
 .data.Bands    0x000000002000022c       0x50 /home/ch/RIOT/examples/lorawan/bin/lora-e5-dev/semtech_loramac_mac_region/RegionEU868.o
 .data._ztimer  0x000000002000027c       0x10 /home/ch/RIOT/examples/lorawan/bin/lora-e5-dev/xtimer/xtimer_core.o
 .data._ztimer_periph_timer
                0x000000002000028c       0x2c /home/ch/RIOT/examples/lorawan/bin/lora-e5-dev/ztimer_core/init.o
 .data          0x00000000200002b8       0x64 /usr/lib/gcc/arm-none-eabi/9.2.1/../../../arm-none-eabi/lib/thumb/v7e-m/nofp/libc_nano.a(lib_a-impure.o)
                0x00000000200002b8                _impure_ptr
 .data          0x000000002000031c      0x16c /usr/lib/gcc/arm-none-eabi/9.2.1/../../../arm-none-eabi/lib/thumb/v7e-m/nofp/libc_nano.a(lib_a-locale.o)
                0x000000002000031c                __global_locale
 *(SORT_BY_NAME(.xfa.*))
 *(.openocd .openocd.*)
 .openocd       0x0000000020000488        0x2 /home/ch/RIOT/examples/lorawan/bin/lora-e5-dev/core/sched.o
                0x0000000020000488                _tcb_name_offset
                0x0000000020000489                max_threads
                0x000000002000048c                . = ALIGN (0x4)
 *fill*         0x000000002000048a        0x2 
                0x000000002000048c                _erelocate = .

.bss            0x0000000020000490     0x1680 load address 0x000000000800da88
                0x0000000020000490                . = ALIGN (0x4)
                0x0000000020000490                _sbss = .
                0x0000000020000490                _szero = .
 *(.bss .bss.*)
 .bss.appeui    0x0000000020000490        0x8 /home/ch/RIOT/examples/lorawan/bin/lora-e5-dev/application_lorawan/main.o
 .bss.appkey    0x0000000020000498       0x10 /home/ch/RIOT/examples/lorawan/bin/lora-e5-dev/application_lorawan/main.o
 .bss.deveui    0x00000000200004a8        0x8 /home/ch/RIOT/examples/lorawan/bin/lora-e5-dev/application_lorawan/main.o
 .bss.loramac   0x00000000200004b0       0x2c /home/ch/RIOT/examples/lorawan/bin/lora-e5-dev/application_lorawan/main.o
 .bss.sender_pid
                0x00000000200004dc        0x2 /home/ch/RIOT/examples/lorawan/bin/lora-e5-dev/application_lorawan/main.o
 .bss.sender_stack
                0x00000000200004de      0x300 /home/ch/RIOT/examples/lorawan/bin/lora-e5-dev/application_lorawan/main.o
 *fill*         0x00000000200007de        0x2 
 .bss.sx126x    0x00000000200007e0       0x24 /home/ch/RIOT/examples/lorawan/bin/lora-e5-dev/application_lorawan/main.o
 .bss.timer     0x0000000020000804       0x10 /home/ch/RIOT/examples/lorawan/bin/lora-e5-dev/application_lorawan/main.o
 .bss.main_stack
                0x0000000020000814      0x600 /home/ch/RIOT/examples/lorawan/bin/lora-e5-dev/core/init.o
 .bss.crashed   0x0000000020000e14        0x4 /home/ch/RIOT/examples/lorawan/bin/lora-e5-dev/core/panic.o
 .bss.runqueue_bitcache
                0x0000000020000e18        0x4 /home/ch/RIOT/examples/lorawan/bin/lora-e5-dev/core/sched.o
 .bss.sched_active_pid
                0x0000000020000e1c        0x2 /home/ch/RIOT/examples/lorawan/bin/lora-e5-dev/core/sched.o
                0x0000000020000e1c                sched_active_pid
 *fill*         0x0000000020000e1e        0x2 
 .bss.sched_active_thread
                0x0000000020000e20        0x4 /home/ch/RIOT/examples/lorawan/bin/lora-e5-dev/core/sched.o
                0x0000000020000e20                sched_active_thread
 .bss.sched_context_switch_request
                0x0000000020000e24        0x4 /home/ch/RIOT/examples/lorawan/bin/lora-e5-dev/core/sched.o
                0x0000000020000e24                sched_context_switch_request
 .bss.sched_num_threads
                0x0000000020000e28        0x4 /home/ch/RIOT/examples/lorawan/bin/lora-e5-dev/core/sched.o
                0x0000000020000e28                sched_num_threads
 .bss.sched_runqueues
                0x0000000020000e2c       0x40 /home/ch/RIOT/examples/lorawan/bin/lora-e5-dev/core/sched.o
                0x0000000020000e2c                sched_runqueues
 .bss.sched_threads
                0x0000000020000e6c       0x84 /home/ch/RIOT/examples/lorawan/bin/lora-e5-dev/core/sched.o
                0x0000000020000e6c                sched_threads
 .bss.lastused  0x0000000020000ef0        0x1 /home/ch/RIOT/examples/lorawan/bin/lora-e5-dev/luid/luid.o
 *fill*         0x0000000020000ef1        0x3 
 .bss._lock     0x0000000020000ef4        0x4 /home/ch/RIOT/examples/lorawan/bin/lora-e5-dev/malloc_thread_safe/malloc_wrappers.o
 .bss.isr_ctx   0x0000000020000ef8       0x80 /home/ch/RIOT/examples/lorawan/bin/lora-e5-dev/periph/gpio_all.o
 .bss.locks     0x0000000020000f78        0x4 /home/ch/RIOT/examples/lorawan/bin/lora-e5-dev/periph/i2c_1.o
 .bss.ovf_arg   0x0000000020000f7c        0x4 /home/ch/RIOT/examples/lorawan/bin/lora-e5-dev/periph/rtt_all.o
 .bss.ovf_cb    0x0000000020000f80        0x4 /home/ch/RIOT/examples/lorawan/bin/lora-e5-dev/periph/rtt_all.o
 .bss.to_arg    0x0000000020000f84        0x4 /home/ch/RIOT/examples/lorawan/bin/lora-e5-dev/periph/rtt_all.o
 .bss.to_cb     0x0000000020000f88        0x4 /home/ch/RIOT/examples/lorawan/bin/lora-e5-dev/periph/rtt_all.o
 .bss.clocks    0x0000000020000f8c        0x8 /home/ch/RIOT/examples/lorawan/bin/lora-e5-dev/periph/spi.o
 .bss.dividers  0x0000000020000f94        0x2 /home/ch/RIOT/examples/lorawan/bin/lora-e5-dev/periph/spi.o
 *fill*         0x0000000020000f96        0x2 
 .bss.locks     0x0000000020000f98        0x8 /home/ch/RIOT/examples/lorawan/bin/lora-e5-dev/periph/spi.o
 .bss.isr_ctx   0x0000000020000fa0        0x8 /home/ch/RIOT/examples/lorawan/bin/lora-e5-dev/periph/timer.o
 .bss.isr_ctx   0x0000000020000fa8       0x24 /home/ch/RIOT/examples/lorawan/bin/lora-e5-dev/periph/uart.o
 *fill*         0x0000000020000fcc        0x4 
 .bss._seed     0x0000000020000fd0        0x8 /home/ch/RIOT/examples/lorawan/bin/lora-e5-dev/random/musl_lcg.o
 .bss._semtech_loramac_msg_queue
                0x0000000020000fd8       0x20 /home/ch/RIOT/examples/lorawan/bin/lora-e5-dev/semtech_loramac_contrib/semtech_loramac.o
 .bss._semtech_loramac_stack
                0x0000000020000ff8      0x400 /home/ch/RIOT/examples/lorawan/bin/lora-e5-dev/semtech_loramac_contrib/semtech_loramac.o
 .bss.loramac_netdev_ptr
                0x00000000200013f8        0x4 /home/ch/RIOT/examples/lorawan/bin/lora-e5-dev/semtech_loramac_contrib/semtech_loramac.o
                0x00000000200013f8                loramac_netdev_ptr
 .bss.semtech_loramac_callbacks
                0x00000000200013fc        0x4 /home/ch/RIOT/examples/lorawan/bin/lora-e5-dev/semtech_loramac_contrib/semtech_loramac.o
                0x00000000200013fc                semtech_loramac_callbacks
 .bss.semtech_loramac_pid
                0x0000000020001400        0x2 /home/ch/RIOT/examples/lorawan/bin/lora-e5-dev/semtech_loramac_contrib/semtech_loramac.o
                0x0000000020001400                semtech_loramac_pid
 *fill*         0x0000000020001402        0x2 
 .bss.semtech_loramac_primitives
                0x0000000020001404       0x10 /home/ch/RIOT/examples/lorawan/bin/lora-e5-dev/semtech_loramac_contrib/semtech_loramac.o
                0x0000000020001404                semtech_loramac_primitives
 .bss.semtech_loramac_radio_events
                0x0000000020001414       0x1c /home/ch/RIOT/examples/lorawan/bin/lora-e5-dev/semtech_loramac_contrib/semtech_loramac.o
                0x0000000020001414                semtech_loramac_radio_events
 .bss.AesCmacCtx
                0x0000000020001430       0x38 /home/ch/RIOT/examples/lorawan/bin/lora-e5-dev/semtech_loramac_mac/LoRaMacCrypto.o
 .bss.AesContext
                0x0000000020001468       0x11 /home/ch/RIOT/examples/lorawan/bin/lora-e5-dev/semtech_loramac_mac/LoRaMacCrypto.o
 .bss.Mic       0x0000000020001479       0x10 /home/ch/RIOT/examples/lorawan/bin/lora-e5-dev/semtech_loramac_mac/LoRaMacCrypto.o
 .bss.sBlock    0x0000000020001489       0x10 /home/ch/RIOT/examples/lorawan/bin/lora-e5-dev/semtech_loramac_mac/LoRaMacCrypto.o
 .bss.AckTimeoutRetry
                0x0000000020001499        0x1 /home/ch/RIOT/examples/lorawan/bin/lora-e5-dev/semtech_loramac_mac/LoRaMac.o
 *fill*         0x000000002000149a        0x2 
 .bss.AckTimeoutTimer
                0x000000002000149c       0x24 /home/ch/RIOT/examples/lorawan/bin/lora-e5-dev/semtech_loramac_mac/LoRaMac.o
 .bss.AdrAckCounter
                0x00000000200014c0        0x4 /home/ch/RIOT/examples/lorawan/bin/lora-e5-dev/semtech_loramac_mac/LoRaMac.o
 .bss.AdrCtrlOn
                0x00000000200014c4        0x1 /home/ch/RIOT/examples/lorawan/bin/lora-e5-dev/semtech_loramac_mac/LoRaMac.o
 *fill*         0x00000000200014c5        0x1 
 .bss.AggregatedDCycle
                0x00000000200014c6        0x2 /home/ch/RIOT/examples/lorawan/bin/lora-e5-dev/semtech_loramac_mac/LoRaMac.o
 .bss.AggregatedLastTxDoneTime
                0x00000000200014c8        0x4 /home/ch/RIOT/examples/lorawan/bin/lora-e5-dev/semtech_loramac_mac/LoRaMac.o
 .bss.AggregatedTimeOff
                0x00000000200014cc        0x4 /home/ch/RIOT/examples/lorawan/bin/lora-e5-dev/semtech_loramac_mac/LoRaMac.o
 .bss.Channel   0x00000000200014d0        0x1 /home/ch/RIOT/examples/lorawan/bin/lora-e5-dev/semtech_loramac_mac/LoRaMac.o
 .bss.ChannelsNbRepCounter
                0x00000000200014d1        0x1 /home/ch/RIOT/examples/lorawan/bin/lora-e5-dev/semtech_loramac_mac/LoRaMac.o
 *fill*         0x00000000200014d2        0x2 
 .bss.DownLinkCounter
                0x00000000200014d4        0x4 /home/ch/RIOT/examples/lorawan/bin/lora-e5-dev/semtech_loramac_mac/LoRaMac.o
 .bss.DutyCycleOn
                0x00000000200014d8        0x1 /home/ch/RIOT/examples/lorawan/bin/lora-e5-dev/semtech_loramac_mac/LoRaMac.o
 .bss.IsLoRaMacNetworkJoined
                0x00000000200014d9        0x1 /home/ch/RIOT/examples/lorawan/bin/lora-e5-dev/semtech_loramac_mac/LoRaMac.o
 .bss.IsUpLinkCounterFixed
                0x00000000200014da        0x1 /home/ch/RIOT/examples/lorawan/bin/lora-e5-dev/semtech_loramac_mac/LoRaMac.o
 .bss.LastTxChannel
                0x00000000200014db        0x1 /home/ch/RIOT/examples/lorawan/bin/lora-e5-dev/semtech_loramac_mac/LoRaMac.o
 .bss.LastTxIsJoinRequest
                0x00000000200014dc        0x1 /home/ch/RIOT/examples/lorawan/bin/lora-e5-dev/semtech_loramac_mac/LoRaMac.o
 *fill*         0x00000000200014dd        0x3 
 .bss.LoRaMacAppEui
                0x00000000200014e0        0x4 /home/ch/RIOT/examples/lorawan/bin/lora-e5-dev/semtech_loramac_mac/LoRaMac.o
 .bss.LoRaMacAppKey
                0x00000000200014e4        0x4 /home/ch/RIOT/examples/lorawan/bin/lora-e5-dev/semtech_loramac_mac/LoRaMac.o
 .bss.LoRaMacAppSKey
                0x00000000200014e8       0x10 /home/ch/RIOT/examples/lorawan/bin/lora-e5-dev/semtech_loramac_mac/LoRaMac.o
 .bss.LoRaMacBuffer
                0x00000000200014f8       0xff /home/ch/RIOT/examples/lorawan/bin/lora-e5-dev/semtech_loramac_mac/LoRaMac.o
 *fill*         0x00000000200015f7        0x1 
 .bss.LoRaMacBufferPktLen
                0x00000000200015f8        0x2 /home/ch/RIOT/examples/lorawan/bin/lora-e5-dev/semtech_loramac_mac/LoRaMac.o
 *fill*         0x00000000200015fa        0x2 
 .bss.LoRaMacCallbacks
                0x00000000200015fc        0x4 /home/ch/RIOT/examples/lorawan/bin/lora-e5-dev/semtech_loramac_mac/LoRaMac.o
 .bss.LoRaMacDevAddr
                0x0000000020001600        0x4 /home/ch/RIOT/examples/lorawan/bin/lora-e5-dev/semtech_loramac_mac/LoRaMac.o
 .bss.LoRaMacDevEui
                0x0000000020001604        0x4 /home/ch/RIOT/examples/lorawan/bin/lora-e5-dev/semtech_loramac_mac/LoRaMac.o
 .bss.LoRaMacDevNonce
                0x0000000020001608        0x2 /home/ch/RIOT/examples/lorawan/bin/lora-e5-dev/semtech_loramac_mac/LoRaMac.o
 .bss.LoRaMacDeviceClass
                0x000000002000160a        0x1 /home/ch/RIOT/examples/lorawan/bin/lora-e5-dev/semtech_loramac_mac/LoRaMac.o
 .bss.LoRaMacFlags
                0x000000002000160b        0x1 /home/ch/RIOT/examples/lorawan/bin/lora-e5-dev/semtech_loramac_mac/LoRaMac.o
                0x000000002000160b                LoRaMacFlags
 .bss.LoRaMacInitializationTime
                0x000000002000160c        0x4 /home/ch/RIOT/examples/lorawan/bin/lora-e5-dev/semtech_loramac_mac/LoRaMac.o
 .bss.LoRaMacNetID
                0x0000000020001610        0x4 /home/ch/RIOT/examples/lorawan/bin/lora-e5-dev/semtech_loramac_mac/LoRaMac.o
 .bss.LoRaMacNwkSKey
                0x0000000020001614       0x10 /home/ch/RIOT/examples/lorawan/bin/lora-e5-dev/semtech_loramac_mac/LoRaMac.o
 .bss.LoRaMacParams
                0x0000000020001624       0x38 /home/ch/RIOT/examples/lorawan/bin/lora-e5-dev/semtech_loramac_mac/LoRaMac.o
                0x0000000020001624                LoRaMacParams
 .bss.LoRaMacParamsDefaults
                0x000000002000165c       0x38 /home/ch/RIOT/examples/lorawan/bin/lora-e5-dev/semtech_loramac_mac/LoRaMac.o
                0x000000002000165c                LoRaMacParamsDefaults
 .bss.LoRaMacPrimitives
                0x0000000020001694        0x4 /home/ch/RIOT/examples/lorawan/bin/lora-e5-dev/semtech_loramac_mac/LoRaMac.o
 .bss.LoRaMacRegion
                0x0000000020001698        0x1 /home/ch/RIOT/examples/lorawan/bin/lora-e5-dev/semtech_loramac_mac/LoRaMac.o
 .bss.LoRaMacRxPayload
                0x0000000020001699       0xff /home/ch/RIOT/examples/lorawan/bin/lora-e5-dev/semtech_loramac_mac/LoRaMac.o
 .bss.LoRaMacState
                0x0000000020001798        0x4 /home/ch/RIOT/examples/lorawan/bin/lora-e5-dev/semtech_loramac_mac/LoRaMac.o
                0x0000000020001798                LoRaMacState
 .bss.LoRaMacTxPayloadLen
                0x000000002000179c        0x1 /home/ch/RIOT/examples/lorawan/bin/lora-e5-dev/semtech_loramac_mac/LoRaMac.o
 .bss.MacCommandsBuffer
                0x000000002000179d       0x80 /home/ch/RIOT/examples/lorawan/bin/lora-e5-dev/semtech_loramac_mac/LoRaMac.o
 .bss.MacCommandsBufferIndex
                0x000000002000181d        0x1 /home/ch/RIOT/examples/lorawan/bin/lora-e5-dev/semtech_loramac_mac/LoRaMac.o
 .bss.MacCommandsBufferToRepeat
                0x000000002000181e       0x80 /home/ch/RIOT/examples/lorawan/bin/lora-e5-dev/semtech_loramac_mac/LoRaMac.o
 .bss.MacCommandsBufferToRepeatIndex
                0x000000002000189e        0x1 /home/ch/RIOT/examples/lorawan/bin/lora-e5-dev/semtech_loramac_mac/LoRaMac.o
 .bss.MacCommandsInNextTx
                0x000000002000189f        0x1 /home/ch/RIOT/examples/lorawan/bin/lora-e5-dev/semtech_loramac_mac/LoRaMac.o
 .bss.MacStateCheckTimer
                0x00000000200018a0       0x24 /home/ch/RIOT/examples/lorawan/bin/lora-e5-dev/semtech_loramac_mac/LoRaMac.o
 .bss.MaxDCycle
                0x00000000200018c4        0x1 /home/ch/RIOT/examples/lorawan/bin/lora-e5-dev/semtech_loramac_mac/LoRaMac.o
 *fill*         0x00000000200018c5        0x3 
 .bss.McpsConfirm
                0x00000000200018c8       0x14 /home/ch/RIOT/examples/lorawan/bin/lora-e5-dev/semtech_loramac_mac/LoRaMac.o
 .bss.McpsIndication
                0x00000000200018dc       0x18 /home/ch/RIOT/examples/lorawan/bin/lora-e5-dev/semtech_loramac_mac/LoRaMac.o
 .bss.MlmeConfirm
                0x00000000200018f4        0xc /home/ch/RIOT/examples/lorawan/bin/lora-e5-dev/semtech_loramac_mac/LoRaMac.o
 .bss.MlmeIndication
                0x0000000020001900        0x1 /home/ch/RIOT/examples/lorawan/bin/lora-e5-dev/semtech_loramac_mac/LoRaMac.o
 *fill*         0x0000000020001901        0x3 
 .bss.MulticastChannels
                0x0000000020001904        0x4 /home/ch/RIOT/examples/lorawan/bin/lora-e5-dev/semtech_loramac_mac/LoRaMac.o
 .bss.NodeAckRequested
                0x0000000020001908        0x1 /home/ch/RIOT/examples/lorawan/bin/lora-e5-dev/semtech_loramac_mac/LoRaMac.o
 .bss.PublicNetwork
                0x0000000020001909        0x1 /home/ch/RIOT/examples/lorawan/bin/lora-e5-dev/semtech_loramac_mac/LoRaMac.o
 .bss.RepeaterSupport
                0x000000002000190a        0x1 /home/ch/RIOT/examples/lorawan/bin/lora-e5-dev/semtech_loramac_mac/LoRaMac.o
 .bss.RxSlot    0x000000002000190b        0x1 /home/ch/RIOT/examples/lorawan/bin/lora-e5-dev/semtech_loramac_mac/LoRaMac.o
 .bss.RxWindow1Config
                0x000000002000190c       0x14 /home/ch/RIOT/examples/lorawan/bin/lora-e5-dev/semtech_loramac_mac/LoRaMac.o
 .bss.RxWindow1Delay
                0x0000000020001920        0x4 /home/ch/RIOT/examples/lorawan/bin/lora-e5-dev/semtech_loramac_mac/LoRaMac.o
 .bss.RxWindow2Config
                0x0000000020001924       0x14 /home/ch/RIOT/examples/lorawan/bin/lora-e5-dev/semtech_loramac_mac/LoRaMac.o
 .bss.RxWindow2Delay
                0x0000000020001938        0x4 /home/ch/RIOT/examples/lorawan/bin/lora-e5-dev/semtech_loramac_mac/LoRaMac.o
 .bss.RxWindowTimer1
                0x000000002000193c       0x24 /home/ch/RIOT/examples/lorawan/bin/lora-e5-dev/semtech_loramac_mac/LoRaMac.o
 .bss.RxWindowTimer2
                0x0000000020001960       0x24 /home/ch/RIOT/examples/lorawan/bin/lora-e5-dev/semtech_loramac_mac/LoRaMac.o
 .bss.SrvAckRequested
                0x0000000020001984        0x1 /home/ch/RIOT/examples/lorawan/bin/lora-e5-dev/semtech_loramac_mac/LoRaMac.o
 *fill*         0x0000000020001985        0x3 
 .bss.TxDelayedTimer
                0x0000000020001988       0x24 /home/ch/RIOT/examples/lorawan/bin/lora-e5-dev/semtech_loramac_mac/LoRaMac.o
 .bss.TxTimeOnAir
                0x00000000200019ac        0x4 /home/ch/RIOT/examples/lorawan/bin/lora-e5-dev/semtech_loramac_mac/LoRaMac.o
                0x00000000200019ac                TxTimeOnAir
 .bss.UpLinkCounter
                0x00000000200019b0        0x4 /home/ch/RIOT/examples/lorawan/bin/lora-e5-dev/semtech_loramac_mac/LoRaMac.o
 .bss.Channels  0x00000000200019b4       0xc0 /home/ch/RIOT/examples/lorawan/bin/lora-e5-dev/semtech_loramac_mac_region/RegionEU868.o
 .bss.ChannelsDefaultMask
                0x0000000020001a74        0x2 /home/ch/RIOT/examples/lorawan/bin/lora-e5-dev/semtech_loramac_mac_region/RegionEU868.o
 .bss.ChannelsMask
                0x0000000020001a76        0x2 /home/ch/RIOT/examples/lorawan/bin/lora-e5-dev/semtech_loramac_mac_region/RegionEU868.o
 .bss._dev      0x0000000020001a78        0x4 /home/ch/RIOT/examples/lorawan/bin/lora-e5-dev/sx126x/sx126x_netdev.o
 .bss._in_handler
                0x0000000020001a7c        0x4 /home/ch/RIOT/examples/lorawan/bin/lora-e5-dev/xtimer/xtimer_core.o
 .bss._lltimer_ongoing
                0x0000000020001a80        0x1 /home/ch/RIOT/examples/lorawan/bin/lora-e5-dev/xtimer/xtimer_core.o
 *fill*         0x0000000020001a81        0x7 
 .bss._xtimer_current_time
                0x0000000020001a88        0x8 /home/ch/RIOT/examples/lorawan/bin/lora-e5-dev/xtimer/xtimer_core.o
                0x0000000020001a88                _xtimer_current_time
 .bss.long_list_head
                0x0000000020001a90        0x4 /home/ch/RIOT/examples/lorawan/bin/lora-e5-dev/xtimer/xtimer_core.o
 .bss.timer_list_head
                0x0000000020001a94        0x4 /home/ch/RIOT/examples/lorawan/bin/lora-e5-dev/xtimer/xtimer_core.o
 .bss._ztimer_convert_frac_msec
                0x0000000020001a98       0x4c /home/ch/RIOT/examples/lorawan/bin/lora-e5-dev/ztimer_core/init.o
 .bss._ztimer_periph_timer_rtt
                0x0000000020001ae4       0x24 /home/ch/RIOT/examples/lorawan/bin/lora-e5-dev/ztimer_core/init.o
 .bss           0x0000000020001b08        0x8 /usr/lib/gcc/arm-none-eabi/9.2.1/../../../arm-none-eabi/lib/thumb/v7e-m/nofp/libc_nano.a(lib_a-nano-mallocr.o)
                0x0000000020001b08                __malloc_free_list
                0x0000000020001b0c                __malloc_sbrk_start
 *(COMMON)
                0x0000000020001b10                . = ALIGN (0x4)
                0x0000000020001b10                _ebss = .
                0x0000000020001b10                _ezero = .

.noinit         0x0000000020001b10        0x0 load address 0x000000000800da88
                0x0000000020001b10                __noinit_start = .
 *(.noinit)
                0x0000000020001b10                . = ALIGN (0x4)
                0x0000000020001b10                __noinit_end = .
                0x0000000020001b10                . = ALIGN (0x4)
                0x0000000020001b10                _sheap = .
                0x0000000020010000                _eheap = (ORIGIN (ram) + LENGTH (ram))
                0x0000000020000000                _sram = ORIGIN (ram)
                0x0000000020010000                _eram = (ORIGIN (ram) + LENGTH (ram))
                0x0000000008000000                _srom = ORIGIN (rom)
                0x0000000008040000                _erom = (ORIGIN (rom) + LENGTH (rom))
                0x000000000800da88                _sbackup_data_load = LOADADDR (.backup.data)

.backup.data    0x0000000000000000        0x0 load address 0x000000000800da88
                0x0000000000000000                _sbackup_data = .
 *(.backup.data)
                0x0000000000000000                _ebackup_data = .
                0x0000000000000000                . = ALIGN (0x4)

.backup.bss     0x0000000000000000        0x0 load address 0x000000000800da88
                0x0000000000000000                _sbackup_bss = .
 *(.backup.bss)
                0x0000000000000000                _ebackup_bss = .
                0x0000000000000000                . = ALIGN (0x4)

.heap3          0x0000000000000000        0x0 load address 0x000000000800da88
                0x0000000000000000                _sheap1 = .
                0x0000000000000000                _eheap1 = (ORIGIN (bkup_ram) + LENGTH (bkup_ram))

.end_fw         0x000000000800da88        0x0
                0x000000000800da88                _end_fw = .
OUTPUT(/home/ch/RIOT/examples/lorawan/bin/lora-e5-dev/lorawan.elf elf32-littlearm)
LOAD linker stubs

.debug_info     0x0000000000000000    0x8f6c3
 .debug_info    0x0000000000000000     0x277a /home/ch/RIOT/examples/lorawan/bin/lora-e5-dev/application_lorawan/main.o
 .debug_info    0x000000000000277a      0xd71 /home/ch/RIOT/examples/lorawan/bin/lora-e5-dev/auto_init/auto_init.o
 .debug_info    0x00000000000034eb     0x213d /home/ch/RIOT/examples/lorawan/bin/lora-e5-dev/board/board.o
 .debug_info    0x0000000000005628      0xe90 /home/ch/RIOT/examples/lorawan/bin/lora-e5-dev/core/init.o
 .debug_info    0x00000000000064b8     0x2860 /home/ch/RIOT/examples/lorawan/bin/lora-e5-dev/core/msg.o
 .debug_info    0x0000000000008d18     0x1b99 /home/ch/RIOT/examples/lorawan/bin/lora-e5-dev/core/mutex.o
 .debug_info    0x000000000000a8b1      0xf0b /home/ch/RIOT/examples/lorawan/bin/lora-e5-dev/core/panic.o
 .debug_info    0x000000000000b7bc     0x14b1 /home/ch/RIOT/examples/lorawan/bin/lora-e5-dev/core/sched.o
 .debug_info    0x000000000000cc6d     0x1e7a /home/ch/RIOT/examples/lorawan/bin/lora-e5-dev/core/thread.o
 .debug_info    0x000000000000eae7     0x1386 /home/ch/RIOT/examples/lorawan/bin/lora-e5-dev/cortexm_common/cortexm_init.o
 .debug_info    0x000000000000fe6d      0xd6b /home/ch/RIOT/examples/lorawan/bin/lora-e5-dev/cortexm_common/panic.o
 .debug_info    0x0000000000010bd8     0x12a1 /home/ch/RIOT/examples/lorawan/bin/lora-e5-dev/cortexm_common/thread_arch.o
 .debug_info    0x0000000000011e79     0x201c /home/ch/RIOT/examples/lorawan/bin/lora-e5-dev/cortexm_common/vectors_cortexm.o
 .debug_info    0x0000000000013e95     0x18d9 /home/ch/RIOT/examples/lorawan/bin/lora-e5-dev/cpu/cpu_common.o
 .debug_info    0x000000000001576e     0x1636 /home/ch/RIOT/examples/lorawan/bin/lora-e5-dev/cpu/cpu_init.o
 .debug_info    0x0000000000016da4     0x110a /home/ch/RIOT/examples/lorawan/bin/lora-e5-dev/crypto/aes.o
 .debug_info    0x0000000000017eae     0x2fc0 /home/ch/RIOT/examples/lorawan/bin/lora-e5-dev/driver_sx126x_hal/driver_sx126x_hal.o
 .debug_info    0x000000000001ae6e     0x42cb /home/ch/RIOT/examples/lorawan/bin/lora-e5-dev/driver_sx126x/sx126x.o
 .debug_info    0x000000000001f139     0x20a0 /home/ch/RIOT/examples/lorawan/bin/lora-e5-dev/fmt/fmt.o
 .debug_info    0x00000000000211d9      0xf73 /home/ch/RIOT/examples/lorawan/bin/lora-e5-dev/frac/frac.o
 .debug_info    0x000000000002214c     0x1a7b /home/ch/RIOT/examples/lorawan/bin/lora-e5-dev/luid/luid.o
 .debug_info    0x0000000000023bc7     0x10e0 /home/ch/RIOT/examples/lorawan/bin/lora-e5-dev/malloc_thread_safe/malloc_wrappers.o
 .debug_info    0x0000000000024ca7     0x271d /home/ch/RIOT/examples/lorawan/bin/lora-e5-dev/newlib_syscalls_default/syscalls.o
 .debug_info    0x00000000000273c4      0xcd1 /home/ch/RIOT/examples/lorawan/bin/lora-e5-dev/periph_common/cpuid.o
 .debug_info    0x0000000000028095     0x15cf /home/ch/RIOT/examples/lorawan/bin/lora-e5-dev/periph_common/init.o
 .debug_info    0x0000000000029664     0x16d4 /home/ch/RIOT/examples/lorawan/bin/lora-e5-dev/periph_common/timer.o
 .debug_info    0x000000000002ad38     0x26f7 /home/ch/RIOT/examples/lorawan/bin/lora-e5-dev/periph/gpio_all.o
 .debug_info    0x000000000002d42f     0x28a1 /home/ch/RIOT/examples/lorawan/bin/lora-e5-dev/periph/i2c_1.o
 .debug_info    0x000000000002fcd0     0x11a8 /home/ch/RIOT/examples/lorawan/bin/lora-e5-dev/periph/pm.o
 .debug_info    0x0000000000030e78     0x2346 /home/ch/RIOT/examples/lorawan/bin/lora-e5-dev/periph/rtt_all.o
 .debug_info    0x00000000000331be     0x1fbc /home/ch/RIOT/examples/lorawan/bin/lora-e5-dev/periph/spi.o
 .debug_info    0x000000000003517a     0x1ec4 /home/ch/RIOT/examples/lorawan/bin/lora-e5-dev/periph/timer.o
 .debug_info    0x000000000003703e     0x2236 /home/ch/RIOT/examples/lorawan/bin/lora-e5-dev/periph/uart.o
 .debug_info    0x0000000000039274     0x11b7 /home/ch/RIOT/examples/lorawan/bin/lora-e5-dev/pm_layered/pm.o
 .debug_info    0x000000000003a42b       0xd5 /home/ch/RIOT/examples/lorawan/bin/lora-e5-dev/random/musl_lcg.o
 .debug_info    0x000000000003a500      0xeb6 /home/ch/RIOT/examples/lorawan/bin/lora-e5-dev/random/random.o
 .debug_info    0x000000000003b3b6      0xb93 /home/ch/RIOT/examples/lorawan/bin/lora-e5-dev/semtech_loramac_arch/utilities.o
 .debug_info    0x000000000003bf49     0x30a0 /home/ch/RIOT/examples/lorawan/bin/lora-e5-dev/semtech_loramac_contrib/semtech_loramac_getset.o
 .debug_info    0x000000000003efe9     0x388e /home/ch/RIOT/examples/lorawan/bin/lora-e5-dev/semtech_loramac_contrib/semtech_loramac.o
 .debug_info    0x0000000000042877     0x3682 /home/ch/RIOT/examples/lorawan/bin/lora-e5-dev/semtech_loramac_contrib/semtech_loramac_radio.o
 .debug_info    0x0000000000045ef9     0x12df /home/ch/RIOT/examples/lorawan/bin/lora-e5-dev/semtech_loramac_contrib/semtech_loramac_timer.o
 .debug_info    0x00000000000471d8      0xe83 /home/ch/RIOT/examples/lorawan/bin/lora-e5-dev/semtech_loramac_crypto/cmac.o
 .debug_info    0x000000000004805b     0x1208 /home/ch/RIOT/examples/lorawan/bin/lora-e5-dev/semtech_loramac_mac/LoRaMacCrypto.o
 .debug_info    0x0000000000049263     0x55b0 /home/ch/RIOT/examples/lorawan/bin/lora-e5-dev/semtech_loramac_mac/LoRaMac.o
 .debug_info    0x000000000004e813     0x1feb /home/ch/RIOT/examples/lorawan/bin/lora-e5-dev/semtech_loramac_mac_region/RegionCommon.o
 .debug_info    0x00000000000507fe     0x32a4 /home/ch/RIOT/examples/lorawan/bin/lora-e5-dev/semtech_loramac_mac_region/RegionEU868.o
 .debug_info    0x0000000000053aa2     0x28f4 /home/ch/RIOT/examples/lorawan/bin/lora-e5-dev/semtech_loramac_mac_region/Region.o
 .debug_info    0x0000000000056396     0x16c6 /home/ch/RIOT/examples/lorawan/bin/lora-e5-dev/stdio_uart/stdio_uart.o
 .debug_info    0x0000000000057a5c     0x195f /home/ch/RIOT/examples/lorawan/bin/lora-e5-dev/stm32_clk/stmclk_common.o
 .debug_info    0x00000000000593bb     0x19ee /home/ch/RIOT/examples/lorawan/bin/lora-e5-dev/stm32_clk/stmclk_l4wx.o
 .debug_info    0x000000000005ada9      0x2a0 /home/ch/RIOT/examples/lorawan/bin/lora-e5-dev/stm32_vectors/STM32WLE5xx.o
 .debug_info    0x000000000005b049     0x341e /home/ch/RIOT/examples/lorawan/bin/lora-e5-dev/sx126x/sx126x_netdev.o
 .debug_info    0x000000000005e467     0x2bef /home/ch/RIOT/examples/lorawan/bin/lora-e5-dev/sx126x/sx126x.o
 .debug_info    0x0000000000061056     0x2338 /home/ch/RIOT/examples/lorawan/bin/lora-e5-dev/xtimer/xtimer_core.o
 .debug_info    0x000000000006338e     0x13cf /home/ch/RIOT/examples/lorawan/bin/lora-e5-dev/ztimer_core/convert_frac.o
 .debug_info    0x000000000006475d      0xfc6 /home/ch/RIOT/examples/lorawan/bin/lora-e5-dev/ztimer_core/convert.o
 .debug_info    0x0000000000065723     0x1db7 /home/ch/RIOT/examples/lorawan/bin/lora-e5-dev/ztimer_core/core.o
 .debug_info    0x00000000000674da     0x19e1 /home/ch/RIOT/examples/lorawan/bin/lora-e5-dev/ztimer_core/init.o
 .debug_info    0x0000000000068ebb     0x19d2 /home/ch/RIOT/examples/lorawan/bin/lora-e5-dev/ztimer_core/periph_rtt.o
 .debug_info    0x000000000006a88d     0x1a33 /home/ch/RIOT/examples/lorawan/bin/lora-e5-dev/ztimer_core/periph_timer.o
 .debug_info    0x000000000006c2c0     0x1c80 /home/ch/RIOT/examples/lorawan/bin/lora-e5-dev/ztimer_core/util.o
 .debug_info    0x000000000006df40      0xa8a /usr/lib/gcc/arm-none-eabi/9.2.1/../../../arm-none-eabi/lib/thumb/v7e-m/nofp/libm.a(lib_a-s_ceil.o)
 .debug_info    0x000000000006e9ca      0xa8a /usr/lib/gcc/arm-none-eabi/9.2.1/../../../arm-none-eabi/lib/thumb/v7e-m/nofp/libm.a(lib_a-s_floor.o)
 .debug_info    0x000000000006f454       0x26 /usr/lib/gcc/arm-none-eabi/9.2.1/thumb/v7e-m/nofp/libgcc.a(_arm_addsubdf3.o)
 .debug_info    0x000000000006f47a       0x26 /usr/lib/gcc/arm-none-eabi/9.2.1/thumb/v7e-m/nofp/libgcc.a(_arm_muldivdf3.o)
 .debug_info    0x000000000006f4a0       0x26 /usr/lib/gcc/arm-none-eabi/9.2.1/thumb/v7e-m/nofp/libgcc.a(_arm_cmpdf2.o)
 .debug_info    0x000000000006f4c6       0x26 /usr/lib/gcc/arm-none-eabi/9.2.1/thumb/v7e-m/nofp/libgcc.a(_arm_fixdfsi.o)
 .debug_info    0x000000000006f4ec       0x26 /usr/lib/gcc/arm-none-eabi/9.2.1/thumb/v7e-m/nofp/libgcc.a(_arm_fixunsdfsi.o)
 .debug_info    0x000000000006f512       0x26 /usr/lib/gcc/arm-none-eabi/9.2.1/thumb/v7e-m/nofp/libgcc.a(_arm_addsubsf3.o)
 .debug_info    0x000000000006f538      0x92a /usr/lib/gcc/arm-none-eabi/9.2.1/../../../arm-none-eabi/lib/thumb/v7e-m/nofp/libc_nano.a(lib_a-impure.o)
 .debug_info    0x000000000006fe62      0x11a /usr/lib/gcc/arm-none-eabi/9.2.1/../../../arm-none-eabi/lib/thumb/v7e-m/nofp/libc_nano.a(lib_a-init.o)
 .debug_info    0x000000000006ff7c      0x9b6 /usr/lib/gcc/arm-none-eabi/9.2.1/../../../arm-none-eabi/lib/thumb/v7e-m/nofp/libc_nano.a(lib_a-malloc.o)
 .debug_info    0x0000000000070932       0x26 /usr/lib/gcc/arm-none-eabi/9.2.1/../../../arm-none-eabi/lib/thumb/v7e-m/nofp/libc_nano.a(lib_a-memcpy.o)
 .debug_info    0x0000000000070958      0xf2b /usr/lib/gcc/arm-none-eabi/9.2.1/../../../arm-none-eabi/lib/thumb/v7e-m/nofp/libc_nano.a(lib_a-memmove.o)
 .debug_info    0x0000000000071883      0xf21 /usr/lib/gcc/arm-none-eabi/9.2.1/../../../arm-none-eabi/lib/thumb/v7e-m/nofp/libc_nano.a(lib_a-memset.o)
 .debug_info    0x00000000000727a4      0xb85 /usr/lib/gcc/arm-none-eabi/9.2.1/../../../arm-none-eabi/lib/thumb/v7e-m/nofp/libc_nano.a(lib_a-nano-freer.o)
 .debug_info    0x0000000000073329      0xc5a /usr/lib/gcc/arm-none-eabi/9.2.1/../../../arm-none-eabi/lib/thumb/v7e-m/nofp/libc_nano.a(lib_a-nano-mallocr.o)
 .debug_info    0x0000000000073f83     0x1adb /usr/lib/gcc/arm-none-eabi/9.2.1/../../../arm-none-eabi/lib/thumb/v7e-m/nofp/libc_nano.a(lib_a-nano-vfprintf_float.o)
 .debug_info    0x0000000000075a5e     0x1592 /usr/lib/gcc/arm-none-eabi/9.2.1/../../../arm-none-eabi/lib/thumb/v7e-m/nofp/libc_nano.a(lib_a-nano-vfprintf_i.o)
 .debug_info    0x0000000000076ff0      0xc67 /usr/lib/gcc/arm-none-eabi/9.2.1/../../../arm-none-eabi/lib/thumb/v7e-m/nofp/libc_nano.a(lib_a-printf.o)
 .debug_info    0x0000000000077c57      0xd13 /usr/lib/gcc/arm-none-eabi/9.2.1/../../../arm-none-eabi/lib/thumb/v7e-m/nofp/libc_nano.a(lib_a-puts.o)
 .debug_info    0x000000000007896a       0x26 /usr/lib/gcc/arm-none-eabi/9.2.1/../../../arm-none-eabi/lib/thumb/v7e-m/nofp/libc_nano.a(lib_a-strlen.o)
 .debug_info    0x0000000000078990      0xc90 /usr/lib/gcc/arm-none-eabi/9.2.1/../../../arm-none-eabi/lib/thumb/v7e-m/nofp/libc_nano.a(lib_a-wbuf.o)
 .debug_info    0x0000000000079620      0xbfa /usr/lib/gcc/arm-none-eabi/9.2.1/../../../arm-none-eabi/lib/thumb/v7e-m/nofp/libc_nano.a(lib_a-wsetup.o)
 .debug_info    0x000000000007a21a     0x1b3c /usr/lib/gcc/arm-none-eabi/9.2.1/../../../arm-none-eabi/lib/thumb/v7e-m/nofp/libc_nano.a(lib_a-dtoa.o)
 .debug_info    0x000000000007bd56      0xd73 /usr/lib/gcc/arm-none-eabi/9.2.1/../../../arm-none-eabi/lib/thumb/v7e-m/nofp/libc_nano.a(lib_a-fflush.o)
 .debug_info    0x000000000007cac9     0x11a8 /usr/lib/gcc/arm-none-eabi/9.2.1/../../../arm-none-eabi/lib/thumb/v7e-m/nofp/libc_nano.a(lib_a-findfp.o)
 .debug_info    0x000000000007dc71      0xa7a /usr/lib/gcc/arm-none-eabi/9.2.1/../../../arm-none-eabi/lib/thumb/v7e-m/nofp/libc_nano.a(lib_a-fprintf.o)
 .debug_info    0x000000000007e6eb      0xca4 /usr/lib/gcc/arm-none-eabi/9.2.1/../../../arm-none-eabi/lib/thumb/v7e-m/nofp/libc_nano.a(lib_a-fwalk.o)
 .debug_info    0x000000000007f38f      0xf49 /usr/lib/gcc/arm-none-eabi/9.2.1/../../../arm-none-eabi/lib/thumb/v7e-m/nofp/libc_nano.a(lib_a-localeconv.o)
 .debug_info    0x00000000000802d8      0xf68 /usr/lib/gcc/arm-none-eabi/9.2.1/../../../arm-none-eabi/lib/thumb/v7e-m/nofp/libc_nano.a(lib_a-makebuf.o)
 .debug_info    0x0000000000081240       0x26 /usr/lib/gcc/arm-none-eabi/9.2.1/../../../arm-none-eabi/lib/thumb/v7e-m/nofp/libc_nano.a(lib_a-memchr.o)
 .debug_info    0x0000000000081266      0x961 /usr/lib/gcc/arm-none-eabi/9.2.1/../../../arm-none-eabi/lib/thumb/v7e-m/nofp/libc_nano.a(lib_a-mlock.o)
 .debug_info    0x0000000000081bc7     0x240f /usr/lib/gcc/arm-none-eabi/9.2.1/../../../arm-none-eabi/lib/thumb/v7e-m/nofp/libc_nano.a(lib_a-mprec.o)
 .debug_info    0x0000000000083fd6      0xafe /usr/lib/gcc/arm-none-eabi/9.2.1/../../../arm-none-eabi/lib/thumb/v7e-m/nofp/libc_nano.a(lib_a-nano-callocr.o)
 .debug_info    0x0000000000084ad4      0xb77 /usr/lib/gcc/arm-none-eabi/9.2.1/../../../arm-none-eabi/lib/thumb/v7e-m/nofp/libc_nano.a(lib_a-nano-reallocr.o)
 .debug_info    0x000000000008564b     0x176a /usr/lib/gcc/arm-none-eabi/9.2.1/../../../arm-none-eabi/lib/thumb/v7e-m/nofp/libc_nano.a(lib_a-nano-vfprintf.o)
 .debug_info    0x0000000000086db5      0xe67 /usr/lib/gcc/arm-none-eabi/9.2.1/../../../arm-none-eabi/lib/thumb/v7e-m/nofp/libc_nano.a(lib_a-stdio.o)
 .debug_info    0x0000000000087c1c      0xa41 /usr/lib/gcc/arm-none-eabi/9.2.1/../../../arm-none-eabi/lib/thumb/v7e-m/nofp/libc_nano.a(lib_a-assert.o)
 .debug_info    0x000000000008865d      0xeed /usr/lib/gcc/arm-none-eabi/9.2.1/../../../arm-none-eabi/lib/thumb/v7e-m/nofp/libc_nano.a(lib_a-fvwrite.o)
 .debug_info    0x000000000008954a     0x10ca /usr/lib/gcc/arm-none-eabi/9.2.1/../../../arm-none-eabi/lib/thumb/v7e-m/nofp/libc_nano.a(lib_a-locale.o)
 .debug_info    0x000000000008a614     0x1044 /usr/lib/gcc/arm-none-eabi/9.2.1/../../../arm-none-eabi/lib/thumb/v7e-m/nofp/libc_nano.a(lib_a-mbtowc_r.o)
 .debug_info    0x000000000008b658      0xaa6 /usr/lib/gcc/arm-none-eabi/9.2.1/../../../arm-none-eabi/lib/thumb/v7e-m/nofp/libc_nano.a(lib_a-nano-msizer.o)
 .debug_info    0x000000000008c0fe      0xffd /usr/lib/gcc/arm-none-eabi/9.2.1/../../../arm-none-eabi/lib/thumb/v7e-m/nofp/libc_nano.a(lib_a-wctomb_r.o)
 .debug_info    0x000000000008d0fb      0x9b5 /usr/lib/gcc/arm-none-eabi/9.2.1/../../../arm-none-eabi/lib/thumb/v7e-m/nofp/libc_nano.a(lib_a-abort.o)
 .debug_info    0x000000000008dab0      0xe91 /usr/lib/gcc/arm-none-eabi/9.2.1/../../../arm-none-eabi/lib/thumb/v7e-m/nofp/libc_nano.a(lib_a-ctype_.o)
 .debug_info    0x000000000008e941      0xd5c /usr/lib/gcc/arm-none-eabi/9.2.1/../../../arm-none-eabi/lib/thumb/v7e-m/nofp/libc_nano.a(lib_a-signal.o)
 .debug_info    0x000000000008f69d       0x26 /usr/lib/gcc/arm-none-eabi/9.2.1/thumb/v7e-m/nofp/libgcc.a(_arm_unorddf2.o)

.debug_abbrev   0x0000000000000000    0x14d5e
 .debug_abbrev  0x0000000000000000      0x3c1 /home/ch/RIOT/examples/lorawan/bin/lora-e5-dev/application_lorawan/main.o
 .debug_abbrev  0x00000000000003c1      0x245 /home/ch/RIOT/examples/lorawan/bin/lora-e5-dev/auto_init/auto_init.o
 .debug_abbrev  0x0000000000000606      0x32d /home/ch/RIOT/examples/lorawan/bin/lora-e5-dev/board/board.o
 .debug_abbrev  0x0000000000000933      0x32c /home/ch/RIOT/examples/lorawan/bin/lora-e5-dev/core/init.o
 .debug_abbrev  0x0000000000000c5f      0x58a /home/ch/RIOT/examples/lorawan/bin/lora-e5-dev/core/msg.o
 .debug_abbrev  0x00000000000011e9      0x40d /home/ch/RIOT/examples/lorawan/bin/lora-e5-dev/core/mutex.o
 .debug_abbrev  0x00000000000015f6      0x364 /home/ch/RIOT/examples/lorawan/bin/lora-e5-dev/core/panic.o
 .debug_abbrev  0x000000000000195a      0x4d7 /home/ch/RIOT/examples/lorawan/bin/lora-e5-dev/core/sched.o
 .debug_abbrev  0x0000000000001e31      0x532 /home/ch/RIOT/examples/lorawan/bin/lora-e5-dev/core/thread.o
 .debug_abbrev  0x0000000000002363      0x3b5 /home/ch/RIOT/examples/lorawan/bin/lora-e5-dev/cortexm_common/cortexm_init.o
 .debug_abbrev  0x0000000000002718      0x2fe /home/ch/RIOT/examples/lorawan/bin/lora-e5-dev/cortexm_common/panic.o
 .debug_abbrev  0x0000000000002a16      0x48e /home/ch/RIOT/examples/lorawan/bin/lora-e5-dev/cortexm_common/thread_arch.o
 .debug_abbrev  0x0000000000002ea4      0x4a6 /home/ch/RIOT/examples/lorawan/bin/lora-e5-dev/cortexm_common/vectors_cortexm.o
 .debug_abbrev  0x000000000000334a      0x37d /home/ch/RIOT/examples/lorawan/bin/lora-e5-dev/cpu/cpu_common.o
 .debug_abbrev  0x00000000000036c7      0x2ee /home/ch/RIOT/examples/lorawan/bin/lora-e5-dev/cpu/cpu_init.o
 .debug_abbrev  0x00000000000039b5      0x333 /home/ch/RIOT/examples/lorawan/bin/lora-e5-dev/crypto/aes.o
 .debug_abbrev  0x0000000000003ce8      0x420 /home/ch/RIOT/examples/lorawan/bin/lora-e5-dev/driver_sx126x_hal/driver_sx126x_hal.o
 .debug_abbrev  0x0000000000004108      0x40f /home/ch/RIOT/examples/lorawan/bin/lora-e5-dev/driver_sx126x/sx126x.o
 .debug_abbrev  0x0000000000004517      0x50b /home/ch/RIOT/examples/lorawan/bin/lora-e5-dev/fmt/fmt.o
 .debug_abbrev  0x0000000000004a22      0x327 /home/ch/RIOT/examples/lorawan/bin/lora-e5-dev/frac/frac.o
 .debug_abbrev  0x0000000000004d49      0x399 /home/ch/RIOT/examples/lorawan/bin/lora-e5-dev/luid/luid.o
 .debug_abbrev  0x00000000000050e2      0x3f1 /home/ch/RIOT/examples/lorawan/bin/lora-e5-dev/malloc_thread_safe/malloc_wrappers.o
 .debug_abbrev  0x00000000000054d3      0x58f /home/ch/RIOT/examples/lorawan/bin/lora-e5-dev/newlib_syscalls_default/syscalls.o
 .debug_abbrev  0x0000000000005a62      0x2ad /home/ch/RIOT/examples/lorawan/bin/lora-e5-dev/periph_common/cpuid.o
 .debug_abbrev  0x0000000000005d0f      0x2f9 /home/ch/RIOT/examples/lorawan/bin/lora-e5-dev/periph_common/init.o
 .debug_abbrev  0x0000000000006008      0x3a8 /home/ch/RIOT/examples/lorawan/bin/lora-e5-dev/periph_common/timer.o
 .debug_abbrev  0x00000000000063b0      0x502 /home/ch/RIOT/examples/lorawan/bin/lora-e5-dev/periph/gpio_all.o
 .debug_abbrev  0x00000000000068b2      0x596 /home/ch/RIOT/examples/lorawan/bin/lora-e5-dev/periph/i2c_1.o
 .debug_abbrev  0x0000000000006e48      0x3cc /home/ch/RIOT/examples/lorawan/bin/lora-e5-dev/periph/pm.o
 .debug_abbrev  0x0000000000007214      0x4a1 /home/ch/RIOT/examples/lorawan/bin/lora-e5-dev/periph/rtt_all.o
 .debug_abbrev  0x00000000000076b5      0x4e9 /home/ch/RIOT/examples/lorawan/bin/lora-e5-dev/periph/spi.o
 .debug_abbrev  0x0000000000007b9e      0x47e /home/ch/RIOT/examples/lorawan/bin/lora-e5-dev/periph/timer.o
 .debug_abbrev  0x000000000000801c      0x52b /home/ch/RIOT/examples/lorawan/bin/lora-e5-dev/periph/uart.o
 .debug_abbrev  0x0000000000008547      0x3a1 /home/ch/RIOT/examples/lorawan/bin/lora-e5-dev/pm_layered/pm.o
 .debug_abbrev  0x00000000000088e8       0x97 /home/ch/RIOT/examples/lorawan/bin/lora-e5-dev/random/musl_lcg.o
 .debug_abbrev  0x000000000000897f      0x2c9 /home/ch/RIOT/examples/lorawan/bin/lora-e5-dev/random/random.o
 .debug_abbrev  0x0000000000008c48      0x257 /home/ch/RIOT/examples/lorawan/bin/lora-e5-dev/semtech_loramac_arch/utilities.o
 .debug_abbrev  0x0000000000008e9f      0x4eb /home/ch/RIOT/examples/lorawan/bin/lora-e5-dev/semtech_loramac_contrib/semtech_loramac_getset.o
 .debug_abbrev  0x000000000000938a      0x62c /home/ch/RIOT/examples/lorawan/bin/lora-e5-dev/semtech_loramac_contrib/semtech_loramac.o
 .debug_abbrev  0x00000000000099b6      0x5d3 /home/ch/RIOT/examples/lorawan/bin/lora-e5-dev/semtech_loramac_contrib/semtech_loramac_radio.o
 .debug_abbrev  0x0000000000009f89      0x3be /home/ch/RIOT/examples/lorawan/bin/lora-e5-dev/semtech_loramac_contrib/semtech_loramac_timer.o
 .debug_abbrev  0x000000000000a347      0x264 /home/ch/RIOT/examples/lorawan/bin/lora-e5-dev/semtech_loramac_crypto/cmac.o
 .debug_abbrev  0x000000000000a5ab      0x252 /home/ch/RIOT/examples/lorawan/bin/lora-e5-dev/semtech_loramac_mac/LoRaMacCrypto.o
 .debug_abbrev  0x000000000000a7fd      0x66d /home/ch/RIOT/examples/lorawan/bin/lora-e5-dev/semtech_loramac_mac/LoRaMac.o
 .debug_abbrev  0x000000000000ae6a      0x50d /home/ch/RIOT/examples/lorawan/bin/lora-e5-dev/semtech_loramac_mac_region/RegionCommon.o
 .debug_abbrev  0x000000000000b377      0x54c /home/ch/RIOT/examples/lorawan/bin/lora-e5-dev/semtech_loramac_mac_region/RegionEU868.o
 .debug_abbrev  0x000000000000b8c3      0x398 /home/ch/RIOT/examples/lorawan/bin/lora-e5-dev/semtech_loramac_mac_region/Region.o
 .debug_abbrev  0x000000000000bc5b      0x344 /home/ch/RIOT/examples/lorawan/bin/lora-e5-dev/stdio_uart/stdio_uart.o
 .debug_abbrev  0x000000000000bf9f      0x2fb /home/ch/RIOT/examples/lorawan/bin/lora-e5-dev/stm32_clk/stmclk_common.o
 .debug_abbrev  0x000000000000c29a      0x39b /home/ch/RIOT/examples/lorawan/bin/lora-e5-dev/stm32_clk/stmclk_l4wx.o
 .debug_abbrev  0x000000000000c635       0xf4 /home/ch/RIOT/examples/lorawan/bin/lora-e5-dev/stm32_vectors/STM32WLE5xx.o
 .debug_abbrev  0x000000000000c729      0x5b3 /home/ch/RIOT/examples/lorawan/bin/lora-e5-dev/sx126x/sx126x_netdev.o
 .debug_abbrev  0x000000000000ccdc      0x526 /home/ch/RIOT/examples/lorawan/bin/lora-e5-dev/sx126x/sx126x.o
 .debug_abbrev  0x000000000000d202      0x586 /home/ch/RIOT/examples/lorawan/bin/lora-e5-dev/xtimer/xtimer_core.o
 .debug_abbrev  0x000000000000d788      0x41d /home/ch/RIOT/examples/lorawan/bin/lora-e5-dev/ztimer_core/convert_frac.o
 .debug_abbrev  0x000000000000dba5      0x2ec /home/ch/RIOT/examples/lorawan/bin/lora-e5-dev/ztimer_core/convert.o
 .debug_abbrev  0x000000000000de91      0x537 /home/ch/RIOT/examples/lorawan/bin/lora-e5-dev/ztimer_core/core.o
 .debug_abbrev  0x000000000000e3c8      0x2e6 /home/ch/RIOT/examples/lorawan/bin/lora-e5-dev/ztimer_core/init.o
 .debug_abbrev  0x000000000000e6ae      0x3ef /home/ch/RIOT/examples/lorawan/bin/lora-e5-dev/ztimer_core/periph_rtt.o
 .debug_abbrev  0x000000000000ea9d      0x3a9 /home/ch/RIOT/examples/lorawan/bin/lora-e5-dev/ztimer_core/periph_timer.o
 .debug_abbrev  0x000000000000ee46      0x4b6 /home/ch/RIOT/examples/lorawan/bin/lora-e5-dev/ztimer_core/util.o
 .debug_abbrev  0x000000000000f2fc      0x264 /usr/lib/gcc/arm-none-eabi/9.2.1/../../../arm-none-eabi/lib/thumb/v7e-m/nofp/libm.a(lib_a-s_ceil.o)
 .debug_abbrev  0x000000000000f560      0x264 /usr/lib/gcc/arm-none-eabi/9.2.1/../../../arm-none-eabi/lib/thumb/v7e-m/nofp/libm.a(lib_a-s_floor.o)
 .debug_abbrev  0x000000000000f7c4       0x14 /usr/lib/gcc/arm-none-eabi/9.2.1/thumb/v7e-m/nofp/libgcc.a(_arm_addsubdf3.o)
 .debug_abbrev  0x000000000000f7d8       0x14 /usr/lib/gcc/arm-none-eabi/9.2.1/thumb/v7e-m/nofp/libgcc.a(_arm_muldivdf3.o)
 .debug_abbrev  0x000000000000f7ec       0x14 /usr/lib/gcc/arm-none-eabi/9.2.1/thumb/v7e-m/nofp/libgcc.a(_arm_cmpdf2.o)
 .debug_abbrev  0x000000000000f800       0x14 /usr/lib/gcc/arm-none-eabi/9.2.1/thumb/v7e-m/nofp/libgcc.a(_arm_fixdfsi.o)
 .debug_abbrev  0x000000000000f814       0x14 /usr/lib/gcc/arm-none-eabi/9.2.1/thumb/v7e-m/nofp/libgcc.a(_arm_fixunsdfsi.o)
 .debug_abbrev  0x000000000000f828       0x14 /usr/lib/gcc/arm-none-eabi/9.2.1/thumb/v7e-m/nofp/libgcc.a(_arm_addsubsf3.o)
 .debug_abbrev  0x000000000000f83c      0x17a /usr/lib/gcc/arm-none-eabi/9.2.1/../../../arm-none-eabi/lib/thumb/v7e-m/nofp/libc_nano.a(lib_a-impure.o)
 .debug_abbrev  0x000000000000f9b6       0xcc /usr/lib/gcc/arm-none-eabi/9.2.1/../../../arm-none-eabi/lib/thumb/v7e-m/nofp/libc_nano.a(lib_a-init.o)
 .debug_abbrev  0x000000000000fa82      0x1f2 /usr/lib/gcc/arm-none-eabi/9.2.1/../../../arm-none-eabi/lib/thumb/v7e-m/nofp/libc_nano.a(lib_a-malloc.o)
 .debug_abbrev  0x000000000000fc74       0x14 /usr/lib/gcc/arm-none-eabi/9.2.1/../../../arm-none-eabi/lib/thumb/v7e-m/nofp/libc_nano.a(lib_a-memcpy.o)
 .debug_abbrev  0x000000000000fc88      0x1de /usr/lib/gcc/arm-none-eabi/9.2.1/../../../arm-none-eabi/lib/thumb/v7e-m/nofp/libc_nano.a(lib_a-memmove.o)
 .debug_abbrev  0x000000000000fe66      0x1d9 /usr/lib/gcc/arm-none-eabi/9.2.1/../../../arm-none-eabi/lib/thumb/v7e-m/nofp/libc_nano.a(lib_a-memset.o)
 .debug_abbrev  0x000000000001003f      0x286 /usr/lib/gcc/arm-none-eabi/9.2.1/../../../arm-none-eabi/lib/thumb/v7e-m/nofp/libc_nano.a(lib_a-nano-freer.o)
 .debug_abbrev  0x00000000000102c5      0x2d1 /usr/lib/gcc/arm-none-eabi/9.2.1/../../../arm-none-eabi/lib/thumb/v7e-m/nofp/libc_nano.a(lib_a-nano-mallocr.o)
 .debug_abbrev  0x0000000000010596      0x351 /usr/lib/gcc/arm-none-eabi/9.2.1/../../../arm-none-eabi/lib/thumb/v7e-m/nofp/libc_nano.a(lib_a-nano-vfprintf_float.o)
 .debug_abbrev  0x00000000000108e7      0x2dc /usr/lib/gcc/arm-none-eabi/9.2.1/../../../arm-none-eabi/lib/thumb/v7e-m/nofp/libc_nano.a(lib_a-nano-vfprintf_i.o)
 .debug_abbrev  0x0000000000010bc3      0x29f /usr/lib/gcc/arm-none-eabi/9.2.1/../../../arm-none-eabi/lib/thumb/v7e-m/nofp/libc_nano.a(lib_a-printf.o)
 .debug_abbrev  0x0000000000010e62      0x2de /usr/lib/gcc/arm-none-eabi/9.2.1/../../../arm-none-eabi/lib/thumb/v7e-m/nofp/libc_nano.a(lib_a-puts.o)
 .debug_abbrev  0x0000000000011140       0x14 /usr/lib/gcc/arm-none-eabi/9.2.1/../../../arm-none-eabi/lib/thumb/v7e-m/nofp/libc_nano.a(lib_a-strlen.o)
 .debug_abbrev  0x0000000000011154      0x285 /usr/lib/gcc/arm-none-eabi/9.2.1/../../../arm-none-eabi/lib/thumb/v7e-m/nofp/libc_nano.a(lib_a-wbuf.o)
 .debug_abbrev  0x00000000000113d9      0x23a /usr/lib/gcc/arm-none-eabi/9.2.1/../../../arm-none-eabi/lib/thumb/v7e-m/nofp/libc_nano.a(lib_a-wsetup.o)
 .debug_abbrev  0x0000000000011613      0x310 /usr/lib/gcc/arm-none-eabi/9.2.1/../../../arm-none-eabi/lib/thumb/v7e-m/nofp/libc_nano.a(lib_a-dtoa.o)
 .debug_abbrev  0x0000000000011923      0x2e4 /usr/lib/gcc/arm-none-eabi/9.2.1/../../../arm-none-eabi/lib/thumb/v7e-m/nofp/libc_nano.a(lib_a-fflush.o)
 .debug_abbrev  0x0000000000011c07      0x3dc /usr/lib/gcc/arm-none-eabi/9.2.1/../../../arm-none-eabi/lib/thumb/v7e-m/nofp/libc_nano.a(lib_a-findfp.o)
 .debug_abbrev  0x0000000000011fe3      0x23c /usr/lib/gcc/arm-none-eabi/9.2.1/../../../arm-none-eabi/lib/thumb/v7e-m/nofp/libc_nano.a(lib_a-fprintf.o)
 .debug_abbrev  0x000000000001221f      0x210 /usr/lib/gcc/arm-none-eabi/9.2.1/../../../arm-none-eabi/lib/thumb/v7e-m/nofp/libc_nano.a(lib_a-fwalk.o)
 .debug_abbrev  0x000000000001242f      0x23f /usr/lib/gcc/arm-none-eabi/9.2.1/../../../arm-none-eabi/lib/thumb/v7e-m/nofp/libc_nano.a(lib_a-localeconv.o)
 .debug_abbrev  0x000000000001266e      0x2f6 /usr/lib/gcc/arm-none-eabi/9.2.1/../../../arm-none-eabi/lib/thumb/v7e-m/nofp/libc_nano.a(lib_a-makebuf.o)
 .debug_abbrev  0x0000000000012964       0x14 /usr/lib/gcc/arm-none-eabi/9.2.1/../../../arm-none-eabi/lib/thumb/v7e-m/nofp/libc_nano.a(lib_a-memchr.o)
 .debug_abbrev  0x0000000000012978      0x1c5 /usr/lib/gcc/arm-none-eabi/9.2.1/../../../arm-none-eabi/lib/thumb/v7e-m/nofp/libc_nano.a(lib_a-mlock.o)
 .debug_abbrev  0x0000000000012b3d      0x474 /usr/lib/gcc/arm-none-eabi/9.2.1/../../../arm-none-eabi/lib/thumb/v7e-m/nofp/libc_nano.a(lib_a-mprec.o)
 .debug_abbrev  0x0000000000012fb1      0x20d /usr/lib/gcc/arm-none-eabi/9.2.1/../../../arm-none-eabi/lib/thumb/v7e-m/nofp/libc_nano.a(lib_a-nano-callocr.o)
 .debug_abbrev  0x00000000000131be      0x22a /usr/lib/gcc/arm-none-eabi/9.2.1/../../../arm-none-eabi/lib/thumb/v7e-m/nofp/libc_nano.a(lib_a-nano-reallocr.o)
 .debug_abbrev  0x00000000000133e8      0x337 /usr/lib/gcc/arm-none-eabi/9.2.1/../../../arm-none-eabi/lib/thumb/v7e-m/nofp/libc_nano.a(lib_a-nano-vfprintf.o)
 .debug_abbrev  0x000000000001371f      0x26f /usr/lib/gcc/arm-none-eabi/9.2.1/../../../arm-none-eabi/lib/thumb/v7e-m/nofp/libc_nano.a(lib_a-stdio.o)
 .debug_abbrev  0x000000000001398e      0x1ff /usr/lib/gcc/arm-none-eabi/9.2.1/../../../arm-none-eabi/lib/thumb/v7e-m/nofp/libc_nano.a(lib_a-assert.o)
 .debug_abbrev  0x0000000000013b8d      0x270 /usr/lib/gcc/arm-none-eabi/9.2.1/../../../arm-none-eabi/lib/thumb/v7e-m/nofp/libc_nano.a(lib_a-fvwrite.o)
 .debug_abbrev  0x0000000000013dfd      0x2aa /usr/lib/gcc/arm-none-eabi/9.2.1/../../../arm-none-eabi/lib/thumb/v7e-m/nofp/libc_nano.a(lib_a-locale.o)
 .debug_abbrev  0x00000000000140a7      0x221 /usr/lib/gcc/arm-none-eabi/9.2.1/../../../arm-none-eabi/lib/thumb/v7e-m/nofp/libc_nano.a(lib_a-mbtowc_r.o)
 .debug_abbrev  0x00000000000142c8      0x1e5 /usr/lib/gcc/arm-none-eabi/9.2.1/../../../arm-none-eabi/lib/thumb/v7e-m/nofp/libc_nano.a(lib_a-nano-msizer.o)
 .debug_abbrev  0x00000000000144ad      0x22b /usr/lib/gcc/arm-none-eabi/9.2.1/../../../arm-none-eabi/lib/thumb/v7e-m/nofp/libc_nano.a(lib_a-wctomb_r.o)
 .debug_abbrev  0x00000000000146d8      0x1cd /usr/lib/gcc/arm-none-eabi/9.2.1/../../../arm-none-eabi/lib/thumb/v7e-m/nofp/libc_nano.a(lib_a-abort.o)
 .debug_abbrev  0x00000000000148a5      0x178 /usr/lib/gcc/arm-none-eabi/9.2.1/../../../arm-none-eabi/lib/thumb/v7e-m/nofp/libc_nano.a(lib_a-ctype_.o)
 .debug_abbrev  0x0000000000014a1d      0x32d /usr/lib/gcc/arm-none-eabi/9.2.1/../../../arm-none-eabi/lib/thumb/v7e-m/nofp/libc_nano.a(lib_a-signal.o)
 .debug_abbrev  0x0000000000014d4a       0x14 /usr/lib/gcc/arm-none-eabi/9.2.1/thumb/v7e-m/nofp/libgcc.a(_arm_unorddf2.o)

.debug_loc      0x0000000000000000    0x23f39
 .debug_loc     0x0000000000000000       0x89 /home/ch/RIOT/examples/lorawan/bin/lora-e5-dev/application_lorawan/main.o
 .debug_loc     0x0000000000000089       0xe8 /home/ch/RIOT/examples/lorawan/bin/lora-e5-dev/board/board.o
 .debug_loc     0x0000000000000171       0x4f /home/ch/RIOT/examples/lorawan/bin/lora-e5-dev/core/init.o
 .debug_loc     0x00000000000001c0     0x13c3 /home/ch/RIOT/examples/lorawan/bin/lora-e5-dev/core/msg.o
 .debug_loc     0x0000000000001583      0x7d2 /home/ch/RIOT/examples/lorawan/bin/lora-e5-dev/core/mutex.o
 .debug_loc     0x0000000000001d55       0x86 /home/ch/RIOT/examples/lorawan/bin/lora-e5-dev/core/panic.o
 .debug_loc     0x0000000000001ddb      0x2ca /home/ch/RIOT/examples/lorawan/bin/lora-e5-dev/core/sched.o
 .debug_loc     0x00000000000020a5      0xb20 /home/ch/RIOT/examples/lorawan/bin/lora-e5-dev/core/thread.o
 .debug_loc     0x0000000000002bc5      0x194 /home/ch/RIOT/examples/lorawan/bin/lora-e5-dev/cortexm_common/cortexm_init.o
 .debug_loc     0x0000000000002d59       0x63 /home/ch/RIOT/examples/lorawan/bin/lora-e5-dev/cortexm_common/panic.o
 .debug_loc     0x0000000000002dbc      0x243 /home/ch/RIOT/examples/lorawan/bin/lora-e5-dev/cortexm_common/thread_arch.o
 .debug_loc     0x0000000000002fff      0x443 /home/ch/RIOT/examples/lorawan/bin/lora-e5-dev/cortexm_common/vectors_cortexm.o
 .debug_loc     0x0000000000003442      0x22f /home/ch/RIOT/examples/lorawan/bin/lora-e5-dev/cpu/cpu_common.o
 .debug_loc     0x0000000000003671       0x2a /home/ch/RIOT/examples/lorawan/bin/lora-e5-dev/cpu/cpu_init.o
 .debug_loc     0x000000000000369b      0xc88 /home/ch/RIOT/examples/lorawan/bin/lora-e5-dev/crypto/aes.o
 .debug_loc     0x0000000000004323      0x5b4 /home/ch/RIOT/examples/lorawan/bin/lora-e5-dev/driver_sx126x_hal/driver_sx126x_hal.o
 .debug_loc     0x00000000000048d7     0x20fe /home/ch/RIOT/examples/lorawan/bin/lora-e5-dev/driver_sx126x/sx126x.o
 .debug_loc     0x00000000000069d5     0x19ef /home/ch/RIOT/examples/lorawan/bin/lora-e5-dev/fmt/fmt.o
 .debug_loc     0x00000000000083c4      0x5bf /home/ch/RIOT/examples/lorawan/bin/lora-e5-dev/frac/frac.o
 .debug_loc     0x0000000000008983      0x537 /home/ch/RIOT/examples/lorawan/bin/lora-e5-dev/luid/luid.o
 .debug_loc     0x0000000000008eba      0x2cc /home/ch/RIOT/examples/lorawan/bin/lora-e5-dev/malloc_thread_safe/malloc_wrappers.o
 .debug_loc     0x0000000000009186      0x734 /home/ch/RIOT/examples/lorawan/bin/lora-e5-dev/newlib_syscalls_default/syscalls.o
 .debug_loc     0x00000000000098ba       0x4f /home/ch/RIOT/examples/lorawan/bin/lora-e5-dev/periph_common/cpuid.o
 .debug_loc     0x0000000000009909       0x80 /home/ch/RIOT/examples/lorawan/bin/lora-e5-dev/periph_common/init.o
 .debug_loc     0x0000000000009989      0x10e /home/ch/RIOT/examples/lorawan/bin/lora-e5-dev/periph_common/timer.o
 .debug_loc     0x0000000000009a97      0x764 /home/ch/RIOT/examples/lorawan/bin/lora-e5-dev/periph/gpio_all.o
 .debug_loc     0x000000000000a1fb      0xf06 /home/ch/RIOT/examples/lorawan/bin/lora-e5-dev/periph/i2c_1.o
 .debug_loc     0x000000000000b101      0x143 /home/ch/RIOT/examples/lorawan/bin/lora-e5-dev/periph/pm.o
 .debug_loc     0x000000000000b244      0x268 /home/ch/RIOT/examples/lorawan/bin/lora-e5-dev/periph/rtt_all.o
 .debug_loc     0x000000000000b4ac      0x979 /home/ch/RIOT/examples/lorawan/bin/lora-e5-dev/periph/spi.o
 .debug_loc     0x000000000000be25      0x432 /home/ch/RIOT/examples/lorawan/bin/lora-e5-dev/periph/timer.o
 .debug_loc     0x000000000000c257      0x52e /home/ch/RIOT/examples/lorawan/bin/lora-e5-dev/periph/uart.o
 .debug_loc     0x000000000000c785      0x26c /home/ch/RIOT/examples/lorawan/bin/lora-e5-dev/pm_layered/pm.o
 .debug_loc     0x000000000000c9f1       0x24 /home/ch/RIOT/examples/lorawan/bin/lora-e5-dev/random/musl_lcg.o
 .debug_loc     0x000000000000ca15      0x261 /home/ch/RIOT/examples/lorawan/bin/lora-e5-dev/random/random.o
 .debug_loc     0x000000000000cc76      0x242 /home/ch/RIOT/examples/lorawan/bin/lora-e5-dev/semtech_loramac_arch/utilities.o
 .debug_loc     0x000000000000ceb8      0xbfd /home/ch/RIOT/examples/lorawan/bin/lora-e5-dev/semtech_loramac_contrib/semtech_loramac_getset.o
 .debug_loc     0x000000000000dab5      0x843 /home/ch/RIOT/examples/lorawan/bin/lora-e5-dev/semtech_loramac_contrib/semtech_loramac.o
 .debug_loc     0x000000000000e2f8      0x843 /home/ch/RIOT/examples/lorawan/bin/lora-e5-dev/semtech_loramac_contrib/semtech_loramac_radio.o
 .debug_loc     0x000000000000eb3b      0x301 /home/ch/RIOT/examples/lorawan/bin/lora-e5-dev/semtech_loramac_contrib/semtech_loramac_timer.o
 .debug_loc     0x000000000000ee3c      0x1ef /home/ch/RIOT/examples/lorawan/bin/lora-e5-dev/semtech_loramac_crypto/cmac.o
 .debug_loc     0x000000000000f02b      0x729 /home/ch/RIOT/examples/lorawan/bin/lora-e5-dev/semtech_loramac_mac/LoRaMacCrypto.o
 .debug_loc     0x000000000000f754     0x2ca7 /home/ch/RIOT/examples/lorawan/bin/lora-e5-dev/semtech_loramac_mac/LoRaMac.o
 .debug_loc     0x00000000000123fb      0xb65 /home/ch/RIOT/examples/lorawan/bin/lora-e5-dev/semtech_loramac_mac_region/RegionCommon.o
 .debug_loc     0x0000000000012f60     0x16bd /home/ch/RIOT/examples/lorawan/bin/lora-e5-dev/semtech_loramac_mac_region/RegionEU868.o
 .debug_loc     0x000000000001461d      0xdf7 /home/ch/RIOT/examples/lorawan/bin/lora-e5-dev/semtech_loramac_mac_region/Region.o
 .debug_loc     0x0000000000015414       0xb0 /home/ch/RIOT/examples/lorawan/bin/lora-e5-dev/stdio_uart/stdio_uart.o
 .debug_loc     0x00000000000154c4       0x2a /home/ch/RIOT/examples/lorawan/bin/lora-e5-dev/stm32_clk/stmclk_common.o
 .debug_loc     0x00000000000154ee       0x93 /home/ch/RIOT/examples/lorawan/bin/lora-e5-dev/stm32_clk/stmclk_l4wx.o
 .debug_loc     0x0000000000015581     0x12a5 /home/ch/RIOT/examples/lorawan/bin/lora-e5-dev/sx126x/sx126x_netdev.o
 .debug_loc     0x0000000000016826      0x5b9 /home/ch/RIOT/examples/lorawan/bin/lora-e5-dev/sx126x/sx126x.o
 .debug_loc     0x0000000000016ddf      0x733 /home/ch/RIOT/examples/lorawan/bin/lora-e5-dev/xtimer/xtimer_core.o
 .debug_loc     0x0000000000017512      0x42b /home/ch/RIOT/examples/lorawan/bin/lora-e5-dev/ztimer_core/convert_frac.o
 .debug_loc     0x000000000001793d      0x159 /home/ch/RIOT/examples/lorawan/bin/lora-e5-dev/ztimer_core/convert.o
 .debug_loc     0x0000000000017a96      0x98c /home/ch/RIOT/examples/lorawan/bin/lora-e5-dev/ztimer_core/core.o
 .debug_loc     0x0000000000018422       0x2a /home/ch/RIOT/examples/lorawan/bin/lora-e5-dev/ztimer_core/init.o
 .debug_loc     0x000000000001844c      0x258 /home/ch/RIOT/examples/lorawan/bin/lora-e5-dev/ztimer_core/periph_rtt.o
 .debug_loc     0x00000000000186a4      0x3b1 /home/ch/RIOT/examples/lorawan/bin/lora-e5-dev/ztimer_core/periph_timer.o
 .debug_loc     0x0000000000018a55      0x9b3 /home/ch/RIOT/examples/lorawan/bin/lora-e5-dev/ztimer_core/util.o
